******************************************************************************
                  TI ARM Linker PC v16.9.6                     
******************************************************************************
>> Linked Wed Jan 31 15:35:56 2018

OUTPUT FILE NAME:   <uart_emulator_launchpad_tirtos.out>
ENTRY POINT SYMBOL: "ResetISR"  address: 00004161


MEMORY CONFIGURATION

         name            origin    length      used     unused   attr    fill
----------------------  --------  ---------  --------  --------  ----  --------
  FLASH                 00000000   00020000  00004f40  0001b0c0  R  X
  GPRAM                 11000000   00002000  00000000  00002000  RW X
  SRAM                  20000000   00005000  00002290  00002d70  RW X


SEGMENT ALLOCATION MAP

run origin  load origin   length   init length attrs members
----------  ----------- ---------- ----------- ----- -------
00000000    00000000    000009c4   000009c4    r--
  00000000    00000000    0000003c   0000003c    r-- .resetVecs
  0000003c    0000003c    000006f8   000006f8    r-- .const
  00000738    00000738    0000028c   0000028c    r-- .cinit
00001000    00001000    0000452c   0000452c    r-x
  00001000    00001000    00000028   00000028    r-- .const:ti_sysbios_heaps_HeapMem_Module__FXNS__C
  00001028    00001028    00000024   00000024    r-- .const:ti_sysbios_gates_GateHwi_Module__FXNS__C
  0000104c    0000104c    00000024   00000024    r-- .const:ti_sysbios_gates_GateMutex_Module__FXNS__C
  00001070    00001070    00000020   00000020    r-- .const:ti_sysbios_family_arm_m3_Hwi_Object__DESC__C
  00001090    00001090    00000020   00000020    r-- .const:ti_sysbios_gates_GateHwi_Object__DESC__C
  000010b0    000010b0    00000020   00000020    r-- .const:ti_sysbios_gates_GateMutex_Object__DESC__C
  000010d0    000010d0    00000020   00000020    r-- .const:ti_sysbios_hal_Hwi_Object__DESC__C
  000010f0    000010f0    00000020   00000020    r-- .const:ti_sysbios_heaps_HeapMem_Object__DESC__C
  00001110    00001110    00000020   00000020    r-- .const:ti_sysbios_knl_Clock_Object__DESC__C
  00001130    00001130    00000020   00000020    r-- .const:ti_sysbios_knl_Event_Object__DESC__C
  00001150    00001150    00000020   00000020    r-- .const:ti_sysbios_knl_Mailbox_Object__DESC__C
  00001170    00001170    00000020   00000020    r-- .const:ti_sysbios_knl_Queue_Object__DESC__C
  00001190    00001190    00000020   00000020    r-- .const:ti_sysbios_knl_Semaphore_Object__DESC__C
  000011b0    000011b0    00000020   00000020    r-- .const:ti_sysbios_knl_Swi_Object__DESC__C
  000011d0    000011d0    00000020   00000020    r-- .const:ti_sysbios_knl_Task_Object__DESC__C
  000011f0    000011f0    00000008   00000008    r-- .const:ti_sysbios_knl_Idle_funcList__C
  000011f8    000011f8    00000004   00000004    r-- .const:ti_sysbios_family_arm_cc26xx_Timer_startupNeeded__C
  000011fc    000011fc    00000004   00000004    r-- .const:ti_sysbios_family_arm_m3_Hwi_E_alreadyDefined__C
  00001200    00001200    00000004   00000004    r-- .const:ti_sysbios_family_arm_m3_Hwi_E_hwiLimitExceeded__C
  00001204    00001204    00000004   00000004    r-- .const:ti_sysbios_family_arm_m3_Hwi_NUM_INTERRUPTS__C
  00001208    00001208    00000004   00000004    r-- .const:ti_sysbios_family_arm_m3_Hwi_Object__count__C
  0000120c    0000120c    00000004   00000004    r-- .const:ti_sysbios_family_arm_m3_Hwi_Object__table__C
  00001210    00001210    00000004   00000004    r-- .const:ti_sysbios_family_arm_m3_Hwi_ccr__C
  00001214    00001214    00000004   00000004    r-- .const:ti_sysbios_family_arm_m3_Hwi_excHandlerFunc__C
  00001218    00001218    00000004   00000004    r-- .const:ti_sysbios_family_arm_m3_Hwi_nullIsrFunc__C
  0000121c    0000121c    00000004   00000004    r-- .const:ti_sysbios_family_arm_m3_Hwi_numSparseInterrupts__C
  00001220    00001220    00000004   00000004    r-- .const:ti_sysbios_family_arm_m3_Hwi_priGroup__C
  00001224    00001224    00000004   00000004    r-- .const:ti_sysbios_family_arm_m3_TaskSupport_stackAlignment__C
  00001228    00001228    00000004   00000004    r-- .const:ti_sysbios_heaps_HeapMem_E_memory__C
  0000122c    0000122c    00000004   00000004    r-- .const:ti_sysbios_heaps_HeapMem_Module__gateObj__C
  00001230    00001230    00000004   00000004    r-- .const:ti_sysbios_heaps_HeapMem_Object__count__C
  00001234    00001234    00000004   00000004    r-- .const:ti_sysbios_heaps_HeapMem_Object__table__C
  00001238    00001238    00000004   00000004    r-- .const:ti_sysbios_heaps_HeapMem_reqAlign__C
  0000123c    0000123c    00000004   00000004    r-- .const:ti_sysbios_knl_Clock_triggerClock__C
  00001240    00001240    00000004   00000004    r-- .const:ti_sysbios_knl_Mailbox_Object__count__C
  00001244    00001244    00000004   00000004    r-- .const:ti_sysbios_knl_Mailbox_Object__table__C
  00001248    00001248    00000004   00000004    r-- .const:ti_sysbios_knl_Mailbox_maxTypeAlign__C
  0000124c    0000124c    00000004   00000004    r-- .const:ti_sysbios_knl_Queue_Object__count__C
  00001250    00001250    00000004   00000004    r-- .const:ti_sysbios_knl_Queue_Object__table__C
  00001254    00001254    00000004   00000004    r-- .const:ti_sysbios_knl_Semaphore_eventPost__C
  00001258    00001258    00000004   00000004    r-- .const:ti_sysbios_knl_Semaphore_eventSync__C
  0000125c    0000125c    00000004   00000004    r-- .const:ti_sysbios_knl_Swi_Object__count__C
  00001260    00001260    00000004   00000004    r-- .const:ti_sysbios_knl_Swi_Object__table__C
  00001264    00001264    00000004   00000004    r-- .const:ti_sysbios_knl_Swi_numPriorities__C
  00001268    00001268    00000004   00000004    r-- .const:ti_sysbios_knl_Task_Object__count__C
  0000126c    0000126c    00000004   00000004    r-- .const:ti_sysbios_knl_Task_Object__table__C
  00001270    00001270    00000004   00000004    r-- .const:ti_sysbios_knl_Task_allBlockedFunc__C
  00001274    00001274    00000004   00000004    r-- .const:ti_sysbios_knl_Task_defaultStackHeap__C
  00001278    00001278    00000004   00000004    r-- .const:ti_sysbios_knl_Task_defaultStackSize__C
  0000127c    0000127c    00000004   00000004    r-- .const:ti_sysbios_knl_Task_numConstructedTasks__C
  00001280    00001280    00000002   00000002    r-- .const:ti_sysbios_family_arm_cc26xx_Timer_Module__id__C
  00001282    00001282    00000002   00000002    r-- .const:ti_sysbios_family_arm_cc26xx_TimestampProvider_useClockTimer__C
  00001284    00001284    00000002   00000002    r-- .const:ti_sysbios_family_arm_m3_Hwi_Module__id__C
  00001286    00001286    00000002   00000002    r-- .const:ti_sysbios_gates_GateHwi_Module__id__C
  00001288    00001288    00000002   00000002    r-- .const:ti_sysbios_gates_GateMutex_Module__id__C
  0000128a    0000128a    00000002   00000002    r-- .const:ti_sysbios_heaps_HeapMem_Module__id__C
  0000128c    0000128c    00000002   00000002    r-- .const:ti_sysbios_knl_Task_initStackFlag__C
  0000128e    0000128e    00000001   00000001    r-- .const:ti_sysbios_knl_Clock_tickMode__C
  00001290    00001290    00000008   00000008    r-- .const:xdc_runtime_Startup_firstFxns__C
  00001298    00001298    00000008   00000008    r-- .const:xdc_runtime_Startup_lastFxns__C
  000012a0    000012a0    00000004   00000004    r-- .const:xdc_runtime_Assert_E_assertFailed__C
  000012a4    000012a4    00000004   00000004    r-- .const:xdc_runtime_Error_E_memory__C
  000012a8    000012a8    00000004   00000004    r-- .const:xdc_runtime_Error_policyFxn__C
  000012ac    000012ac    00000004   00000004    r-- .const:xdc_runtime_Error_raiseHook__C
  000012b0    000012b0    00000004   00000004    r-- .const:xdc_runtime_IGateProvider_Interface__BASE__C
  000012b4    000012b4    00000004   00000004    r-- .const:xdc_runtime_IHeap_Interface__BASE__C
  000012b8    000012b8    00000004   00000004    r-- .const:xdc_runtime_IModule_Interface__BASE__C
  000012bc    000012bc    00000004   00000004    r-- .const:xdc_runtime_Memory_defaultHeapInstance__C
  000012c0    000012c0    00000004   00000004    r-- .const:xdc_runtime_Startup_execImpl__C
  000012c4    000012c4    00000004   00000004    r-- .const:xdc_runtime_Startup_maxPasses__C
  000012c8    000012c8    00000004   00000004    r-- .const:xdc_runtime_Startup_sfxnRts__C
  000012cc    000012cc    00000004   00000004    r-- .const:xdc_runtime_Startup_sfxnTab__C
  000012d0    000012d0    00000004   00000004    r-- .const:xdc_runtime_Startup_startModsFxn__C
  000012d4    000012d4    00000004   00000004    r-- .const:xdc_runtime_SysCallback_abortFxn__C
  000012d8    000012d8    00000004   00000004    r-- .const:xdc_runtime_SysCallback_exitFxn__C
  000012dc    000012dc    00000004   00000004    r-- .const:xdc_runtime_System_abortFxn__C
  000012e0    000012e0    00000004   00000004    r-- .const:xdc_runtime_System_exitFxn__C
  000012e4    000012e4    00000004   00000004    r-- .const:xdc_runtime_System_maxAtexitHandlers__C
  000012e8    000012e8    00000004   00000004    r-- .const:xdc_runtime_Text_charTab__C
  000012ec    000012ec    00000004   00000004    r-- .const:xdc_runtime_Text_nameEmpty__C
  000012f0    000012f0    00000004   00000004    r-- .const:xdc_runtime_Text_nameStatic__C
  000012f4    000012f4    00000004   00000004    r-- .const:xdc_runtime_Text_nameUnknown__C
  000012f8    000012f8    00000002   00000002    r-- .const:xdc_runtime_Error_maxDepth__C
  000012fa    000012fa    00000002   00000002    r-- .const:xdc_runtime_Memory_Module__id__C
  000012fc    000012fc    00000002   00000002    r-- .const:xdc_runtime_Text_charCnt__C
  000012fe    000012fe    00000002   00000002    r-- .const:xdc_runtime_Text_isLoaded__C
  00001300    00001300    00000001   00000001    r-- .const:xdc_runtime_Error_policy__C
  00001304    00001304    00000004   00000004    r-- .const:ti_sysbios_rom_ROM_ti_sysbios_family_arm_cc26xx_Timer_getCount64__E
  00001308    00001308    00000004   00000004    r-- .const:ti_sysbios_rom_ROM_ti_sysbios_family_arm_cc26xx_Timer_getCurrentTick__E
  0000130c    0000130c    00000004   00000004    r-- .const:ti_sysbios_rom_ROM_ti_sysbios_family_arm_cc26xx_Timer_getMaxTicks__E
  00001310    00001310    00000004   00000004    r-- .const:ti_sysbios_rom_ROM_ti_sysbios_family_arm_cc26xx_Timer_initDevice__I
  00001314    00001314    00000004   00000004    r-- .const:ti_sysbios_rom_ROM_ti_sysbios_family_arm_cc26xx_Timer_setNextTick__E
  00001318    00001318    00000004   00000004    r-- .const:ti_sysbios_rom_ROM_ti_sysbios_family_arm_cc26xx_Timer_setThreshold__I
  0000131c    0000131c    00000004   00000004    r-- .const:ti_sysbios_rom_ROM_ti_sysbios_family_arm_cc26xx_Timer_start__E
  00001320    00001320    00000004   00000004    r-- .const:ti_sysbios_rom_ROM_ti_sysbios_family_arm_cc26xx_TimestampProvider_get32__E
  00001324    00001324    00000004   00000004    r-- .const:ti_sysbios_rom_ROM_xdc_runtime_Startup_getState__I
  00001328    00001328    00000004   00000004    r-- .const:ti_sysbios_rom_ROM_xdc_runtime_System_SupportProxy_abort__E
  0000132c    0000132c    00000004   00000004    r-- .const:ti_sysbios_rom_ROM_xdc_runtime_System_SupportProxy_exit__E
  00001330    00001330    000041fc   000041fc    r-x .text
0001ffa8    0001ffa8    00000058   00000058    r--
  0001ffa8    0001ffa8    00000058   00000058    r-- .ccfg
20000100    20000100    00001ecf   00000000    rw-
  20000100    20000100    00000044   00000000    rw- .data:ti_sysbios_knl_Task_Module__state__V
  20000144    20000144    00000034   00000000    rw- .data:ti_sysbios_family_arm_m3_Hwi_Module__state__V
  20000178    20000178    0000002c   00000000    rw- .data:ti_sysbios_knl_Clock_Module__state__V
  200001a4    200001a4    00000024   00000000    rw- .data:ti_sysbios_BIOS_Module__state__V
  200001c8    200001c8    0000001c   00000000    rw- .data:ti_sysbios_knl_Swi_Module__state__V
  200001e4    200001e4    00000008   00000000    rw- .data:ti_sysbios_family_arm_cc26xx_Timer_Module__state__V
  200001ec    200001ec    00000004   00000000    rw- .data:ti_sysbios_family_arm_cc26xx_TimestampProvider_Module__state__V
  200001f0    200001f0    00000008   00000000    rw- .data:xdc_runtime_Startup_Module__state__V
  200001f8    200001f8    00000008   00000000    rw- .data:xdc_runtime_System_Module__state__V
  20000200    20000200    00000004   00000000    rw- .data:xdc_runtime_Memory_Module__state__V
  20000204    20000204    00000002   00000000    rw- .data:xdc_runtime_Error_Module__state__V
  20000208    20000208    00001883   00000000    rw- .bss
  20001a90    20001a90    0000053f   00000000    rw- .data
20004d00    20004d00    00000300   00000000    rw-
  20004d00    20004d00    00000300   00000000    rw- .stack


SECTION ALLOCATION MAP

 output                                  attributes/
section   page    origin      length       input sections
--------  ----  ----------  ----------   ----------------
.binit     0    00000000    00000000     

.const     0    0000003c    000006f8     
                  0000003c    00000444     scif.obj (.const:pAuxRamImage)
                  00000480    0000004c     drivers_cc26x0r2.aem3 : PowerCC26XX.oem3 (.const:resourceDB)
                  000004cc    00000048     rom_pem3.oem3 (.const:.string)
                  00000514    00000040     drivers_cc26x0r2.aem3 : UARTCC26XX.oem3 (.const:$O1$$)
                  00000554    00000040                           : GPIOCC26XX.oem3 (.const:$O2$$)
                  00000594    00000030     scif.obj (.const:scifDriverSetup)
                  000005c4    0000002c     CC2640R2_LAUNCHXL.obj (.const:BoardGpioInitTable)
                  000005f0    00000028     drivers_cc26x0r2.aem3 : UARTCC26XX.oem3 (.const:UARTCC26XX_fxnTable)
                  00000618    00000028     rom_pem3.oem3 (.const:xdc_runtime_Startup_sfxnTab__A)
                  00000640    00000024     drivers_cc26x0r2.aem3 : UART.oem3 (.const:UART_defaultParams)
                  00000664    00000020     CC2640R2_LAUNCHXL.obj (.const:uartCC26XXHWAttrs)
                  00000684    00000018     CC2640R2_LAUNCHXL.obj (.const:PowerCC26XX_config)
                  0000069c    00000014     CC2640R2_LAUNCHXL.obj (.const:GPIOCC26XX_config)
                  000006b0    00000014     rom_pem3.oem3 (.const:xdc_runtime_Startup_sfxnRts__A)
                  000006c4    00000010     scif.obj (.const:.string:pAuxIoIndexToMcuIocfgOffsetLut)
                  000006d4    00000010     scif.obj (.const:pScifTaskDataStructInfoLut)
                  000006e4    0000000c     main_tirtos.obj (.const:BoardGpioInitTable1)
                  000006f0    0000000c     CC2640R2_LAUNCHXL.obj (.const:UART_config)
                  000006fc    0000000c     rom_pem3.oem3 (.const:xdc_runtime_Startup_firstFxns__A)
                  00000708    00000009     CC2640R2_LAUNCHXL.obj (.const)
                  00000711    00000001     rom_pem3.oem3 (.const:xdc_runtime_Text_charTab__A)
                  00000712    00000002     rom_pem3.oem3 (.const:xdc_runtime_SysMin_flushAtExit__C)
                  00000714    00000008     CC2640R2_LAUNCHXL.obj (.const:PINCC26XX_hwAttrs)
                  0000071c    00000004     rom_pem3.oem3 (.const:ti_sysbios_family_arm_m3_Hwi_swiDisable__C)
                  00000720    00000004     rom_pem3.oem3 (.const:ti_sysbios_family_arm_m3_Hwi_swiRestoreHwi__C)
                  00000724    00000004     rom_pem3.oem3 (.const:ti_sysbios_knl_Clock_tickPeriod__C)
                  00000728    00000004     rom_pem3.oem3 (.const:ti_sysbios_knl_Idle_funcList__A)
                  0000072c    00000004     rom_pem3.oem3 (.const:xdc_runtime_SysMin_bufSize__C)
                  00000730    00000004     rom_pem3.oem3 (.const:xdc_runtime_SysMin_outputFunc__C)

.text      0    00001330    000041fc     
                  00001330    00000314     drivers_cc26x0r2.aem3 : PowerCC26XX_calibrateRCOSC.oem3 (.text:PowerCC26XX_auxISR)
                  00001644    00000244                           : PowerCC26XX.oem3 (.text:Power_sleep)
                  00001888    0000020c     driverlib.lib : sys_ctrl.obj (.text:NOROM_SysCtrlSetRechargeBeforePowerDown)
                  00001a94    000001f4     rtsv7M3_T_le_eabi.lib : ull_div_t2.obj (.text)
                  00001c88    000001bc     drivers_cc26x0r2.aem3 : PINCC26XX.oem3 (.text:PIN_init)
                  00001e44    00000190                           : PowerCC26XX_calibrateRCOSC.oem3 (.text:PowerCC26XX_doCalibrate)
                  00001fd4    0000015c                           : UARTCC26XX.oem3 (.text:UARTCC26XX_open)
                  00002130    0000012c                           : PowerCC26XX.oem3 (.text:Power_init)
                  0000225c    0000011c                           : UARTCC26XX.oem3 (.text:UARTCC26XX_read)
                  00002378    00000112                           : UARTCC26XX.oem3 (.text:UARTCC26XX_hwiIntFxn)
                  0000248a    00000002                           : PowerCC26XX.oem3 (.text:emptyClockFunc)
                  0000248c    00000100     scif_framework.obj (.text:scifInit)
                  0000258c    000000fc     drivers_cc26x0r2.aem3 : UARTCC26XX.oem3 (.text:UARTCC26XX_write)
                  00002688    000000f0                           : GPIOCC26XX.oem3 (.text:GPIO_setConfig)
                  00002778    000000e8     dpl_cc26x0r2.aem3 : PowerCC26XX_tirtos.oem3 (.text:PowerCC26XX_standbyPolicy)
                  00002860    000000e0     scif_framework.obj (.text:scifCtrlTasksNbl)
                  00002940    000000dc     drivers_cc26x0r2.aem3 : PINCC26XX.oem3 (.text:PINCC26XX_setIoCfg)
                  00002a1c    000000bc                           : GPIOCC26XX.oem3 (.text:GPIO_init)
                  00002ad8    000000bc                           : PowerCC26XX.oem3 (.text:Power_releaseDependency)
                  00002b94    000000b4                           : PowerCC26XX.oem3 (.text:Power_setDependency)
                  00002c48    000000b0                           : UARTCC26XX.oem3 (.text:UARTCC26XX_initHw)
                  00002cf8    000000b0     rom_sysbios.aem3 : rom_sysbios.obj (.text:xdc_runtime_Error_policyDefault__E)
                  00002da8    000000ac     driverlib.lib : setup.obj (.text:NOROM_SetupTrimDevice)
                  00002e54    000000a4     drivers_cc26x0r2.aem3 : PowerCC26XX.oem3 (.text:switchXOSCHFclockFunc)
                  00002ef8    000000a0     auto_init.aem3 : auto_init.oem3 (.text)
                  00002f98    0000009c     rtsv7M3_T_le_eabi.lib : memcpy_t2.obj (.text)
                  00003034    00000098     drivers_cc26x0r2.aem3 : PINCC26XX.oem3 (.text:PIN_open)
                  000030cc    00000098                           : UARTCC26XX.oem3 (.text:UARTCC26XX_initIO)
                  00003164    00000098     rom_sysbios.aem3 : rom_sysbios.obj (.text:ti_sysbios_knl_Clock_workFuncDynamic__E)
                  000031fc    0000008c     driverlib.lib : setup.obj (.text:TrimAfterColdResetWakeupFromShutDown)
                  00003288    0000008c     drivers_cc26x0r2.aem3 : UARTCC26XX.oem3 (.text:UARTCC26XX_close)
                  00003314    0000008c                           : UARTCC26XX.oem3 (.text:UARTCC26XX_writeCancel)
                  000033a0    0000008c     scif_framework.obj (.text:scifInitIo)
                  0000342c    0000008c     drivers_cc26x0r2.aem3 : UARTCC26XX.oem3 (.text:writeFinishedDoCallback)
                  000034b8    00000080     main_tirtos.obj (.text:main)
                  00003538    0000007a     rtsv7M3_T_le_eabi.lib : memset_t2.obj (.text)
                  000035b2    00000078     drivers_cc26x0r2.aem3 : UARTCC26XX.oem3 (.text:writeTxFifoFlush)
                  0000362a    00000002     main_tirtos.obj (.text:scCtrlReadyCallback)
                  0000362c    00000074     scif.obj (.text:scifUartSetBaudRate)
                  000036a0    00000074     rom_sysbios.aem3 : rom_sysbios.obj (.text:ti_sysbios_family_arm_cc26xx_Timer_start__E)
                  00003714    00000070     driverlib.lib : sys_ctrl.obj (.text:NOROM_SysCtrlAdjustRechargeAfterPowerDown)
                  00003784    00000070     drivers_cc26x0r2.aem3 : PowerCC26XX.oem3 (.text:lfClockReadyCallback)
                  000037f4    0000006c     driverlib.lib : osc.obj (.text:NOROM_OSCHF_AttemptToSwitchToXosc)
                  00003860    0000006c     drivers_cc26x0r2.aem3 : PowerCC26XX_calibrateRCOSC.oem3 (.text:PowerCC26XX_initiateCalibration)
                  000038cc    0000006c                           : PowerCC26XX.oem3 (.text:configureXOSCHF)
                  00003938    00000068     driverlib.lib : sys_ctrl.obj (.text:NOROM_SysCtrl_DCDC_VoltageConditionalControl)
                  000039a0    00000068     drivers_cc26x0r2.aem3 : UARTCC26XX.oem3 (.text:UARTCC26XX_readCancel)
                  00003a08    00000068     rtsv7M3_T_le_eabi.lib : copy_decompress_lzss.obj (.text:decompress:lzss)
                  00003a70    00000068                           : trgmsg.obj (.text)
                  00003ad8    00000064     drivers_cc26x0r2.aem3 : PINCC26XX.oem3 (.text:PIN_add)
                  00003b3c    00000064     main_tirtos.obj (.text:taskFxn1)
                  00003ba0    0000005c     drivers_cc26x0r2.aem3 : PowerCC26XX_calibrateRCOSC.oem3 (.text:PowerCC26XX_RCOSC_clockFunc)
                  00003bfc    0000005c                           : PowerCC26XX.oem3 (.text:PowerCC26XX_calibrate)
                  00003c58    0000005c     rom_pem3.oem3 (.text:xdc_runtime_Startup_getState__I)
                  00003cb4    00000058     drivers_cc26x0r2.aem3 : PINCC26XX.oem3 (.text:PIN_remove)
                  00003d0c    00000058                           : UARTCC26XX.oem3 (.text:UARTCC26XX_control)
                  00003d64    00000058     rtsv7M3_T_le_eabi.lib : hostwrite.obj (.text)
                  00003dbc    00000058     scif_framework.obj (.text:scifReinitIo)
                  00003e14    00000058     scif_framework.obj (.text:scifUninitIo)
                  00003e6c    00000058     main_tirtos.obj (.text:taskFxn)
                  00003ec4    00000054     drivers_cc26x0r2.aem3 : GPIOCC26XX.oem3 (.text:GPIO_write)
                  00003f18    00000050                           : UARTCC26XX.oem3 (.text:startTxFifoEmptyClk)
                  00003f68    0000004c                           : GPIOCC26XX.oem3 (.text:powerPostNotify)
                  00003fb4    0000004c     rtsv7M3_T_le_eabi.lib : cpy_tbl.obj (.text)
                  00004000    00000048     dpl_cc26x0r2.aem3 : ClockP_tirtos.oem3 (.text:ClockP_construct)
                  00004048    00000048     drivers_cc26x0r2.aem3 : PINCC26XX.oem3 (.text:PIN_setOutputEnable)
                  00004090    00000048     rom_sysbios.aem3 : rom_sysbios.obj (.text:ti_sysbios_family_arm_cc26xx_Timer_setThreshold__I)
                  000040d8    00000044     driverlib.lib : osc.obj (.text:NOROM_OSCHF_SwitchToRcOscTurnOffXosc)
                  0000411c    00000044     drivers_cc26x0r2.aem3 : RingBuf.oem3 (.text:RingBuf_put)
                  00004160    00000044     boot.aem3 : boot.oem3 (.text)
                  000041a4    00000044     drivers_cc26x0r2.aem3 : PowerCC26XX.oem3 (.text:notify)
                  000041e8    00000044     rom_sysbios.aem3 : rom_sysbios.obj (.text:xdc_runtime_Error_setX__E)
                  0000422c    00000044                      : rom_sysbios.obj (.text:xdc_runtime_SysMin_flush__E)
                  00004270    00000040     drivers_cc26x0r2.aem3 : PINCC26XX.oem3 (.text:PIN_swi)
                  000042b0    00000040                           : UART.oem3 (.text:UART_init)
                  000042f0    00000040                           : UART.oem3 (.text:UART_open)
                  00004330    00000040     scif.obj (.text:scifUartGetRxFifoCount)
                  00004370    0000003e     dpl_cc26x0r2.aem3 : HwiP_tirtos.oem3 (.text:HwiP_construct)
                  000043ae    0000003e     drivers_cc26x0r2.aem3 : RingBuf.oem3 (.text:RingBuf_get)
                  000043ec    0000003c     driverlib.lib : osc.obj (.text:NOROM_OSC_HPOSCRelativeFrequencyOffsetGet)
                  00004428    0000003c     dpl_cc26x0r2.aem3 : SwiP_tirtos.oem3 (.text:SwiP_construct)
                  00004464    0000003c     drivers_cc26x0r2.aem3 : PowerCC26XX.oem3 (.text:disableLfClkQualifiersEnableClkLoss)
                  000044a0    0000003c     scif.obj (.text:scifUartRxGetChar)
                  000044dc    0000003c     scif.obj (.text:scifUartTxPutChar)
                  00004518    0000003c     rom_sysbios.aem3 : rom_sysbios.obj (.text:ti_sysbios_family_arm_m3_Hwi_construct2__E)
                  00004554    00000038     drivers_cc26x0r2.aem3 : GPIOCC26XX.oem3 (.text:GPIO_enableInt)
                  0000458c    00000038                           : PINCC26XX.oem3 (.text:PIN_setOutputValue)
                  000045c4    00000038                           : UARTCC26XX.oem3 (.text:UARTCC26XX_swiIntFxn)
                  000045fc    00000038     rom_sysbios.aem3 : rom_sysbios.obj (.text:ti_sysbios_family_arm_cc26xx_Timer_getCurrentTick__E)
                  00004634    00000038                      : rom_sysbios.obj (.text:xdc_runtime_SysMin_putch__E)
                  0000466c    00000034     drivers_cc26x0r2.aem3 : GPIOCC26XX.oem3 (.text:GPIO_setCallback)
                  000046a0    00000034                           : PINCC26XX.oem3 (.text:PIN_setConfig)
                  000046d4    00000034                           : PowerCC26XX.oem3 (.text:Power_releaseConstraint)
                  00004708    00000034     scif_framework.obj (.text:scifAckAlertEvents)
                  0000473c    00000034     scif_framework.obj (.text:scifOsalInit)
                  00004770    00000034     rom_sysbios.aem3 : rom_sysbios.obj (.text:ti_sysbios_family_arm_cc26xx_Timer_initDevice__I)
                  000047a4    00000032     main_tirtos.obj (.text:scTaskAlertCallback)
                  000047d6    00000032     rom_sysbios.aem3 : rom_sysbios.obj (.text:ti_sysbios_family_arm_cc26xx_Timer_setNextTick__E)
                  00004808    00000030     drivers_cc26x0r2.aem3 : PowerCC26XX.oem3 (.text:Power_setConstraint)
                  00004838    00000030     scif_framework.obj (.text:osalRegisterCtrlReadyInt)
                  00004868    00000030     scif_framework.obj (.text:osalRegisterTaskAlertInt)
                  00004898    00000030     rom_pem3.oem3 (.text:ti_sysbios_BIOS_atExitFunc__I)
                  000048c8    00000030     rom_pem3.oem3 (.text:ti_sysbios_BIOS_startFunc__I)
                  000048f8    00000030     rom_sysbios.aem3 : rom_sysbios.obj (.text:xdc_runtime_SysMin_abort__E)
                  00004928    0000002e     drivers_cc26x0r2.aem3 : UARTCC26XX.oem3 (.text:readData)
                  00004956    0000002e                           : UARTCC26XX.oem3 (.text:writeData)
                  00004984    0000002c     driverlib.lib : chipinfo.obj (.text:NOROM_ChipInfo_GetChipFamily)
                  000049b0    0000002c     drivers_cc26x0r2.aem3 : PINCC26XX.oem3 (.text:PINCC26XX_setMux)
                  000049dc    0000002c     dpl_cc26x0r2.aem3 : SemaphoreP_tirtos.oem3 (.text:SemaphoreP_constructBinary)
                  00004a08    0000002c                       : SemaphoreP_tirtos.oem3 (.text:SemaphoreP_createBinary)
                  00004a34    0000002c     scif_framework.obj (.text:osalIndicateCtrlReady)
                  00004a60    0000002c     scif_framework.obj (.text:osalLockCtrlTaskNbl)
                  00004a8c    0000002c     rom_sysbios.aem3 : rom_sysbios.obj (.text:ti_sysbios_knl_Clock_getTicksUntilInterrupt__E)
                  00004ab8    00000028     driverlib.lib : chipinfo.obj (.text:NOROM_ChipInfo_GetChipType)
                  00004ae0    00000028     drivers_cc26x0r2.aem3 : PowerCC26XX.oem3 (.text:Power_registerNotify)
                  00004b08    00000028     driverlib.lib : adi.obj (.text:SafeHapiVoid)
                  00004b30    00000028     drivers_cc26x0r2.aem3 : UARTCC26XX.oem3 (.text:readData2RingBuf)
                  00004b58    00000024                           : GPIOCC26XX.oem3 (.text:GPIO_hwiIntFxn)
                  00004b7c    00000024     driverlib.lib : osc.obj (.text:NOROM_OSCHF_TurnOnXosc)
                  00004ba0    00000024     main_tirtos.obj (.text:Uart_rxcallback)
                  00004bc4    00000024     scif.obj (.text:scifUartSetEventMask)
                  00004be8    00000024     rom_pem3.oem3 (.text:ti_sysbios_BIOS_registerRTSLock__I)
                  00004c0c    00000024     rom_pem3.oem3 (.text:ti_sysbios_BIOS_removeRTSLock__I)
                  00004c30    00000024     rom_sysbios.aem3 : rom_sysbios.obj (.text:ti_sysbios_family_arm_cc26xx_Timer_getMaxTicks__E)
                  00004c54    00000022     drivers_cc26x0r2.aem3 : List.oem3 (.text:List_put)
                  00004c76    00000022     driverlib.lib : uart.obj (.text:NOROM_UARTConfigSetExpClk)
                  00004c98    00000022     rom_pem3.oem3 (.text:xdc_runtime_SysMin_output__I)
                  00004cba    00000002     rom_pem3.oem3 (.text:ti_sysbios_BIOS_nullFunc__I)
                  00004cbc    00000020     driverlib.lib : uart.obj (.text:NOROM_UARTDisable)
                  00004cdc    00000020     dpl_cc26x0r2.aem3 : PowerCC26XX_tirtos.oem3 (.text:PowerCC26XX_schedulerDisable)
                  00004cfc    00000020                       : PowerCC26XX_tirtos.oem3 (.text:PowerCC26XX_schedulerRestore)
                  00004d1c    00000020     drivers_cc26x0r2.aem3 : PowerCC26XX.oem3 (.text:Power_unregisterNotify)
                  00004d3c    00000020     rom_pem3.oem3 (.text:ti_sysbios_BIOS_rtsLock__I)
                  00004d5c    00000020     rom_sysbios.aem3 : rom_sysbios.obj (.text:ti_sysbios_family_arm_cc26xx_Timer_dynamicStub__E)
                  00004d7c    00000020                      : rom_sysbios.obj (.text:xdc_runtime_SysMin_Module_startup__E)
                  00004d9c    0000001e     drivers_cc26x0r2.aem3 : PINCC26XX.oem3 (.text:PIN_close)
                  00004dba    0000001e                           : PowerCC26XX.oem3 (.text:Power_getTransitionLatency)
                  00004dd8    0000001e     scif.obj (.text:scifTaskResourceInit)
                  00004df6    00000002     rom_pem3.oem3 (.text:ti_sysbios_rom_cortexm_cc26xx_r2_CC26xx_badRomRevision__E)
                  00004df8    0000001c     drivers_cc26x0r2.aem3 : PINCC26XX.oem3 (.text:PINCC26XX_setIoCfgMux)
                  00004e14    0000001c                           : PINCC26XX.oem3 (.text:PIN_hwi)
                  00004e30    0000001c     rom_sysbios.aem3 : rom_sysbios.obj (.text:ti_sysbios_family_arm_m3_Hwi_clearInterrupt__E)
                  00004e4c    0000001c                      : rom_sysbios.obj (.text:ti_sysbios_knl_Swi_construct2__E)
                  00004e68    0000001c                      : rom_sysbios.obj (.text:xdc_runtime_SysMin_exit__E)
                  00004e84    00000018     driverlib.lib : chipinfo.obj (.text:NOROM_ChipInfo_GetPackageType)
                  00004e9c    00000018     drivers_cc26x0r2.aem3 : PowerCC26XX.oem3 (.text:Power_idleFunc)
                  00004eb4    00000018                           : UARTCC26XX.oem3 (.text:UARTCC26XX_init)
                  00004ecc    00000018                           : UART.oem3 (.text:UART_Params_init)
                  00004ee4    00000018                           : PowerCC26XX.oem3 (.text:configureRFCoreClocks)
                  00004efc    00000018     rtsv7M3_T_le_eabi.lib : args_main.obj (.text)
                  00004f14    00000018                           : ll_mul_t2.obj (.text)
                  00004f2c    00000018     scif_framework.obj (.text:scifClearAlertIntSource)
                  00004f44    00000018     scif.obj (.text:scifUartRxEnable)
                  00004f5c    00000018     scif.obj (.text:scifUartSetRxEnableReqIdleCount)
                  00004f74    00000018     scif.obj (.text:scifUartSetRxFifoThr)
                  00004f8c    00000018     scif.obj (.text:scifUartSetRxTimeout)
                  00004fa4    00000018     rom_pem3.oem3 (.text:ti_sysbios_BIOS_rtsUnlock__I)
                  00004fbc    00000018     rom_sysbios.aem3 : rom_sysbios.obj (.text:ti_sysbios_knl_Swi_or__E)
                  00004fd4    00000018     rom_pem3.oem3 (.text:ti_sysbios_rom_cortexm_cc26xx_r2_CC26xx_checkRevision__E)
                  00004fec    00000018     rom_sysbios.aem3 : rom_sysbios.obj (.text:xdc_runtime_Error_init__E)
                  00005004    00000016     drivers_cc26x0r2.aem3 : List.oem3 (.text:List_remove)
                  0000501a    00000016     rom_pem3.oem3 (.text:ti_sysbios_BIOS_errorRaiseHook__I)
                  00005030    00000016     rom_pem3.oem3 (.text:ti_sysbios_BIOS_exitFunc__I)
                  00005046    00000016     scif_framework.obj (.text:ti_sysbios_family_arm_m3_Hwi_Params_init)
                  0000505c    00000016     scif_framework.obj (.text:ti_sysbios_knl_Semaphore_Params_init)
                  00005072    00000016     main_tirtos.obj (.text:ti_sysbios_knl_Task_Params_init)
                  00005088    00000014     driverlib.lib : ioc.obj (.text:NOROM_IOCIntEnable)
                  0000509c    00000014     scif_framework.obj (.text:osalIndicateTaskAlert)
                  000050b0    00000014     rtsv7M3_T_le_eabi.lib : _lock.obj (.text)
                  000050c4    00000014     scif_framework.obj (.text:scifOsalRegisterCtrlReadyCallback)
                  000050d8    00000014     scif_framework.obj (.text:scifOsalRegisterTaskAlertCallback)
                  000050ec    00000014     scif.obj (.text:scifTaskResourceUninit)
                  00005100    00000014     rom_sysbios.aem3 : rom_sysbios.obj (.text:ti_sysbios_family_arm_cc26xx_Timer_getCount64__E)
                  00005114    00000014     rom_pem3.oem3 (.text:ti_sysbios_knl_Clock_doTick__I)
                  00005128    00000012     drivers_cc26x0r2.aem3 : RingBuf.oem3 (.text:RingBuf_construct)
                  0000513a    00000012     dpl_cc26x0r2.aem3 : SemaphoreP_tirtos.oem3 (.text:SemaphoreP_pend)
                  0000514c    00000012     scif_framework.obj (.text:scifExecuteTasksOnceNbl)
                  0000515e    00000012     rom_pem3.oem3 (.text:xdc_runtime_Startup_exec__I)
                  00005170    00000010     dpl_cc26x0r2.aem3 : HwiP_tirtos.oem3 (.text:HwiP_Params_init)
                  00005180    00000010     drivers_cc26x0r2.aem3 : PINCC26XX.oem3 (.text:PINCC26XX_getPinCount)
                  00005190    00000010     dpl_cc26x0r2.aem3 : SwiP_tirtos.oem3 (.text:SwiP_Params_init)
                  000051a0    00000010     drivers_cc26x0r2.aem3 : UARTCC26XX.oem3 (.text:uartPostNotify)
                  000051b0    0000000e     driverlib.lib : chipinfo.obj (.text:NOROM_ThisLibraryIsFor_CC26x0R2_HaltIfViolated)
                  000051be    0000000e                   : uart.obj (.text:NOROM_UARTCharGetNonBlocking)
                  000051cc    0000000e                   : uart.obj (.text:NOROM_UARTCharPutNonBlocking)
                  000051da    0000000e     rtsv7M3_T_le_eabi.lib : copy_decompress_none.obj (.text:decompress:none)
                  000051e8    0000000e     scif_framework.obj (.text:osalCtrlReadyIsr)
                  000051f6    0000000e     scif_framework.obj (.text:osalTaskAlertIsr)
                  00005204    0000000e     rom_sysbios.aem3 : rom_sysbios.obj (.text:ti_sysbios_family_arm_cc26xx_TimestampProvider_get32__E)
                  00005212    0000000c     drivers_cc26x0r2.aem3 : List.oem3 (.text:List_empty)
                  0000521e    0000000c     driverlib.lib : cpu.obj (.text:NOROM_CPUcpsid)
                  0000522a    0000000c                   : cpu.obj (.text:NOROM_CPUcpsie)
                  00005236    0000000c                   : osc.obj (.text:NOROM_OSC_HPOSCRelativeFrequencyOffsetToRFCoreFormatConvert)
                  00005242    0000000c     drivers_cc26x0r2.aem3 : PINCC26XX.oem3 (.text:PIN_registerIntCb)
                  0000524e    00000002     rom_sysbios.aem3 : rom_sysbios.obj (.text:xdc_runtime_SysCallback_defaultAbort)
                  00005250    0000000c     drivers_cc26x0r2.aem3 : PowerCC26XX.oem3 (.text:Power_getConstraintMask)
                  0000525c    0000000c                           : PowerCC26XX.oem3 (.text:Power_getDependencyCount)
                  00005268    0000000c     dpl_cc26x0r2.aem3 : SemaphoreP_tirtos.oem3 (.text:SemaphoreP_delete)
                  00005274    0000000c     rtsv7M3_T_le_eabi.lib : copy_zero_init.obj (.text:decompress:ZI)
                  00005280    0000000c     scif_framework.obj (.text:osalUnlockCtrlTaskNbl)
                  0000528c    0000000c     scif_framework.obj (.text:scifOsalLeaveCriticalSection)
                  00005298    0000000c     scif.obj (.text:scifUartClearEvents)
                  000052a4    0000000c     scif_framework.obj (.text:ti_sysbios_knl_Semaphore_handle)
                  000052b0    0000000c     rom_sysbios.aem3 : rom_sysbios.obj (.text:ti_sysbios_knl_Swi_getTrigger__E)
                  000052bc    0000000c     rom_pem3.oem3 (.text:xdc_runtime_Startup_reset__I)
                  000052c8    0000000a     drivers_cc26x0r2.aem3 : UART.oem3 (.text:UART_read)
                  000052d2    0000000a                           : UART.oem3 (.text:UART_write)
                  000052dc    0000000a     scif_framework.obj (.text:osalClearCtrlReadyInt)
                  000052e6    0000000a     scif_framework.obj (.text:osalClearTaskAlertInt)
                  000052f0    0000000a     scif_framework.obj (.text:osalDisableCtrlReadyInt)
                  000052fa    0000000a     scif_framework.obj (.text:osalEnableCtrlReadyInt)
                  00005304    0000000a     scif_framework.obj (.text:scifOsalDisableTaskAlertInt)
                  0000530e    0000000a     scif_framework.obj (.text:scifOsalEnableTaskAlertInt)
                  00005318    00000008     drivers_cc26x0r2.aem3 : UARTCC26XX.oem3 (.text:readSemCallback)
                  00005320    00000008     scif_framework.obj (.text:scifOsalEnterCriticalSection)
                  00005328    00000008     drivers_cc26x0r2.aem3 : UARTCC26XX.oem3 (.text:writeSemCallback)
                  00005330    00000006     dpl_cc26x0r2.aem3 : ClockP_tirtos.oem3 (.text:ClockP_Params_init)
                  00005336    00000006     drivers_cc26x0r2.aem3 : UARTCC26XX.oem3 (.text:UARTCC26XX_readPolling)
                  0000533c    00000006                           : UARTCC26XX.oem3 (.text:UARTCC26XX_writePolling)
                  00005342    00000004     dpl_cc26x0r2.aem3 : PowerCC26XX_tirtos.oem3 (.text:CPUwfi)
                  00005346    00000004                       : ClockP_tirtos.oem3 (.text:ClockP_destruct)
                  0000534a    00000004                       : ClockP_tirtos.oem3 (.text:ClockP_getCpuFreq)
                  0000534e    00000004                       : ClockP_tirtos.oem3 (.text:ClockP_setTimeout)
                  00005352    00000004                       : ClockP_tirtos.oem3 (.text:ClockP_start)
                  00005356    00000004                       : ClockP_tirtos.oem3 (.text:ClockP_stop)
                  0000535a    00000004                       : HwiP_tirtos.oem3 (.text:HwiP_destruct)
                  0000535e    00000004                       : HwiP_tirtos.oem3 (.text:HwiP_disable)
                  00005362    00000004     drivers_cc26x0r2.aem3 : List.oem3 (.text:List_head)
                  00005366    00000004                           : List.oem3 (.text:List_next)
                  0000536a    00000004     dpl_cc26x0r2.aem3 : SemaphoreP_tirtos.oem3 (.text:SemaphoreP_destruct)
                  0000536e    00000004                       : SemaphoreP_tirtos.oem3 (.text:SemaphoreP_post)
                  00005372    00000004                       : SwiP_tirtos.oem3 (.text:SwiP_destruct)
                  00005376    00000004                       : SwiP_tirtos.oem3 (.text:SwiP_disable)
                  0000537a    00000004                       : SwiP_tirtos.oem3 (.text:SwiP_getTrigger)
                  0000537e    00000004                       : SwiP_tirtos.oem3 (.text:SwiP_or)
                  00005382    00000004                       : SwiP_tirtos.oem3 (.text:SwiP_post)
                  00005386    00000004     drivers_cc26x0r2.aem3 : PowerCC26XX.oem3 (.text:nopResourceHandler)
                  0000538a    00000002     rom_sysbios.aem3 : rom_sysbios.obj (.text:xdc_runtime_SysCallback_defaultExit)
                  0000538c    00000008     (.tramp.ti_sysbios_knl_Swi_destruct.1)
                  00005394    00000008     (.tramp.ti_sysbios_knl_Semaphore_destruct.1)
                  0000539c    00000008     (.tramp.ti_sysbios_family_arm_m3_Hwi_destruct.1)
                  000053a4    00000008     (.tramp.ti_sysbios_BIOS_getCpuFreq__E.1)
                  000053ac    00000008     (.tramp.ti_sysbios_knl_Clock_destruct.1)
                  000053b4    00000008     (.tramp.ti_sysbios_family_arm_m3_Hwi_enableInterrupt__E.1)
                  000053bc    00000008     (.tramp.ti_sysbios_family_arm_m3_Hwi_disableInterrupt__E.1)
                  000053c4    00000008     (.tramp.ti_sysbios_knl_Semaphore_delete.1)
                  000053cc    00000008     (.tramp.xdc_runtime_Startup_startMods__I.1)
                  000053d4    00000008     (.tramp.ti_sysbios_knl_Semaphore_pend__E.1)
                  000053dc    00000008     (.tramp.ti_sysbios_knl_Clock_logTick__E.1)
                  000053e4    00000008     (.tramp.ti_sysbios_knl_Task_Params__init__S.1)
                  000053ec    00000008     (.tramp.ti_sysbios_knl_Swi_post__E.1)
                  000053f4    00000008     (.tramp.ti_sysbios_BIOS_RtsGateProxy_leave__E.1)
                  000053fc    00000008     (.tramp.ti_sysbios_knl_Swi_construct.1)
                  00005404    00000008     (.tramp.ti_sysbios_BIOS_RtsGateProxy_enter__E.1)
                  0000540c    00000008     (.tramp.ti_sysbios_knl_Task_restore__E.1)
                  00005414    00000008     (.tramp.ti_sysbios_family_arm_m3_Hwi_disableFxn__E.1)
                  0000541c    00000008     (.tramp.ti_sysbios_knl_Semaphore_post__E.1)
                  00005424    00000008     (.tramp.ti_sysbios_knl_Semaphore_create.1)
                  0000542c    00000008     (.tramp.ti_sysbios_knl_Semaphore_Params__init__S.1)
                  00005434    00000008     (.tramp.ti_sysbios_knl_Task_startup__E.1)
                  0000543c    00000008     (.tramp.ti_sysbios_knl_Swi_startup__E.1)
                  00005444    00000008     (.tramp.ti_sysbios_hal_Hwi_startup__E.1)
                  0000544c    00000008     (.tramp.ti_sysbios_family_arm_cc26xx_Timer_startup__E.1)
                  00005454    00000008     (.tramp.xdc_runtime_System_atexit__E.1)
                  0000545c    00000008     (.tramp.ti_sysbios_BIOS_linkedWithIncorrectBootLibrary__E.1)
                  00005464    00000008     (.tramp.xdc_runtime_Startup_rtsDone__E.1)
                  0000546c    00000008     (.tramp.ti_sysbios_BIOS_setThreadType__E.1)
                  00005474    00000008     (.tramp.ti_sysbios_knl_Task_disable__E.1)
                  0000547c    00000008     (.tramp.ti_sysbios_knl_Swi_disable__E.1)
                  00005484    00000008     (.tramp.ti_sysbios_knl_Semaphore_construct.1)
                  0000548c    00000008     (.tramp.ti_sysbios_family_arm_m3_Hwi_construct.1)
                  00005494    00000008     (.tramp.ti_sysbios_knl_Swi_Params__init__S.1)
                  0000549c    00000008     (.tramp.ti_sysbios_family_arm_m3_Hwi_Params__init__S.1)
                  000054a4    00000008     (.tramp.xdc_runtime_Text_ropeText__E.1)
                  000054ac    00000008     (.tramp.xdc_runtime_System_exit__E.1)
                  000054b4    00000008     (.tramp.ti_sysbios_knl_Clock_construct.1)
                  000054bc    00000008     (.tramp.ti_sysbios_knl_Clock_Params__init__S.1)
                  000054c4    00000008     (.tramp.ti_sysbios_BIOS_start__E.1)
                  000054cc    00000008     (.tramp.ti_sysbios_knl_Task_construct.1)
                  000054d4    00000008     (.tramp.ti_sysbios_knl_Clock_scheduleNextTick__E.1)
                  000054dc    00000008     (.tramp.ti_sysbios_knl_Clock_walkQueueDynamic__E.1)
                  000054e4    00000008     (.tramp.ti_sysbios_knl_Clock_TimerProxy_getCurrentTick__E.1)
                  000054ec    00000008     (.tramp.xdc_runtime_System_abort__E.1)
                  000054f4    00000008     (.tramp.xdc_runtime_Gate_leaveSystem__E.1)
                  000054fc    00000008     (.tramp.xdc_runtime_Gate_enterSystem__E.1)
                  00005504    00000008     (.tramp.ti_sysbios_knl_Clock_stop__E.1)
                  0000550c    00000008     (.tramp.ti_sysbios_knl_Clock_start__E.1)
                  00005514    00000008     (.tramp.ti_sysbios_knl_Clock_setTimeout__E.1)
                  0000551c    00000008     (.tramp.ti_sysbios_family_arm_m3_Hwi_restoreFxn__E.1)
                  00005524    00000008     (.tramp.ti_sysbios_knl_Swi_restore__E.1)

.cinit     0    00000738    0000028c     
                  00000738    00000145     (.cinit..data.load) [load image, compression = lzss]
                  0000087d    00000028     (.cinit..data:ti_sysbios_family_arm_m3_Hwi_Module__state__V.load) [load image, compression = lzss]
                  000008a5    00000021     (.cinit..data:ti_sysbios_knl_Task_Module__state__V.load) [load image, compression = lzss]
                  000008c6    0000001f     (.cinit..data:ti_sysbios_BIOS_Module__state__V.load) [load image, compression = lzss]
                  000008e5    0000001d     (.cinit..data:ti_sysbios_knl_Clock_Module__state__V.load) [load image, compression = lzss]
                  00000902    00000010     (.cinit..data:ti_sysbios_knl_Swi_Module__state__V.load) [load image, compression = lzss]
                  00000912    00000002     --HOLE-- [fill = 0]
                  00000914    0000000c     (__TI_handler_table)
                  00000920    0000000b     (.cinit..data:ti_sysbios_family_arm_cc26xx_Timer_Module__state__V.load) [load image, compression = lzss]
                  0000092b    0000000b     (.cinit..data:xdc_runtime_System_Module__state__V.load) [load image, compression = lzss]
                  00000936    00000002     --HOLE-- [fill = 0]
                  00000938    00000008     (.cinit..bss.load) [load image, compression = zero_init]
                  00000940    00000008     (.cinit..data:xdc_runtime_Memory_Module__state__V.load) [load image, compression = lzss]
                  00000948    00000007     (.cinit..data:ti_sysbios_family_arm_cc26xx_TimestampProvider_Module__state__V.load) [load image, compression = lzss]
                  0000094f    00000007     (.cinit..data:xdc_runtime_Startup_Module__state__V.load) [load image, compression = lzss]
                  00000956    00000006     (.cinit..data:xdc_runtime_Error_Module__state__V.load) [load image, compression = lzss]
                  0000095c    00000068     (__TI_cinit_table)

.init_array 
*          0    00000000    00000000     UNINITIALIZED

.ccfg      0    0001ffa8    00000058     
                  0001ffa8    00000058     ccfg.obj (.ccfg:retain)

.bss       0    20000208    00001883     UNINITIALIZED
                  20000208    00000800     (.common:ti_sysbios_heaps_HeapMem_Instance_State_0_buf__A)
                  20000a08    00000400     (.common:myTaskStack)
                  20000e08    00000400     (.common:myTaskStack1)
                  20001208    00000200     rom_pem3.oem3 (.bss:taskStackSection)
                  20001408    000001f4     (.common:xdc_runtime_SysMin_Module_State_0_outbuf__A)
                  200015fc    0000012c     (.common:uartCC26XXObjects)
                  20001728    00000120     rtsv7M3_T_le_eabi.lib : trgmsg.obj (.bss:_CIOBUF_)
                  20001848    000000c8     (.common:ti_sysbios_family_arm_m3_Hwi_dispatchTable)
                  20001910    00000050     (.common:myTask)
                  20001960    00000050     (.common:myTask1)
                  200019b0    00000030     scif_framework.obj (.bss:scifData)
                  200019e0    00000020     (.common:uartCC26XXRingBuffer)
                  20001a00    0000001c     scif_framework.obj (.bss:hwiCtrlReady)
                  20001a1c    0000001c     scif_framework.obj (.bss:hwiTaskAlert)
                  20001a38    0000001c     scif_framework.obj (.bss:semCtrlReady)
                  20001a54    00000014     driverlib.lib : osc.obj (.bss:oscHfGlobals)
                  20001a68    00000008     dpl_cc26x0r2.aem3 : PowerCC26XX_tirtos.oem3 (.bss:$O1$$)
                  20001a70    00000008     driverlib.lib : sys_ctrl.obj (.bss:powerQualGlobals)
                  20001a78    00000008     (.common:parmbuf)
                  20001a80    00000004     (.common:ClockP_tickPeriod)
                  20001a84    00000004     (.common:uart)
                  20001a88    00000002     drivers_cc26x0r2.aem3 : UARTCC26XX.oem3 (.bss)
                  20001a8a    00000001     (.common:driverlib_release_0_49664)

.data      0    20001a90    0000053f     UNINITIALIZED
                  20001a90    00000114     drivers_cc26x0r2.aem3 : PINCC26XX.oem3 (.data:$O1$$)
                  20001ba4    00000114                           : PowerCC26XX.oem3 (.data:PowerCC26XX_module)
                  20001cb8    00000080     rom_pem3.oem3 (.data:ti_sysbios_knl_Swi_Module_State_0_readyQ__A)
                  20001d38    00000054     drivers_cc26x0r2.aem3 : GPIOCC26XX.oem3 (.data:$O1$$)
                  20001d8c    0000004c     rom_pem3.oem3 (.data:ti_sysbios_knl_Task_Object__table__V)
                  20001dd8    00000048     rom_pem3.oem3 (.data:ti_sysbios_family_arm_cc26xx_Timer_Object__table__V)
                  20001e20    00000038     rom_pem3.oem3 (.data:ti_sysbios_gates_GateMutex_Object__table__V)
                  20001e58    00000030     rom_pem3.oem3 (.data:ti_sysbios_knl_Swi_Object__table__V)
                  20001e88    00000020     rom_pem3.oem3 (.data:ti_sysbios_knl_Clock_Object__table__V)
                  20001ea8    00000020     rom_pem3.oem3 (.data:ti_sysbios_knl_Task_Module_State_0_readyQ__A)
                  20001ec8    00000020     rom_pem3.oem3 (.data:xdc_runtime_Error_IgnoreBlock)
                  20001ee8    00000018     rom_pem3.oem3 (.data:ti_sysbios_family_arm_m3_Hwi_Object__table__V)
                  20001f00    00000018     rom_pem3.oem3 (.data:ti_sysbios_heaps_HeapMem_Object__table__V)
                  20001f18    00000014     CC2640R2_LAUNCHXL.obj (.data:gpioPinConfigs)
                  20001f2c    0000000c     scif_framework.obj (.data)
                  20001f38    0000000c     rom_pem3.oem3 (.data:xdc_runtime_SysMin_Module__state__V)
                  20001f44    00000008     rtsv7M3_T_le_eabi.lib : _lock.obj (.data:$O1$$)
                  20001f4c    00000008     CC2640R2_LAUNCHXL.obj (.data:gpioCallbackFunctions)
                  20001f54    00000008     rom_pem3.oem3 (.data:ti_sysbios_family_arm_m3_Hwi_Module__root__V)
                  20001f5c    00000008     rom_pem3.oem3 (.data:ti_sysbios_gates_GateHwi_Module__root__V)
                  20001f64    00000008     rom_pem3.oem3 (.data:ti_sysbios_gates_GateMutex_Module__root__V)
                  20001f6c    00000008     rom_pem3.oem3 (.data:ti_sysbios_hal_Hwi_Module__root__V)
                  20001f74    00000008     rom_pem3.oem3 (.data:ti_sysbios_heaps_HeapMem_Module__root__V)
                  20001f7c    00000008     rom_pem3.oem3 (.data:ti_sysbios_knl_Clock_Module__root__V)
                  20001f84    00000008     rom_pem3.oem3 (.data:ti_sysbios_knl_Event_Module__root__V)
                  20001f8c    00000008     rom_pem3.oem3 (.data:ti_sysbios_knl_Mailbox_Module__root__V)
                  20001f94    00000008     rom_pem3.oem3 (.data:ti_sysbios_knl_Queue_Module__root__V)
                  20001f9c    00000008     rom_pem3.oem3 (.data:ti_sysbios_knl_Semaphore_Module__root__V)
                  20001fa4    00000008     rom_pem3.oem3 (.data:ti_sysbios_knl_Swi_Module__root__V)
                  20001fac    00000008     rom_pem3.oem3 (.data:ti_sysbios_knl_Task_Module__root__V)
                  20001fb4    00000008     rom_pem3.oem3 (.data:xdc_runtime_System_Module_State_0_atexitHandlers__A)
                  20001fbc    00000004     rtsv7M3_T_le_eabi.lib : stkdepth_vars.obj (.data)
                  20001fc0    00000004     rom_pem3.oem3 (.data:ti_sysbios_family_arm_m3_Hwi_Module_State_0_excContext__A)
                  20001fc4    00000004     rom_pem3.oem3 (.data:ti_sysbios_family_arm_m3_Hwi_Module_State_0_excStack__A)
                  20001fc8    00000004     rom_pem3.oem3 (.data:ti_sysbios_knl_Task_Module_State_0_idleTask__A)
                  20001fcc    00000002     rom_pem3.oem3 (.data:ti_sysbios_family_arm_m3_Hwi_Module_State_0_excActive__A)
                  20001fce    00000001     drivers_cc26x0r2.aem3 : UART.oem3 (.data)

.stack     0    20004d00    00000300     UNINITIALIZED
                  20004d00    00000300     --HOLE--

.resetVecs 
*          0    00000000    0000003c     
                  00000000    0000003c     rom_pem3.oem3 (.resetVecs)

.const:ti_sysbios_heaps_HeapMem_Module__FXNS__C 
*          0    00001000    00000028     
                  00001000    00000028     rom_pem3.oem3 (.const:ti_sysbios_heaps_HeapMem_Module__FXNS__C)

.const:ti_sysbios_gates_GateHwi_Module__FXNS__C 
*          0    00001028    00000024     
                  00001028    00000024     rom_pem3.oem3 (.const:ti_sysbios_gates_GateHwi_Module__FXNS__C)

.const:ti_sysbios_gates_GateMutex_Module__FXNS__C 
*          0    0000104c    00000024     
                  0000104c    00000024     rom_pem3.oem3 (.const:ti_sysbios_gates_GateMutex_Module__FXNS__C)

.const:ti_sysbios_family_arm_m3_Hwi_Object__DESC__C 
*          0    00001070    00000020     
                  00001070    00000020     rom_pem3.oem3 (.const:ti_sysbios_family_arm_m3_Hwi_Object__DESC__C)

.const:ti_sysbios_gates_GateHwi_Object__DESC__C 
*          0    00001090    00000020     
                  00001090    00000020     rom_pem3.oem3 (.const:ti_sysbios_gates_GateHwi_Object__DESC__C)

.const:ti_sysbios_gates_GateMutex_Object__DESC__C 
*          0    000010b0    00000020     
                  000010b0    00000020     rom_pem3.oem3 (.const:ti_sysbios_gates_GateMutex_Object__DESC__C)

.const:ti_sysbios_hal_Hwi_Object__DESC__C 
*          0    000010d0    00000020     
                  000010d0    00000020     rom_pem3.oem3 (.const:ti_sysbios_hal_Hwi_Object__DESC__C)

.const:ti_sysbios_heaps_HeapMem_Object__DESC__C 
*          0    000010f0    00000020     
                  000010f0    00000020     rom_pem3.oem3 (.const:ti_sysbios_heaps_HeapMem_Object__DESC__C)

.const:ti_sysbios_knl_Clock_Object__DESC__C 
*          0    00001110    00000020     
                  00001110    00000020     rom_pem3.oem3 (.const:ti_sysbios_knl_Clock_Object__DESC__C)

.const:ti_sysbios_knl_Event_Object__DESC__C 
*          0    00001130    00000020     
                  00001130    00000020     rom_pem3.oem3 (.const:ti_sysbios_knl_Event_Object__DESC__C)

.const:ti_sysbios_knl_Mailbox_Object__DESC__C 
*          0    00001150    00000020     
                  00001150    00000020     rom_pem3.oem3 (.const:ti_sysbios_knl_Mailbox_Object__DESC__C)

.const:ti_sysbios_knl_Queue_Object__DESC__C 
*          0    00001170    00000020     
                  00001170    00000020     rom_pem3.oem3 (.const:ti_sysbios_knl_Queue_Object__DESC__C)

.const:ti_sysbios_knl_Semaphore_Object__DESC__C 
*          0    00001190    00000020     
                  00001190    00000020     rom_pem3.oem3 (.const:ti_sysbios_knl_Semaphore_Object__DESC__C)

.const:ti_sysbios_knl_Swi_Object__DESC__C 
*          0    000011b0    00000020     
                  000011b0    00000020     rom_pem3.oem3 (.const:ti_sysbios_knl_Swi_Object__DESC__C)

.const:ti_sysbios_knl_Task_Object__DESC__C 
*          0    000011d0    00000020     
                  000011d0    00000020     rom_pem3.oem3 (.const:ti_sysbios_knl_Task_Object__DESC__C)

.const:ti_sysbios_knl_Idle_funcList__C 
*          0    000011f0    00000008     
                  000011f0    00000008     rom_pem3.oem3 (.const:ti_sysbios_knl_Idle_funcList__C)

.const:ti_sysbios_family_arm_cc26xx_Timer_startupNeeded__C 
*          0    000011f8    00000004     
                  000011f8    00000004     rom_pem3.oem3 (.const:ti_sysbios_family_arm_cc26xx_Timer_startupNeeded__C)

.const:ti_sysbios_family_arm_m3_Hwi_E_alreadyDefined__C 
*          0    000011fc    00000004     
                  000011fc    00000004     rom_pem3.oem3 (.const:ti_sysbios_family_arm_m3_Hwi_E_alreadyDefined__C)

.const:ti_sysbios_family_arm_m3_Hwi_E_hwiLimitExceeded__C 
*          0    00001200    00000004     
                  00001200    00000004     rom_pem3.oem3 (.const:ti_sysbios_family_arm_m3_Hwi_E_hwiLimitExceeded__C)

.const:ti_sysbios_family_arm_m3_Hwi_NUM_INTERRUPTS__C 
*          0    00001204    00000004     
                  00001204    00000004     rom_pem3.oem3 (.const:ti_sysbios_family_arm_m3_Hwi_NUM_INTERRUPTS__C)

.const:ti_sysbios_family_arm_m3_Hwi_Object__count__C 
*          0    00001208    00000004     
                  00001208    00000004     rom_pem3.oem3 (.const:ti_sysbios_family_arm_m3_Hwi_Object__count__C)

.const:ti_sysbios_family_arm_m3_Hwi_Object__table__C 
*          0    0000120c    00000004     
                  0000120c    00000004     rom_pem3.oem3 (.const:ti_sysbios_family_arm_m3_Hwi_Object__table__C)

.const:ti_sysbios_family_arm_m3_Hwi_ccr__C 
*          0    00001210    00000004     
                  00001210    00000004     rom_pem3.oem3 (.const:ti_sysbios_family_arm_m3_Hwi_ccr__C)

.const:ti_sysbios_family_arm_m3_Hwi_excHandlerFunc__C 
*          0    00001214    00000004     
                  00001214    00000004     rom_pem3.oem3 (.const:ti_sysbios_family_arm_m3_Hwi_excHandlerFunc__C)

.const:ti_sysbios_family_arm_m3_Hwi_nullIsrFunc__C 
*          0    00001218    00000004     
                  00001218    00000004     rom_pem3.oem3 (.const:ti_sysbios_family_arm_m3_Hwi_nullIsrFunc__C)

.const:ti_sysbios_family_arm_m3_Hwi_numSparseInterrupts__C 
*          0    0000121c    00000004     
                  0000121c    00000004     rom_pem3.oem3 (.const:ti_sysbios_family_arm_m3_Hwi_numSparseInterrupts__C)

.const:ti_sysbios_family_arm_m3_Hwi_priGroup__C 
*          0    00001220    00000004     
                  00001220    00000004     rom_pem3.oem3 (.const:ti_sysbios_family_arm_m3_Hwi_priGroup__C)

.const:ti_sysbios_family_arm_m3_TaskSupport_stackAlignment__C 
*          0    00001224    00000004     
                  00001224    00000004     rom_pem3.oem3 (.const:ti_sysbios_family_arm_m3_TaskSupport_stackAlignment__C)

.const:ti_sysbios_heaps_HeapMem_E_memory__C 
*          0    00001228    00000004     
                  00001228    00000004     rom_pem3.oem3 (.const:ti_sysbios_heaps_HeapMem_E_memory__C)

.const:ti_sysbios_heaps_HeapMem_Module__gateObj__C 
*          0    0000122c    00000004     
                  0000122c    00000004     rom_pem3.oem3 (.const:ti_sysbios_heaps_HeapMem_Module__gateObj__C)

.const:ti_sysbios_heaps_HeapMem_Object__count__C 
*          0    00001230    00000004     
                  00001230    00000004     rom_pem3.oem3 (.const:ti_sysbios_heaps_HeapMem_Object__count__C)

.const:ti_sysbios_heaps_HeapMem_Object__table__C 
*          0    00001234    00000004     
                  00001234    00000004     rom_pem3.oem3 (.const:ti_sysbios_heaps_HeapMem_Object__table__C)

.const:ti_sysbios_heaps_HeapMem_reqAlign__C 
*          0    00001238    00000004     
                  00001238    00000004     rom_pem3.oem3 (.const:ti_sysbios_heaps_HeapMem_reqAlign__C)

.const:ti_sysbios_knl_Clock_triggerClock__C 
*          0    0000123c    00000004     
                  0000123c    00000004     rom_pem3.oem3 (.const:ti_sysbios_knl_Clock_triggerClock__C)

.const:ti_sysbios_knl_Mailbox_Object__count__C 
*          0    00001240    00000004     
                  00001240    00000004     rom_pem3.oem3 (.const:ti_sysbios_knl_Mailbox_Object__count__C)

.const:ti_sysbios_knl_Mailbox_Object__table__C 
*          0    00001244    00000004     
                  00001244    00000004     rom_pem3.oem3 (.const:ti_sysbios_knl_Mailbox_Object__table__C)

.const:ti_sysbios_knl_Mailbox_maxTypeAlign__C 
*          0    00001248    00000004     
                  00001248    00000004     rom_pem3.oem3 (.const:ti_sysbios_knl_Mailbox_maxTypeAlign__C)

.const:ti_sysbios_knl_Queue_Object__count__C 
*          0    0000124c    00000004     
                  0000124c    00000004     rom_pem3.oem3 (.const:ti_sysbios_knl_Queue_Object__count__C)

.const:ti_sysbios_knl_Queue_Object__table__C 
*          0    00001250    00000004     
                  00001250    00000004     rom_pem3.oem3 (.const:ti_sysbios_knl_Queue_Object__table__C)

.const:ti_sysbios_knl_Semaphore_eventPost__C 
*          0    00001254    00000004     
                  00001254    00000004     rom_pem3.oem3 (.const:ti_sysbios_knl_Semaphore_eventPost__C)

.const:ti_sysbios_knl_Semaphore_eventSync__C 
*          0    00001258    00000004     
                  00001258    00000004     rom_pem3.oem3 (.const:ti_sysbios_knl_Semaphore_eventSync__C)

.const:ti_sysbios_knl_Swi_Object__count__C 
*          0    0000125c    00000004     
                  0000125c    00000004     rom_pem3.oem3 (.const:ti_sysbios_knl_Swi_Object__count__C)

.const:ti_sysbios_knl_Swi_Object__table__C 
*          0    00001260    00000004     
                  00001260    00000004     rom_pem3.oem3 (.const:ti_sysbios_knl_Swi_Object__table__C)

.const:ti_sysbios_knl_Swi_numPriorities__C 
*          0    00001264    00000004     
                  00001264    00000004     rom_pem3.oem3 (.const:ti_sysbios_knl_Swi_numPriorities__C)

.const:ti_sysbios_knl_Task_Object__count__C 
*          0    00001268    00000004     
                  00001268    00000004     rom_pem3.oem3 (.const:ti_sysbios_knl_Task_Object__count__C)

.const:ti_sysbios_knl_Task_Object__table__C 
*          0    0000126c    00000004     
                  0000126c    00000004     rom_pem3.oem3 (.const:ti_sysbios_knl_Task_Object__table__C)

.const:ti_sysbios_knl_Task_allBlockedFunc__C 
*          0    00001270    00000004     
                  00001270    00000004     rom_pem3.oem3 (.const:ti_sysbios_knl_Task_allBlockedFunc__C)

.const:ti_sysbios_knl_Task_defaultStackHeap__C 
*          0    00001274    00000004     
                  00001274    00000004     rom_pem3.oem3 (.const:ti_sysbios_knl_Task_defaultStackHeap__C)

.const:ti_sysbios_knl_Task_defaultStackSize__C 
*          0    00001278    00000004     
                  00001278    00000004     rom_pem3.oem3 (.const:ti_sysbios_knl_Task_defaultStackSize__C)

.const:ti_sysbios_knl_Task_numConstructedTasks__C 
*          0    0000127c    00000004     
                  0000127c    00000004     rom_pem3.oem3 (.const:ti_sysbios_knl_Task_numConstructedTasks__C)

.const:ti_sysbios_family_arm_cc26xx_Timer_Module__id__C 
*          0    00001280    00000002     
                  00001280    00000002     rom_pem3.oem3 (.const:ti_sysbios_family_arm_cc26xx_Timer_Module__id__C)

.const:ti_sysbios_family_arm_cc26xx_TimestampProvider_useClockTimer__C 
*          0    00001282    00000002     
                  00001282    00000002     rom_pem3.oem3 (.const:ti_sysbios_family_arm_cc26xx_TimestampProvider_useClockTimer__C)

.const:ti_sysbios_family_arm_m3_Hwi_Module__id__C 
*          0    00001284    00000002     
                  00001284    00000002     rom_pem3.oem3 (.const:ti_sysbios_family_arm_m3_Hwi_Module__id__C)

.const:ti_sysbios_gates_GateHwi_Module__id__C 
*          0    00001286    00000002     
                  00001286    00000002     rom_pem3.oem3 (.const:ti_sysbios_gates_GateHwi_Module__id__C)

.const:ti_sysbios_gates_GateMutex_Module__id__C 
*          0    00001288    00000002     
                  00001288    00000002     rom_pem3.oem3 (.const:ti_sysbios_gates_GateMutex_Module__id__C)

.const:ti_sysbios_heaps_HeapMem_Module__id__C 
*          0    0000128a    00000002     
                  0000128a    00000002     rom_pem3.oem3 (.const:ti_sysbios_heaps_HeapMem_Module__id__C)

.const:ti_sysbios_knl_Task_initStackFlag__C 
*          0    0000128c    00000002     
                  0000128c    00000002     rom_pem3.oem3 (.const:ti_sysbios_knl_Task_initStackFlag__C)

.const:ti_sysbios_knl_Clock_tickMode__C 
*          0    0000128e    00000001     
                  0000128e    00000001     rom_pem3.oem3 (.const:ti_sysbios_knl_Clock_tickMode__C)

.const:xdc_runtime_Startup_firstFxns__C 
*          0    00001290    00000008     
                  00001290    00000008     rom_pem3.oem3 (.const:xdc_runtime_Startup_firstFxns__C)

.const:xdc_runtime_Startup_lastFxns__C 
*          0    00001298    00000008     
                  00001298    00000008     rom_pem3.oem3 (.const:xdc_runtime_Startup_lastFxns__C)

.const:xdc_runtime_Assert_E_assertFailed__C 
*          0    000012a0    00000004     
                  000012a0    00000004     rom_pem3.oem3 (.const:xdc_runtime_Assert_E_assertFailed__C)

.const:xdc_runtime_Error_E_memory__C 
*          0    000012a4    00000004     
                  000012a4    00000004     rom_pem3.oem3 (.const:xdc_runtime_Error_E_memory__C)

.const:xdc_runtime_Error_policyFxn__C 
*          0    000012a8    00000004     
                  000012a8    00000004     rom_pem3.oem3 (.const:xdc_runtime_Error_policyFxn__C)

.const:xdc_runtime_Error_raiseHook__C 
*          0    000012ac    00000004     
                  000012ac    00000004     rom_pem3.oem3 (.const:xdc_runtime_Error_raiseHook__C)

.const:xdc_runtime_IGateProvider_Interface__BASE__C 
*          0    000012b0    00000004     
                  000012b0    00000004     rom_pem3.oem3 (.const:xdc_runtime_IGateProvider_Interface__BASE__C)

.const:xdc_runtime_IHeap_Interface__BASE__C 
*          0    000012b4    00000004     
                  000012b4    00000004     rom_pem3.oem3 (.const:xdc_runtime_IHeap_Interface__BASE__C)

.const:xdc_runtime_IModule_Interface__BASE__C 
*          0    000012b8    00000004     
                  000012b8    00000004     rom_pem3.oem3 (.const:xdc_runtime_IModule_Interface__BASE__C)

.const:xdc_runtime_Memory_defaultHeapInstance__C 
*          0    000012bc    00000004     
                  000012bc    00000004     rom_pem3.oem3 (.const:xdc_runtime_Memory_defaultHeapInstance__C)

.const:xdc_runtime_Startup_execImpl__C 
*          0    000012c0    00000004     
                  000012c0    00000004     rom_pem3.oem3 (.const:xdc_runtime_Startup_execImpl__C)

.const:xdc_runtime_Startup_maxPasses__C 
*          0    000012c4    00000004     
                  000012c4    00000004     rom_pem3.oem3 (.const:xdc_runtime_Startup_maxPasses__C)

.const:xdc_runtime_Startup_sfxnRts__C 
*          0    000012c8    00000004     
                  000012c8    00000004     rom_pem3.oem3 (.const:xdc_runtime_Startup_sfxnRts__C)

.const:xdc_runtime_Startup_sfxnTab__C 
*          0    000012cc    00000004     
                  000012cc    00000004     rom_pem3.oem3 (.const:xdc_runtime_Startup_sfxnTab__C)

.const:xdc_runtime_Startup_startModsFxn__C 
*          0    000012d0    00000004     
                  000012d0    00000004     rom_pem3.oem3 (.const:xdc_runtime_Startup_startModsFxn__C)

.const:xdc_runtime_SysCallback_abortFxn__C 
*          0    000012d4    00000004     
                  000012d4    00000004     rom_pem3.oem3 (.const:xdc_runtime_SysCallback_abortFxn__C)

.const:xdc_runtime_SysCallback_exitFxn__C 
*          0    000012d8    00000004     
                  000012d8    00000004     rom_pem3.oem3 (.const:xdc_runtime_SysCallback_exitFxn__C)

.const:xdc_runtime_System_abortFxn__C 
*          0    000012dc    00000004     
                  000012dc    00000004     rom_pem3.oem3 (.const:xdc_runtime_System_abortFxn__C)

.const:xdc_runtime_System_exitFxn__C 
*          0    000012e0    00000004     
                  000012e0    00000004     rom_pem3.oem3 (.const:xdc_runtime_System_exitFxn__C)

.const:xdc_runtime_System_maxAtexitHandlers__C 
*          0    000012e4    00000004     
                  000012e4    00000004     rom_pem3.oem3 (.const:xdc_runtime_System_maxAtexitHandlers__C)

.const:xdc_runtime_Text_charTab__C 
*          0    000012e8    00000004     
                  000012e8    00000004     rom_pem3.oem3 (.const:xdc_runtime_Text_charTab__C)

.const:xdc_runtime_Text_nameEmpty__C 
*          0    000012ec    00000004     
                  000012ec    00000004     rom_pem3.oem3 (.const:xdc_runtime_Text_nameEmpty__C)

.const:xdc_runtime_Text_nameStatic__C 
*          0    000012f0    00000004     
                  000012f0    00000004     rom_pem3.oem3 (.const:xdc_runtime_Text_nameStatic__C)

.const:xdc_runtime_Text_nameUnknown__C 
*          0    000012f4    00000004     
                  000012f4    00000004     rom_pem3.oem3 (.const:xdc_runtime_Text_nameUnknown__C)

.const:xdc_runtime_Error_maxDepth__C 
*          0    000012f8    00000002     
                  000012f8    00000002     rom_pem3.oem3 (.const:xdc_runtime_Error_maxDepth__C)

.const:xdc_runtime_Memory_Module__id__C 
*          0    000012fa    00000002     
                  000012fa    00000002     rom_pem3.oem3 (.const:xdc_runtime_Memory_Module__id__C)

.const:xdc_runtime_Text_charCnt__C 
*          0    000012fc    00000002     
                  000012fc    00000002     rom_pem3.oem3 (.const:xdc_runtime_Text_charCnt__C)

.const:xdc_runtime_Text_isLoaded__C 
*          0    000012fe    00000002     
                  000012fe    00000002     rom_pem3.oem3 (.const:xdc_runtime_Text_isLoaded__C)

.const:xdc_runtime_Error_policy__C 
*          0    00001300    00000001     
                  00001300    00000001     rom_pem3.oem3 (.const:xdc_runtime_Error_policy__C)

.const:ti_sysbios_rom_ROM_ti_sysbios_family_arm_cc26xx_Timer_getCount64__E 
*          0    00001304    00000004     
                  00001304    00000004     rom_pem3.oem3 (.const:ti_sysbios_rom_ROM_ti_sysbios_family_arm_cc26xx_Timer_getCount64__E)

.const:ti_sysbios_rom_ROM_ti_sysbios_family_arm_cc26xx_Timer_getCurrentTick__E 
*          0    00001308    00000004     
                  00001308    00000004     rom_pem3.oem3 (.const:ti_sysbios_rom_ROM_ti_sysbios_family_arm_cc26xx_Timer_getCurrentTick__E)

.const:ti_sysbios_rom_ROM_ti_sysbios_family_arm_cc26xx_Timer_getMaxTicks__E 
*          0    0000130c    00000004     
                  0000130c    00000004     rom_pem3.oem3 (.const:ti_sysbios_rom_ROM_ti_sysbios_family_arm_cc26xx_Timer_getMaxTicks__E)

.const:ti_sysbios_rom_ROM_ti_sysbios_family_arm_cc26xx_Timer_initDevice__I 
*          0    00001310    00000004     
                  00001310    00000004     rom_pem3.oem3 (.const:ti_sysbios_rom_ROM_ti_sysbios_family_arm_cc26xx_Timer_initDevice__I)

.const:ti_sysbios_rom_ROM_ti_sysbios_family_arm_cc26xx_Timer_setNextTick__E 
*          0    00001314    00000004     
                  00001314    00000004     rom_pem3.oem3 (.const:ti_sysbios_rom_ROM_ti_sysbios_family_arm_cc26xx_Timer_setNextTick__E)

.const:ti_sysbios_rom_ROM_ti_sysbios_family_arm_cc26xx_Timer_setThreshold__I 
*          0    00001318    00000004     
                  00001318    00000004     rom_pem3.oem3 (.const:ti_sysbios_rom_ROM_ti_sysbios_family_arm_cc26xx_Timer_setThreshold__I)

.const:ti_sysbios_rom_ROM_ti_sysbios_family_arm_cc26xx_Timer_start__E 
*          0    0000131c    00000004     
                  0000131c    00000004     rom_pem3.oem3 (.const:ti_sysbios_rom_ROM_ti_sysbios_family_arm_cc26xx_Timer_start__E)

.const:ti_sysbios_rom_ROM_ti_sysbios_family_arm_cc26xx_TimestampProvider_get32__E 
*          0    00001320    00000004     
                  00001320    00000004     rom_pem3.oem3 (.const:ti_sysbios_rom_ROM_ti_sysbios_family_arm_cc26xx_TimestampProvider_get32__E)

.const:ti_sysbios_rom_ROM_xdc_runtime_Startup_getState__I 
*          0    00001324    00000004     
                  00001324    00000004     rom_pem3.oem3 (.const:ti_sysbios_rom_ROM_xdc_runtime_Startup_getState__I)

.const:ti_sysbios_rom_ROM_xdc_runtime_System_SupportProxy_abort__E 
*          0    00001328    00000004     
                  00001328    00000004     rom_pem3.oem3 (.const:ti_sysbios_rom_ROM_xdc_runtime_System_SupportProxy_abort__E)

.const:ti_sysbios_rom_ROM_xdc_runtime_System_SupportProxy_exit__E 
*          0    0000132c    00000004     
                  0000132c    00000004     rom_pem3.oem3 (.const:ti_sysbios_rom_ROM_xdc_runtime_System_SupportProxy_exit__E)

.vecs      0    20000000    000000c8     NOLOAD SECTION
                  20000000    000000c8     rom_pem3.oem3 (.vecs)

.data:ti_sysbios_knl_Task_Module__state__V 
*          0    20000100    00000044     UNINITIALIZED
                  20000100    00000044     rom_pem3.oem3 (.data:ti_sysbios_knl_Task_Module__state__V)

.data:ti_sysbios_family_arm_m3_Hwi_Module__state__V 
*          0    20000144    00000034     UNINITIALIZED
                  20000144    00000034     rom_pem3.oem3 (.data:ti_sysbios_family_arm_m3_Hwi_Module__state__V)

.data:ti_sysbios_knl_Clock_Module__state__V 
*          0    20000178    0000002c     UNINITIALIZED
                  20000178    0000002c     rom_pem3.oem3 (.data:ti_sysbios_knl_Clock_Module__state__V)

.data:ti_sysbios_BIOS_Module__state__V 
*          0    200001a4    00000024     UNINITIALIZED
                  200001a4    00000024     rom_pem3.oem3 (.data:ti_sysbios_BIOS_Module__state__V)

.data:ti_sysbios_knl_Swi_Module__state__V 
*          0    200001c8    0000001c     UNINITIALIZED
                  200001c8    0000001c     rom_pem3.oem3 (.data:ti_sysbios_knl_Swi_Module__state__V)

.data:ti_sysbios_family_arm_cc26xx_Timer_Module__state__V 
*          0    200001e4    00000008     UNINITIALIZED
                  200001e4    00000008     rom_pem3.oem3 (.data:ti_sysbios_family_arm_cc26xx_Timer_Module__state__V)

.data:ti_sysbios_family_arm_cc26xx_TimestampProvider_Module__state__V 
*          0    200001ec    00000004     UNINITIALIZED
                  200001ec    00000004     rom_pem3.oem3 (.data:ti_sysbios_family_arm_cc26xx_TimestampProvider_Module__state__V)

.data:xdc_runtime_Startup_Module__state__V 
*          0    200001f0    00000008     UNINITIALIZED
                  200001f0    00000008     rom_pem3.oem3 (.data:xdc_runtime_Startup_Module__state__V)

.data:xdc_runtime_System_Module__state__V 
*          0    200001f8    00000008     UNINITIALIZED
                  200001f8    00000008     rom_pem3.oem3 (.data:xdc_runtime_System_Module__state__V)

.data:xdc_runtime_Memory_Module__state__V 
*          0    20000200    00000004     UNINITIALIZED
                  20000200    00000004     rom_pem3.oem3 (.data:xdc_runtime_Memory_Module__state__V)

.data:xdc_runtime_Error_Module__state__V 
*          0    20000204    00000002     UNINITIALIZED
                  20000204    00000002     rom_pem3.oem3 (.data:xdc_runtime_Error_Module__state__V)

.bootVecs 
*          0    00000000    00000008     DSECT
                  00000000    00000008     boot.aem3 : boot.oem3 (.bootVecs)

xdc.meta   0    00000000    000000f7     COPY SECTION
                  00000000    000000f7     rom_pem3.oem3 (xdc.meta)

xdc.noload 
*          0    00000000    00000000     COPY SECTION

MODULE SUMMARY

       Module                            code    ro data   rw data
       ------                            ----    -------   -------
    .\
       main_tirtos.obj                   426     12        2212   
       scif.obj                          494     1172      0      
       scif_framework.obj                1362    0         144    
    +--+---------------------------------+-------+---------+---------+
       Total:                            2282    1184      2356   
                                                                  
    .\sdk_files__do_not_edit\
       CC2640R2_LAUNCHXL.obj             0       149       360    
       ccfg.obj                          0       88        0      
    +--+---------------------------------+-------+---------+---------+
       Total:                            0       237       360    
                                                                  
    C:\Users\x0263641\workspace_v7\uart_emulator_launchpad_tirtos\Debug\configPkg\package\cfg\
       rom_pem3.oem3                     472     1043      4376   
    +--+---------------------------------+-------+---------+---------+
       Total:                            472     1043      4376   
                                                                  
    C:/ti/simplelink_cc2640r2_sdk_1_50_00_58/kernel/tirtos/packages/ti/dpl/lib/dpl_cc26x0r2.aem3
       PowerCC26XX_tirtos.oem3           300     0         8      
       SemaphoreP_tirtos.oem3            126     0         0      
       ClockP_tirtos.oem3                98      0         4      
       SwiP_tirtos.oem3                  96      0         0      
       HwiP_tirtos.oem3                  86      0         0      
    +--+---------------------------------+-------+---------+---------+
       Total:                            706     0         12     
                                                                  
    C:/ti/simplelink_cc2640r2_sdk_1_50_00_58/source/ti/devices/cc26x0r2/driverlib/bin/ccs/driverlib.lib
       sys_ctrl.obj                      740     0         8      
       setup.obj                         312     0         0      
       osc.obj                           284     0         20     
       chipinfo.obj                      122     0         0      
       uart.obj                          94      0         0      
       adi.obj                           40      0         0      
       cpu.obj                           24      0         0      
       ioc.obj                           20      0         0      
       driverlib_release.obj             0       0         1      
    +--+---------------------------------+-------+---------+---------+
       Total:                            1636    0         29     
                                                                  
    C:/ti/simplelink_cc2640r2_sdk_1_50_00_58/source/ti/drivers/lib/drivers_cc26x0r2.aem3
       UARTCC26XX.oem3                   2554    104       2      
       PowerCC26XX.oem3                  2132    76        276    
       PINCC26XX.oem3                    1406    0         276    
       PowerCC26XX_calibrateRCOSC.oem3   1388    0         0      
       GPIOCC26XX.oem3                   732     64        84     
       UART.oem3                         172     36        1      
       RingBuf.oem3                      148     0         0      
       List.oem3                         76      0         0      
    +--+---------------------------------+-------+---------+---------+
       Total:                            8608    280       639    
                                                                  
    C:\TI\ccsv7\tools\compiler\ti-cgt-arm_16.9.6.LTS\lib\rtsv7M3_T_le_eabi.lib
       ull_div_t2.obj                    500     0         0      
       trgmsg.obj                        104     0         288    
       memcpy_t2.obj                     156     0         0      
       memset_t2.obj                     122     0         0      
       copy_decompress_lzss.obj          104     0         0      
       hostwrite.obj                     88      0         0      
       cpy_tbl.obj                       76      0         0      
       _lock.obj                         20      0         8      
       args_main.obj                     24      0         0      
       ll_mul_t2.obj                     24      0         0      
       copy_decompress_none.obj          14      0         0      
       copy_zero_init.obj                12      0         0      
       hostopen.obj                      0       0         8      
       stkdepth_vars.obj                 0       0         4      
    +--+---------------------------------+-------+---------+---------+
       Total:                            1244    0         308    
                                                                  
    C:\TI\simplelink_cc2640r2_sdk_1_50_00_58\kernel\tirtos\packages\ti\targets\arm\rtsarm\lib\auto_init.aem3
       auto_init.oem3                    160     0         0      
    +--+---------------------------------+-------+---------+---------+
       Total:                            160     0         0      
                                                                  
    C:\TI\simplelink_cc2640r2_sdk_1_50_00_58\kernel\tirtos\packages\ti\targets\arm\rtsarm\lib\boot.aem3
       boot.oem3                         68      0         0      
    +--+---------------------------------+-------+---------+---------+
       Total:                            68      0         0      
                                                                  
    C:\Users\x0263641\workspace_v7\uart_emulator_launchpad_tirtos\src\sysbios\rom_sysbios.aem3
       rom_sysbios.obj                   1300    0         0      
    +--+---------------------------------+-------+---------+---------+
       Total:                            1300    0         0      
                                                                  
       Stack:                            0       0         768    
       Linker Generated:                 416     648       0      
    +--+---------------------------------+-------+---------+---------+
       Grand Total:                      16892   3392      8848   


LINKER GENERATED COPY TABLES

__TI_cinit_table @ 0000095c records: 13, size/record: 8, table size: 104
	.data: load addr=00000738, load size=00000145 bytes, run addr=20001a90, run size=0000053f bytes, compression=lzss
	.data:ti_sysbios_family_arm_m3_Hwi_Module__state__V: load addr=0000087d, load size=00000028 bytes, run addr=20000144, run size=00000034 bytes, compression=lzss
	.data:ti_sysbios_knl_Task_Module__state__V: load addr=000008a5, load size=00000021 bytes, run addr=20000100, run size=00000044 bytes, compression=lzss
	.data:ti_sysbios_BIOS_Module__state__V: load addr=000008c6, load size=0000001f bytes, run addr=200001a4, run size=00000024 bytes, compression=lzss
	.data:ti_sysbios_knl_Clock_Module__state__V: load addr=000008e5, load size=0000001d bytes, run addr=20000178, run size=0000002c bytes, compression=lzss
	.data:ti_sysbios_knl_Swi_Module__state__V: load addr=00000902, load size=00000010 bytes, run addr=200001c8, run size=0000001c bytes, compression=lzss
	.data:ti_sysbios_family_arm_cc26xx_Timer_Module__state__V: load addr=00000920, load size=0000000b bytes, run addr=200001e4, run size=00000008 bytes, compression=lzss
	.data:xdc_runtime_System_Module__state__V: load addr=0000092b, load size=0000000b bytes, run addr=200001f8, run size=00000008 bytes, compression=lzss
	.bss: load addr=00000938, load size=00000008 bytes, run addr=20000208, run size=00001883 bytes, compression=zero_init
	.data:xdc_runtime_Memory_Module__state__V: load addr=00000940, load size=00000008 bytes, run addr=20000200, run size=00000004 bytes, compression=lzss
	.data:ti_sysbios_family_arm_cc26xx_TimestampProvider_Module__state__V: load addr=00000948, load size=00000007 bytes, run addr=200001ec, run size=00000004 bytes, compression=lzss
	.data:xdc_runtime_Startup_Module__state__V: load addr=0000094f, load size=00000007 bytes, run addr=200001f0, run size=00000008 bytes, compression=lzss
	.data:xdc_runtime_Error_Module__state__V: load addr=00000956, load size=00000006 bytes, run addr=20000204, run size=00000002 bytes, compression=lzss


LINKER GENERATED HANDLER TABLE

__TI_handler_table @ 00000914 records: 3, size/record: 4, table size: 12
	index: 0, handler: __TI_decompress_lzss
	index: 1, handler: __TI_decompress_none
	index: 2, handler: __TI_zero_init


FAR CALL TRAMPOLINES

callee name               trampoline name
   callee addr  tramp addr   call addr  call info
--------------  -----------  ---------  ----------------
ti_sysbios_knl_Swi_destruct  $Tramp$TT$L$PI$$ti_sysbios_knl_Swi_destruct
   1001c115     0000538c     00005372   dpl_cc26x0r2.aem3 : SwiP_tirtos.oem3 (.text:SwiP_destruct)
ti_sysbios_knl_Semaphore_destruct  $Tramp$TT$L$PI$$ti_sysbios_knl_Semaphore_destruct
   1001c10d     00005394     0000536a   dpl_cc26x0r2.aem3 : SemaphoreP_tirtos.oem3 (.text:SemaphoreP_destruct)
ti_sysbios_family_arm_m3_Hwi_destruct  $Tramp$TT$L$PI$$ti_sysbios_family_arm_m3_Hwi_destruct
   1001c0a9     0000539c     0000535a   dpl_cc26x0r2.aem3 : HwiP_tirtos.oem3 (.text:HwiP_destruct)
ti_sysbios_BIOS_getCpuFreq__E  $Tramp$TT$L$PI$$ti_sysbios_BIOS_getCpuFreq__E
   1001be91     000053a4     0000534a   dpl_cc26x0r2.aem3 : ClockP_tirtos.oem3 (.text:ClockP_getCpuFreq)
ti_sysbios_knl_Clock_destruct  $Tramp$TT$L$PI$$ti_sysbios_knl_Clock_destruct
   1001c0dd     000053ac     00005346   dpl_cc26x0r2.aem3 : ClockP_tirtos.oem3 (.text:ClockP_destruct)
ti_sysbios_family_arm_m3_Hwi_enableInterrupt__E  $Tramp$TT$L$PI$$ti_sysbios_family_arm_m3_Hwi_enableInterrupt__E
   1001af89     000053b4     000052fe   scif_framework.obj (.text:osalEnableCtrlReadyInt)
                             00005312   scif_framework.obj (.text:scifOsalEnableTaskAlertInt)
ti_sysbios_family_arm_m3_Hwi_disableInterrupt__E  $Tramp$TT$L$PI$$ti_sysbios_family_arm_m3_Hwi_disableInterrupt__E
   1001af45     000053bc     000052f4   scif_framework.obj (.text:osalDisableCtrlReadyInt)
                             00005308   scif_framework.obj (.text:scifOsalDisableTaskAlertInt)
ti_sysbios_knl_Semaphore_delete  $Tramp$TT$L$PI$$ti_sysbios_knl_Semaphore_delete
   1001c109     000053c4     0000526e   dpl_cc26x0r2.aem3 : SemaphoreP_tirtos.oem3 (.text:SemaphoreP_delete)
xdc_runtime_Startup_startMods__I  $Tramp$TT$L$PI$$xdc_runtime_Startup_startMods__I
   1001c129     000053cc     00005168   rom_pem3.oem3 (.text:xdc_runtime_Startup_exec__I)
ti_sysbios_knl_Semaphore_pend__E  $Tramp$TT$L$PI$$ti_sysbios_knl_Semaphore_pend__E
   10019b05     000053d4     0000513c   dpl_cc26x0r2.aem3 : SemaphoreP_tirtos.oem3 (.text:SemaphoreP_pend)
ti_sysbios_knl_Clock_logTick__E  $Tramp$TT$L$PI$$ti_sysbios_knl_Clock_logTick__E
   1001b843     000053dc     00005116   rom_pem3.oem3 (.text:ti_sysbios_knl_Clock_doTick__I)
ti_sysbios_knl_Task_Params__init__S  $Tramp$TT$L$PI$$ti_sysbios_knl_Task_Params__init__S
   1001c021     000053e4     00005082   main_tirtos.obj (.text:ti_sysbios_knl_Task_Params_init)
ti_sysbios_knl_Swi_post__E  $Tramp$TT$L$PI$$ti_sysbios_knl_Swi_post__E
   1001b011     000053ec     00004fd0   rom_sysbios.aem3 : rom_sysbios.obj (.text:ti_sysbios_knl_Swi_or__E)
                             0000511e   rom_pem3.oem3 (.text:ti_sysbios_knl_Clock_doTick__I)
                             00005382   dpl_cc26x0r2.aem3 : SwiP_tirtos.oem3 (.text:SwiP_post)
ti_sysbios_BIOS_RtsGateProxy_leave__E  $Tramp$TT$L$PI$$ti_sysbios_BIOS_RtsGateProxy_leave__E
   1001c095     000053f4     00004fb2   rom_pem3.oem3 (.text:ti_sysbios_BIOS_rtsUnlock__I)
ti_sysbios_knl_Swi_construct  $Tramp$TT$L$PI$$ti_sysbios_knl_Swi_construct
   1001ad79     000053fc     00004e52   rom_sysbios.aem3 : rom_sysbios.obj (.text:ti_sysbios_knl_Swi_construct2__E)
ti_sysbios_BIOS_RtsGateProxy_enter__E  $Tramp$TT$L$PI$$ti_sysbios_BIOS_RtsGateProxy_enter__E
   1001c091     00005404     00004d42   rom_pem3.oem3 (.text:ti_sysbios_BIOS_rtsLock__I)
ti_sysbios_knl_Task_restore__E  $Tramp$TT$L$PI$$ti_sysbios_knl_Task_restore__E
   1001b7f5     0000540c     00004d0e   dpl_cc26x0r2.aem3 : PowerCC26XX_tirtos.oem3 (.text:PowerCC26XX_schedulerRestore)
ti_sysbios_family_arm_m3_Hwi_disableFxn__E  $Tramp$TT$L$PI$$ti_sysbios_family_arm_m3_Hwi_disableFxn__E
   1001bf85     00005414     00004a62   scif_framework.obj (.text:osalLockCtrlTaskNbl)
                             00005322   scif_framework.obj (.text:scifOsalEnterCriticalSection)
                             0000535e   dpl_cc26x0r2.aem3 : HwiP_tirtos.oem3 (.text:HwiP_disable)
ti_sysbios_knl_Semaphore_post__E  $Tramp$TT$L$PI$$ti_sysbios_knl_Semaphore_post__E
   1001a3e1     0000541c     00004a42   scif_framework.obj (.text:osalIndicateCtrlReady)
                             0000536e   dpl_cc26x0r2.aem3 : SemaphoreP_tirtos.oem3 (.text:SemaphoreP_post)
ti_sysbios_knl_Semaphore_create  $Tramp$TT$L$PI$$ti_sysbios_knl_Semaphore_create
   1001b2d1     00005424     00004a28   dpl_cc26x0r2.aem3 : SemaphoreP_tirtos.oem3 (.text:SemaphoreP_createBinary)
ti_sysbios_knl_Semaphore_Params__init__S  $Tramp$TT$L$PI$$ti_sysbios_knl_Semaphore_Params__init__S
   1001c009     0000542c     000049ee   dpl_cc26x0r2.aem3 : SemaphoreP_tirtos.oem3 (.text:SemaphoreP_constructBinary)
                             00004a18                     : SemaphoreP_tirtos.oem3 (.text:SemaphoreP_createBinary)
                             0000506c   scif_framework.obj (.text:ti_sysbios_knl_Semaphore_Params_init)
ti_sysbios_knl_Task_startup__E  $Tramp$TT$L$PI$$ti_sysbios_knl_Task_startup__E
   1001c125     00005434     000048ec   rom_pem3.oem3 (.text:ti_sysbios_BIOS_startFunc__I)
ti_sysbios_knl_Swi_startup__E  $Tramp$TT$L$PI$$ti_sysbios_knl_Swi_startup__E
   1001c085     0000543c     000048e8   rom_pem3.oem3 (.text:ti_sysbios_BIOS_startFunc__I)
ti_sysbios_hal_Hwi_startup__E  $Tramp$TT$L$PI$$ti_sysbios_hal_Hwi_startup__E
   1001c04b     00005444     000048e4   rom_pem3.oem3 (.text:ti_sysbios_BIOS_startFunc__I)
ti_sysbios_family_arm_cc26xx_Timer_startup__E  $Tramp$TT$L$PI$$ti_sysbios_family_arm_cc26xx_Timer_startup__E
   1001b4e9     0000544c     000048e0   rom_pem3.oem3 (.text:ti_sysbios_BIOS_startFunc__I)
xdc_runtime_System_atexit__E  $Tramp$TT$L$PI$$xdc_runtime_System_atexit__E
   1001c581     00005454     000048d8   rom_pem3.oem3 (.text:ti_sysbios_BIOS_startFunc__I)
ti_sysbios_BIOS_linkedWithIncorrectBootLibrary__E  $Tramp$TT$L$PI$$ti_sysbios_BIOS_linkedWithIncorrectBootLibrary__E
   1001a683     0000545c     000048d2   rom_pem3.oem3 (.text:ti_sysbios_BIOS_startFunc__I)
xdc_runtime_Startup_rtsDone__E  $Tramp$TT$L$PI$$xdc_runtime_Startup_rtsDone__E
   1001c769     00005464     000048ca   rom_pem3.oem3 (.text:ti_sysbios_BIOS_startFunc__I)
ti_sysbios_BIOS_setThreadType__E  $Tramp$TT$L$PI$$ti_sysbios_BIOS_setThreadType__E
   1001bea1     0000546c     000048a4   rom_pem3.oem3 (.text:ti_sysbios_BIOS_atExitFunc__I)
                             0000502a   rom_pem3.oem3 (.text:ti_sysbios_BIOS_errorRaiseHook__I)
                             0000503a   rom_pem3.oem3 (.text:ti_sysbios_BIOS_exitFunc__I)
ti_sysbios_knl_Task_disable__E  $Tramp$TT$L$PI$$ti_sysbios_knl_Task_disable__E
   1001bf31     00005474     0000489e   rom_pem3.oem3 (.text:ti_sysbios_BIOS_atExitFunc__I)
                             00004cde   dpl_cc26x0r2.aem3 : PowerCC26XX_tirtos.oem3 (.text:PowerCC26XX_schedulerDisable)
ti_sysbios_knl_Swi_disable__E  $Tramp$TT$L$PI$$ti_sysbios_knl_Swi_disable__E
   1001bf11     0000547c     0000489a   rom_pem3.oem3 (.text:ti_sysbios_BIOS_atExitFunc__I)
                             00005376   dpl_cc26x0r2.aem3 : SwiP_tirtos.oem3 (.text:SwiP_disable)
ti_sysbios_knl_Semaphore_construct  $Tramp$TT$L$PI$$ti_sysbios_knl_Semaphore_construct
   1001b45d     00005484     00004760   scif_framework.obj (.text:scifOsalInit)
                             000049fe   dpl_cc26x0r2.aem3 : SemaphoreP_tirtos.oem3 (.text:SemaphoreP_constructBinary)
ti_sysbios_family_arm_m3_Hwi_construct  $Tramp$TT$L$PI$$ti_sysbios_family_arm_m3_Hwi_construct
   1001aabd     0000548c     00004532   rom_sysbios.aem3 : rom_sysbios.obj (.text:ti_sysbios_family_arm_m3_Hwi_construct2__E)
                             00004856   scif_framework.obj (.text:osalRegisterCtrlReadyInt)
                             00004886   scif_framework.obj (.text:osalRegisterTaskAlertInt)
ti_sysbios_knl_Swi_Params__init__S  $Tramp$TT$L$PI$$ti_sysbios_knl_Swi_Params__init__S
   1001c015     00005494     00004442   dpl_cc26x0r2.aem3 : SwiP_tirtos.oem3 (.text:SwiP_construct)
ti_sysbios_family_arm_m3_Hwi_Params__init__S  $Tramp$TT$L$PI$$ti_sysbios_family_arm_m3_Hwi_Params__init__S
   1001bf79     0000549c     0000438c   dpl_cc26x0r2.aem3 : HwiP_tirtos.oem3 (.text:HwiP_construct)
                             00005056   scif_framework.obj (.text:ti_sysbios_family_arm_m3_Hwi_Params_init)
xdc_runtime_Text_ropeText__E  $Tramp$TT$L$PI$$xdc_runtime_Text_ropeText__E
   1001c6ed     000054a4     00004212   rom_sysbios.aem3 : rom_sysbios.obj (.text:xdc_runtime_Error_setX__E)
xdc_runtime_System_exit__E  $Tramp$TT$L$PI$$xdc_runtime_System_exit__E
   1001c6d5     000054ac     0000418c   boot.aem3 : boot.oem3 (.text)
                             00005040   rom_pem3.oem3 (.text:ti_sysbios_BIOS_exitFunc__I)
ti_sysbios_knl_Clock_construct  $Tramp$TT$L$PI$$ti_sysbios_knl_Clock_construct
   1001b269     000054b4     0000402c   dpl_cc26x0r2.aem3 : ClockP_tirtos.oem3 (.text:ClockP_construct)
ti_sysbios_knl_Clock_Params__init__S  $Tramp$TT$L$PI$$ti_sysbios_knl_Clock_Params__init__S
   1001bfc1     000054bc     0000401c   dpl_cc26x0r2.aem3 : ClockP_tirtos.oem3 (.text:ClockP_construct)
ti_sysbios_BIOS_start__E  $Tramp$TT$L$PI$$ti_sysbios_BIOS_start__E
   1001beb1     000054c4     0000350e   main_tirtos.obj (.text:main)
ti_sysbios_knl_Task_construct  $Tramp$TT$L$PI$$ti_sysbios_knl_Task_construct
   1001ae19     000054cc     000034ea   main_tirtos.obj (.text:main)
                             0000350a   main_tirtos.obj (.text:main)
ti_sysbios_knl_Clock_scheduleNextTick__E  $Tramp$TT$L$PI$$ti_sysbios_knl_Clock_scheduleNextTick__E
   1001bca9     000054d4     000031e2   rom_sysbios.aem3 : rom_sysbios.obj (.text:ti_sysbios_knl_Clock_workFuncDynamic__E)
ti_sysbios_knl_Clock_walkQueueDynamic__E  $Tramp$TT$L$PI$$ti_sysbios_knl_Clock_walkQueueDynamic__E
   1001a2f1     000054dc     000031aa   rom_sysbios.aem3 : rom_sysbios.obj (.text:ti_sysbios_knl_Clock_workFuncDynamic__E)
                             000031c6                    : rom_sysbios.obj (.text:ti_sysbios_knl_Clock_workFuncDynamic__E)
ti_sysbios_knl_Clock_TimerProxy_getCurrentTick__E  $Tramp$TT$L$PI$$ti_sysbios_knl_Clock_TimerProxy_getCurrentTick__E
   1001bee1     000054e4     00003178   rom_sysbios.aem3 : rom_sysbios.obj (.text:ti_sysbios_knl_Clock_workFuncDynamic__E)
                             00004a9e                    : rom_sysbios.obj (.text:ti_sysbios_knl_Clock_getTicksUntilInterrupt__E)
xdc_runtime_System_abort__E  $Tramp$TT$L$PI$$xdc_runtime_System_abort__E
   1001c64d     000054ec     00002d52   rom_sysbios.aem3 : rom_sysbios.obj (.text:xdc_runtime_Error_policyDefault__E)
xdc_runtime_Gate_leaveSystem__E  $Tramp$TT$L$PI$$xdc_runtime_Gate_leaveSystem__E
   1001c789     000054f4     00002d32   rom_sysbios.aem3 : rom_sysbios.obj (.text:xdc_runtime_Error_policyDefault__E)
                             00002d60                    : rom_sysbios.obj (.text:xdc_runtime_Error_policyDefault__E)
                             0000425c                    : rom_sysbios.obj (.text:xdc_runtime_SysMin_flush__E)
                             0000465c                    : rom_sysbios.obj (.text:xdc_runtime_SysMin_putch__E)
xdc_runtime_Gate_enterSystem__E  $Tramp$TT$L$PI$$xdc_runtime_Gate_enterSystem__E
   1001c795     000054fc     00002d26   rom_sysbios.aem3 : rom_sysbios.obj (.text:xdc_runtime_Error_policyDefault__E)
                             00002d56                    : rom_sysbios.obj (.text:xdc_runtime_Error_policyDefault__E)
                             0000422e                    : rom_sysbios.obj (.text:xdc_runtime_SysMin_flush__E)
                             0000463e                    : rom_sysbios.obj (.text:xdc_runtime_SysMin_putch__E)
ti_sysbios_knl_Clock_stop__E  $Tramp$TT$L$PI$$ti_sysbios_knl_Clock_stop__E
   1001bab9     00005504     000027dc   dpl_cc26x0r2.aem3 : PowerCC26XX_tirtos.oem3 (.text:PowerCC26XX_standbyPolicy)
                             00005356                     : ClockP_tirtos.oem3 (.text:ClockP_stop)
ti_sysbios_knl_Clock_start__E  $Tramp$TT$L$PI$$ti_sysbios_knl_Clock_start__E
   1001be1f     0000550c     000027d0   dpl_cc26x0r2.aem3 : PowerCC26XX_tirtos.oem3 (.text:PowerCC26XX_standbyPolicy)
                             00005352                     : ClockP_tirtos.oem3 (.text:ClockP_start)
ti_sysbios_knl_Clock_setTimeout__E  $Tramp$TT$L$PI$$ti_sysbios_knl_Clock_setTimeout__E
   1001c0e5     00005514     000027ca   dpl_cc26x0r2.aem3 : PowerCC26XX_tirtos.oem3 (.text:PowerCC26XX_standbyPolicy)
                             0000534e                     : ClockP_tirtos.oem3 (.text:ClockP_setTimeout)
ti_sysbios_family_arm_m3_Hwi_restoreFxn__E  $Tramp$TT$L$PI$$ti_sysbios_family_arm_m3_Hwi_restoreFxn__E
   1001c061     0000551c     00001fea   drivers_cc26x0r2.aem3 : UARTCC26XX.oem3 (.text:UARTCC26XX_open)
                             00001ff6                         : UARTCC26XX.oem3 (.text:UARTCC26XX_open)
                             0000207c                         : UARTCC26XX.oem3 (.text:UARTCC26XX_open)
                             00002298                         : UARTCC26XX.oem3 (.text:UARTCC26XX_read)
                             000022d8                         : UARTCC26XX.oem3 (.text:UARTCC26XX_read)
                             000022f4                         : UARTCC26XX.oem3 (.text:UARTCC26XX_read)
                             00002340                         : UARTCC26XX.oem3 (.text:UARTCC26XX_read)
                             000025ba                         : UARTCC26XX.oem3 (.text:UARTCC26XX_write)
                             000025d6                         : UARTCC26XX.oem3 (.text:UARTCC26XX_write)
                             00002674                         : UARTCC26XX.oem3 (.text:UARTCC26XX_write)
                             000026f6                         : GPIOCC26XX.oem3 (.text:GPIO_setConfig)
                             00002726                         : GPIOCC26XX.oem3 (.text:GPIO_setConfig)
                             000029f0                         : PINCC26XX.oem3 (.text:PINCC26XX_setIoCfg)
                             00002a34                         : GPIOCC26XX.oem3 (.text:GPIO_init)
                             00002a3a                         : GPIOCC26XX.oem3 (.text:GPIO_init)
                             00002b7a                         : PowerCC26XX.oem3 (.text:Power_releaseDependency)
                             00002c30                         : PowerCC26XX.oem3 (.text:Power_setDependency)
                             00002edc                         : PowerCC26XX.oem3 (.text:switchXOSCHFclockFunc)
                             000032fe                         : UARTCC26XX.oem3 (.text:UARTCC26XX_close)
                             0000332e                         : UARTCC26XX.oem3 (.text:UARTCC26XX_writeCancel)
                             0000333a                         : UARTCC26XX.oem3 (.text:UARTCC26XX_writeCancel)
                             00003380                         : UARTCC26XX.oem3 (.text:UARTCC26XX_writeCancel)
                             0000345c                         : UARTCC26XX.oem3 (.text:writeFinishedDoCallback)
                             00003886                         : PowerCC26XX_calibrateRCOSC.oem3 (.text:PowerCC26XX_initiateCalibration)
                             000039d4                         : UARTCC26XX.oem3 (.text:UARTCC26XX_readCancel)
                             000039e0                         : UARTCC26XX.oem3 (.text:UARTCC26XX_readCancel)
                             000039ea                         : UARTCC26XX.oem3 (.text:UARTCC26XX_readCancel)
                             00003d4c                         : UARTCC26XX.oem3 (.text:UARTCC26XX_control)
                             00003f0a                         : GPIOCC26XX.oem3 (.text:GPIO_write)
                             0000407e                         : PINCC26XX.oem3 (.text:PIN_setOutputEnable)
                             0000412e                         : RingBuf.oem3 (.text:RingBuf_put)
                             00004158                         : RingBuf.oem3 (.text:RingBuf_put)
                             000042de                         : UART.oem3 (.text:UART_init)
                             000043da                         : RingBuf.oem3 (.text:RingBuf_get)
                             000043e2                         : RingBuf.oem3 (.text:RingBuf_get)
                             0000457c                         : GPIOCC26XX.oem3 (.text:GPIO_enableInt)
                             000045e2                         : UARTCC26XX.oem3 (.text:UARTCC26XX_swiIntFxn)
                             000046fa                         : PowerCC26XX.oem3 (.text:Power_releaseConstraint)
                             0000482c                         : PowerCC26XX.oem3 (.text:Power_setConstraint)
                             00004a70   scif_framework.obj (.text:osalLockCtrlTaskNbl)
                             00004a80   scif_framework.obj (.text:osalLockCtrlTaskNbl)
                             00004c70   drivers_cc26x0r2.aem3 : List.oem3 (.text:List_put)
                             00004d30                         : PowerCC26XX.oem3 (.text:Power_unregisterNotify)
                             00005292   scif_framework.obj (.text:scifOsalLeaveCriticalSection)
ti_sysbios_knl_Swi_restore__E  $Tramp$TT$L$PI$$ti_sysbios_knl_Swi_restore__E
   1001b305     00005524     0000181c   drivers_cc26x0r2.aem3 : PowerCC26XX.oem3 (.text:Power_sleep)

[52 trampolines]
[125 trampoline calls]


GLOBAL SYMBOLS: SORTED ALPHABETICALLY BY Name 

address   name                                                                      
-------   ----                                                                      
00000708  ADCBuf_count                                                              
00000709  ADC_count                                                                 
000005c4  BoardGpioInitTable                                                        
000006e4  BoardGpioInitTable1                                                       
00003a9f  C$$IO$$                                                                   
00005331  ClockP_Params_init                                                        
00004001  ClockP_construct                                                          
00005347  ClockP_destruct                                                           
0000534b  ClockP_getCpuFreq                                                         
1001b29d  ClockP_getSystemTicks                                                     
0000534f  ClockP_setTimeout                                                         
00005353  ClockP_start                                                              
00005357  ClockP_stop                                                               
20001a80  ClockP_tickPeriod                                                         
0000070a  Display_count                                                             
0000069c  GPIOCC26XX_config                                                         
00004555  GPIO_enableInt                                                            
00004b59  GPIO_hwiIntFxn                                                            
00002a1d  GPIO_init                                                                 
0000466d  GPIO_setCallback                                                          
00002689  GPIO_setConfig                                                            
00003ec5  GPIO_write                                                                
00003d65  HOSTwrite                                                                 
00005171  HwiP_Params_init                                                          
00004371  HwiP_construct                                                            
0000535b  HwiP_destruct                                                             
0000535f  HwiP_disable                                                              
1001c061  HwiP_restore                                                              
0000070b  I2C_count                                                                 
00005213  List_empty                                                                
00005363  List_head                                                                 
00005367  List_next                                                                 
00004c55  List_put                                                                  
00005005  List_remove                                                               
0000521f  NOROM_CPUcpsid                                                            
0000522b  NOROM_CPUcpsie                                                            
00004985  NOROM_ChipInfo_GetChipFamily                                              
00004ab9  NOROM_ChipInfo_GetChipType                                                
00004e85  NOROM_ChipInfo_GetPackageType                                             
00005089  NOROM_IOCIntEnable                                                        
000037f5  NOROM_OSCHF_AttemptToSwitchToXosc                                         
000040d9  NOROM_OSCHF_SwitchToRcOscTurnOffXosc                                      
00004b7d  NOROM_OSCHF_TurnOnXosc                                                    
000043ed  NOROM_OSC_HPOSCRelativeFrequencyOffsetGet                                 
00005237  NOROM_OSC_HPOSCRelativeFrequencyOffsetToRFCoreFormatConvert               
00002da9  NOROM_SetupTrimDevice                                                     
00003715  NOROM_SysCtrlAdjustRechargeAfterPowerDown                                 
00001889  NOROM_SysCtrlSetRechargeBeforePowerDown                                   
00003939  NOROM_SysCtrl_DCDC_VoltageConditionalControl                              
000051b1  NOROM_ThisLibraryIsFor_CC26x0R2_HaltIfViolated                            
000051bf  NOROM_UARTCharGetNonBlocking                                              
000051cd  NOROM_UARTCharPutNonBlocking                                              
00004c77  NOROM_UARTConfigSetExpClk                                                 
00004cbd  NOROM_UARTDisable                                                         
0000070c  NVS_count                                                                 
00005181  PINCC26XX_getPinCount                                                     
00000714  PINCC26XX_hwAttrs                                                         
000049b1  PINCC26XX_setMux                                                          
00003ad9  PIN_add                                                                   
00004d9d  PIN_close                                                                 
00001c89  PIN_init                                                                  
00003035  PIN_open                                                                  
00005243  PIN_registerIntCb                                                         
00003cb5  PIN_remove                                                                
000046a1  PIN_setConfig                                                             
00004049  PIN_setOutputEnable                                                       
0000458d  PIN_setOutputValue                                                        
0000070d  PWM_count                                                                 
00003ba1  PowerCC26XX_RCOSC_clockFunc                                               
00001331  PowerCC26XX_auxISR                                                        
00003bfd  PowerCC26XX_calibrate                                                     
00000684  PowerCC26XX_config                                                        
00001e45  PowerCC26XX_doCalibrate                                                   
00003861  PowerCC26XX_initiateCalibration                                           
20001ba4  PowerCC26XX_module                                                        
00004cdd  PowerCC26XX_schedulerDisable                                              
00004cfd  PowerCC26XX_schedulerRestore                                              
00002779  PowerCC26XX_standbyPolicy                                                 
20001a6c  PowerCC26XX_swiKey                                                        
20001a68  PowerCC26XX_taskKey                                                       
00005251  Power_getConstraintMask                                                   
0000525d  Power_getDependencyCount                                                  
00004dbb  Power_getTransitionLatency                                                
00004e9d  Power_idleFunc                                                            
00002131  Power_init                                                                
00004ae1  Power_registerNotify                                                      
000046d5  Power_releaseConstraint                                                   
00002ad9  Power_releaseDependency                                                   
00004809  Power_setConstraint                                                       
00002b95  Power_setDependency                                                       
00001645  Power_sleep                                                               
00004d1d  Power_unregisterNotify                                                    
00004161  ResetISR                                                                  
00005129  RingBuf_construct                                                         
000043af  RingBuf_get                                                               
0000411d  RingBuf_put                                                               
UNDEFED   SHT$$INIT_ARRAY$$Base                                                     
UNDEFED   SHT$$INIT_ARRAY$$Limit                                                    
0000070e  SPI_count                                                                 
00004b09  SafeHapiVoid                                                              
000049dd  SemaphoreP_constructBinary                                                
00004a09  SemaphoreP_createBinary                                                   
00005269  SemaphoreP_delete                                                         
0000536b  SemaphoreP_destruct                                                       
0000513b  SemaphoreP_pend                                                           
0000536f  SemaphoreP_post                                                           
00005191  SwiP_Params_init                                                          
00004429  SwiP_construct                                                            
00005373  SwiP_destruct                                                             
00005377  SwiP_disable                                                              
0000537b  SwiP_getTrigger                                                           
0000537f  SwiP_or                                                                   
00005383  SwiP_post                                                                 
1001b305  SwiP_restore                                                              
00003289  UARTCC26XX_close                                                          
00003d0d  UARTCC26XX_control                                                        
000005f0  UARTCC26XX_fxnTable                                                       
00002379  UARTCC26XX_hwiIntFxn                                                      
00004eb5  UARTCC26XX_init                                                           
00001fd5  UARTCC26XX_open                                                           
0000225d  UARTCC26XX_read                                                           
000039a1  UARTCC26XX_readCancel                                                     
00005337  UARTCC26XX_readPolling                                                    
000045c5  UARTCC26XX_swiIntFxn                                                      
0000258d  UARTCC26XX_write                                                          
00003315  UARTCC26XX_writeCancel                                                    
0000533d  UARTCC26XX_writePolling                                                   
00004ecd  UART_Params_init                                                          
000006f0  UART_config                                                               
0000070f  UART_count                                                                
00000640  UART_defaultParams                                                        
000042b1  UART_init                                                                 
000042f1  UART_open                                                                 
000052c9  UART_read                                                                 
000052d3  UART_write                                                                
00004ba1  Uart_rxcallback                                                           
00000710  Watchdog_count                                                            
00000000  __ASM__                                                                   
20001728  __CIOBUF_                                                                 
00000071  __ISA__                                                                   
00000083  __PLAT__                                                                  
20005000  __STACK_END                                                               
00000300  __STACK_SIZE                                                              
20005000  __STACK_TOP                                                               
000000aa  __TARG__                                                                  
0000095c  __TI_CINIT_Base                                                           
000009c4  __TI_CINIT_Limit                                                          
00000914  __TI_Handler_Table_Base                                                   
00000920  __TI_Handler_Table_Limit                                                  
00002ef9  __TI_auto_init                                                            
00003a09  __TI_decompress_lzss                                                      
000051db  __TI_decompress_none                                                      
ffffffff  __TI_pprof_out_hndl                                                       
ffffffff  __TI_prof_data_size                                                       
ffffffff  __TI_prof_data_start                                                      
00003aa3  __TI_readmsg                                                              
00000000  __TI_static_base__                                                        
00003a71  __TI_writemsg                                                             
00005275  __TI_zero_init                                                            
000000cf  __TRDR__                                                                  
00004f15  __aeabi_lmul                                                              
00003539  __aeabi_memclr                                                            
00003539  __aeabi_memclr4                                                           
00003539  __aeabi_memclr8                                                           
00002f99  __aeabi_memcpy                                                            
00002f99  __aeabi_memcpy4                                                           
00002f99  __aeabi_memcpy8                                                           
0000353b  __aeabi_memset                                                            
0000353b  __aeabi_memset4                                                           
0000353b  __aeabi_memset8                                                           
00001a95  __aeabi_uldivmod                                                          
ffffffff  __binit__                                                                 
ffffffff  __c_args__                                                                
0001ffa8  __ccfg                                                                    
20004d00  __stack                                                                   
00004efd  _args_main                                                                
00004161  _c_int00                                                                  
20001f44  _lock                                                                     
000050bf  _nop                                                                      
000050b7  _register_lock                                                            
000050b1  _register_unlock                                                          
20001f48  _unlock                                                                   
ffffffff  binit                                                                     
00003fb5  copy_in                                                                   
20001a8a  driverlib_release_0_49664                                                 
20001f4c  gpioCallbackFunctions                                                     
20001f18  gpioPinConfigs                                                            
00000554  inPinTypes                                                                
000034b9  main                                                                      
20001fbc  main_func_sp                                                              
00002f99  memcpy                                                                    
00003541  memset                                                                    
20001910  myTask                                                                    
20001960  myTask1                                                                   
20000a08  myTaskStack                                                               
20000e08  myTaskStack1                                                              
00000560  outPinStrengths                                                           
0000056c  outPinTypes                                                               
20001a78  parmbuf                                                                   
20001b28  pinHandleTable                                                            
20001a94  pinLowerBound                                                             
20001a90  pinUpperBound                                                             
00000480  resourceDB                                                                
0000362b  scCtrlReadyCallback                                                       
000047a5  scTaskAlertCallback                                                       
00004709  scifAckAlertEvents                                                        
00004f2d  scifClearAlertIntSource                                                   
00000594  scifDriverSetup                                                           
0000514d  scifExecuteTasksOnceNbl                                                   
0000248d  scifInit                                                                  
000033a1  scifInitIo                                                                
00005305  scifOsalDisableTaskAlertInt                                               
0000530f  scifOsalEnableTaskAlertInt                                                
00005321  scifOsalEnterCriticalSection                                              
0000473d  scifOsalInit                                                              
0000528d  scifOsalLeaveCriticalSection                                              
000050c5  scifOsalRegisterCtrlReadyCallback                                         
000050d9  scifOsalRegisterTaskAlertCallback                                         
00003dbd  scifReinitIo                                                              
00005299  scifUartClearEvents                                                       
00004331  scifUartGetRxFifoCount                                                    
00004f45  scifUartRxEnable                                                          
000044a1  scifUartRxGetChar                                                         
0000362d  scifUartSetBaudRate                                                       
00004bc5  scifUartSetEventMask                                                      
00004f5d  scifUartSetRxEnableReqIdleCount                                           
00004f75  scifUartSetRxFifoThr                                                      
00004f8d  scifUartSetRxTimeout                                                      
000044dd  scifUartTxPutChar                                                         
00003e15  scifUninitIo                                                              
00003e6d  taskFxn                                                                   
00003b3d  taskFxn1                                                                  
200001a4  ti_sysbios_BIOS_Module__state__V                                          
1001b9d9  ti_sysbios_BIOS_RtsGateProxy_Handle__label__S                             
1001b9d9  ti_sysbios_BIOS_RtsGateProxy_Handle__label__S__mangled__                  
1001b88d  ti_sysbios_BIOS_RtsGateProxy_Object__delete__S                            
1001bfb5  ti_sysbios_BIOS_RtsGateProxy_Params__init__S                              
1001bfb5  ti_sysbios_BIOS_RtsGateProxy_Params__init__S__mangled__                   
1001c091  ti_sysbios_BIOS_RtsGateProxy_enter__E                                     
1001c095  ti_sysbios_BIOS_RtsGateProxy_leave__E                                     
1001c0bd  ti_sysbios_BIOS_RtsGateProxy_query__E                                     
1001c0bd  ti_sysbios_BIOS_RtsGateProxy_query__E__mangled__                          
00004899  ti_sysbios_BIOS_atExitFunc__I                                             
0000501b  ti_sysbios_BIOS_errorRaiseHook__I                                         
00005031  ti_sysbios_BIOS_exitFunc__I                                               
1001be81  ti_sysbios_BIOS_exit__E                                                   
1001be91  ti_sysbios_BIOS_getCpuFreq__E                                             
1001a683  ti_sysbios_BIOS_linkedWithIncorrectBootLibrary__E                         
00004cbb  ti_sysbios_BIOS_nullFunc__I                                               
00004be9  ti_sysbios_BIOS_registerRTSLock__I                                        
00004c0d  ti_sysbios_BIOS_removeRTSLock__I                                          
00004d3d  ti_sysbios_BIOS_rtsLock__I                                                
00004fa5  ti_sysbios_BIOS_rtsUnlock__I                                              
1001bea1  ti_sysbios_BIOS_setThreadType__E                                          
000048c9  ti_sysbios_BIOS_startFunc__I                                              
1001beb1  ti_sysbios_BIOS_start__E                                                  
00002da9  ti_sysbios_family_arm_cc26xx_Boot_trimDevice                              
00001280  ti_sysbios_family_arm_cc26xx_Timer_Module__id__C                          
1001b8f9  ti_sysbios_family_arm_cc26xx_Timer_Module__startupDone__S                 
200001e4  ti_sysbios_family_arm_cc26xx_Timer_Module__state__V                       
1001b845  ti_sysbios_family_arm_cc26xx_Timer_Module_startup__E                      
20001dd8  ti_sysbios_family_arm_cc26xx_Timer_Object__table__V                       
00004d5d  ti_sysbios_family_arm_cc26xx_Timer_dynamicStub__E                         
00005101  ti_sysbios_family_arm_cc26xx_Timer_getCount64__E                          
000045fd  ti_sysbios_family_arm_cc26xx_Timer_getCurrentTick__E                      
1001c099  ti_sysbios_family_arm_cc26xx_Timer_getExpiredTicks__E                     
00004c31  ti_sysbios_family_arm_cc26xx_Timer_getMaxTicks__E                         
1001c09d  ti_sysbios_family_arm_cc26xx_Timer_getPeriod__E                           
00004771  ti_sysbios_family_arm_cc26xx_Timer_initDevice__I                          
10019f25  ti_sysbios_family_arm_cc26xx_Timer_periodicStub__E                        
1001b4bd  ti_sysbios_family_arm_cc26xx_Timer_postInit__I                            
000047d7  ti_sysbios_family_arm_cc26xx_Timer_setNextTick__E                         
1001c0a1  ti_sysbios_family_arm_cc26xx_Timer_setPeriod__E                           
00004091  ti_sysbios_family_arm_cc26xx_Timer_setThreshold__I                        
000036a1  ti_sysbios_family_arm_cc26xx_Timer_start__E                               
000011f8  ti_sysbios_family_arm_cc26xx_Timer_startupNeeded__C                       
1001b4e9  ti_sysbios_family_arm_cc26xx_Timer_startup__E                             
200001ec  ti_sysbios_family_arm_cc26xx_TimestampProvider_Module__state__V           
1001b919  ti_sysbios_family_arm_cc26xx_TimestampProvider_Module_startup__E          
00005205  ti_sysbios_family_arm_cc26xx_TimestampProvider_get32__E                   
1001b77d  ti_sysbios_family_arm_cc26xx_TimestampProvider_get64__E                   
1001bf6b  ti_sysbios_family_arm_cc26xx_TimestampProvider_getFreq__E                 
00001282  ti_sysbios_family_arm_cc26xx_TimestampProvider_useClockTimer__C           
000011fc  ti_sysbios_family_arm_m3_Hwi_E_alreadyDefined__C                          
00001200  ti_sysbios_family_arm_m3_Hwi_E_hwiLimitExceeded__C                        
1001a755  ti_sysbios_family_arm_m3_Hwi_Instance_finalize__E                         
10019fc1  ti_sysbios_family_arm_m3_Hwi_Instance_init__E                             
20001fcc  ti_sysbios_family_arm_m3_Hwi_Module_State_0_excActive__A                  
20001fc0  ti_sysbios_family_arm_m3_Hwi_Module_State_0_excContext__A                 
20001fc4  ti_sysbios_family_arm_m3_Hwi_Module_State_0_excStack__A                   
00001284  ti_sysbios_family_arm_m3_Hwi_Module__id__C                                
20001f54  ti_sysbios_family_arm_m3_Hwi_Module__root__V                              
1001b939  ti_sysbios_family_arm_m3_Hwi_Module__startupDone__S                       
20000144  ti_sysbios_family_arm_m3_Hwi_Module__state__V                             
1001aeb5  ti_sysbios_family_arm_m3_Hwi_Module_startup__E                            
00001204  ti_sysbios_family_arm_m3_Hwi_NUM_INTERRUPTS__C                            
00001070  ti_sysbios_family_arm_m3_Hwi_Object__DESC__C                              
1001c9e8  ti_sysbios_family_arm_m3_Hwi_Object__PARAMS__C                            
00001208  ti_sysbios_family_arm_m3_Hwi_Object__count__C                             
1001a7b9  ti_sysbios_family_arm_m3_Hwi_Object__create__S                            
1001b959  ti_sysbios_family_arm_m3_Hwi_Object__delete__S                            
1001bc39  ti_sysbios_family_arm_m3_Hwi_Object__destruct__S                          
1001b515  ti_sysbios_family_arm_m3_Hwi_Object__get__S                               
0000120c  ti_sysbios_family_arm_m3_Hwi_Object__table__C                             
20001ee8  ti_sysbios_family_arm_m3_Hwi_Object__table__V                             
1001bf79  ti_sysbios_family_arm_m3_Hwi_Params__init__S                              
00001210  ti_sysbios_family_arm_m3_Hwi_ccr__C                                       
00004e31  ti_sysbios_family_arm_m3_Hwi_clearInterrupt__E                            
1001aabd  ti_sysbios_family_arm_m3_Hwi_construct                                    
00004519  ti_sysbios_family_arm_m3_Hwi_construct2__E                                
1001a8e5  ti_sysbios_family_arm_m3_Hwi_create                                       
1001c0a5  ti_sysbios_family_arm_m3_Hwi_delete                                       
1001c0a9  ti_sysbios_family_arm_m3_Hwi_destruct                                     
1001bf85  ti_sysbios_family_arm_m3_Hwi_disableFxn__E                                
1001af45  ti_sysbios_family_arm_m3_Hwi_disableInterrupt__E                          
1001a81d  ti_sysbios_family_arm_m3_Hwi_dispatchC__I                                 
20001848  ti_sysbios_family_arm_m3_Hwi_dispatchTable                                
1001c7a5  ti_sysbios_family_arm_m3_Hwi_dispatch__I                                  
1001c043  ti_sysbios_family_arm_m3_Hwi_doSwiRestore__I                              
1001c05b  ti_sysbios_family_arm_m3_Hwi_doTaskRestore__I                             
1001bf91  ti_sysbios_family_arm_m3_Hwi_enableFxn__E                                 
1001af89  ti_sysbios_family_arm_m3_Hwi_enableInterrupt__E                           
1001c901  ti_sysbios_family_arm_m3_Hwi_excHandlerAsm__I                             
00001214  ti_sysbios_family_arm_m3_Hwi_excHandlerFunc__C                            
1001b979  ti_sysbios_family_arm_m3_Hwi_excHandler__I                                
1001b099  ti_sysbios_family_arm_m3_Hwi_getStackInfo__E                              
1001a171  ti_sysbios_family_arm_m3_Hwi_initNVIC__E                                  
1001c8b9  ti_sysbios_family_arm_m3_Hwi_initStacks__E                                
00001218  ti_sysbios_family_arm_m3_Hwi_nullIsrFunc__C                               
0000121c  ti_sysbios_family_arm_m3_Hwi_numSparseInterrupts__C                       
e000e000  ti_sysbios_family_arm_m3_Hwi_nvic                                         
1001c93f  ti_sysbios_family_arm_m3_Hwi_pendSV__I                                    
1001bdc1  ti_sysbios_family_arm_m3_Hwi_plug__E                                      
10019e75  ti_sysbios_family_arm_m3_Hwi_postInit__I                                  
00001220  ti_sysbios_family_arm_m3_Hwi_priGroup__C                                  
20000000  ti_sysbios_family_arm_m3_Hwi_ramVectors                                   
00000000  ti_sysbios_family_arm_m3_Hwi_resetVectors                                 
1001c061  ti_sysbios_family_arm_m3_Hwi_restoreFxn__E                                
1001c957  ti_sysbios_family_arm_m3_Hwi_return                                       
1001bc55  ti_sysbios_family_arm_m3_Hwi_setPriority__E                               
1001c04b  ti_sysbios_family_arm_m3_Hwi_startup__E                                   
0000071c  ti_sysbios_family_arm_m3_Hwi_swiDisable__C                                
00000720  ti_sysbios_family_arm_m3_Hwi_swiRestoreHwi__C                             
1001be35  ti_sysbios_family_arm_m3_Hwi_switchFromBootStack__E                       
1001c0ad  ti_sysbios_family_arm_m3_TaskSupport_Module__startupDone__S               
1001c86d  ti_sysbios_family_arm_m3_TaskSupport_buildTaskStack                       
1001bf9d  ti_sysbios_family_arm_m3_TaskSupport_getStackAlignment__E                 
1001c959  ti_sysbios_family_arm_m3_TaskSupport_glue                                 
00001224  ti_sysbios_family_arm_m3_TaskSupport_stackAlignment__C                    
1001b155  ti_sysbios_family_arm_m3_TaskSupport_start__E                             
1001c969  ti_sysbios_family_arm_m3_TaskSupport_swap__E                              
1001c921  ti_sysbios_family_xxx_Hwi_switchAndRunFunc                                
1001b999  ti_sysbios_gates_GateHwi_Handle__label__S                                 
1001b153  ti_sysbios_gates_GateHwi_Instance_init__E                                 
00001028  ti_sysbios_gates_GateHwi_Module__FXNS__C                                  
00001286  ti_sysbios_gates_GateHwi_Module__id__C                                    
20001f5c  ti_sysbios_gates_GateHwi_Module__root__V                                  
00001090  ti_sysbios_gates_GateHwi_Object__DESC__C                                  
1001cad8  ti_sysbios_gates_GateHwi_Object__PARAMS__C                                
1001b869  ti_sysbios_gates_GateHwi_Object__create__S                                
1001b9b9  ti_sysbios_gates_GateHwi_Object__delete__S                                
1001bfa9  ti_sysbios_gates_GateHwi_enter__E                                         
1001c067  ti_sysbios_gates_GateHwi_leave__E                                         
1001c0b1  ti_sysbios_gates_GateHwi_query__E                                         
1001b9d9  ti_sysbios_gates_GateMutex_Handle__label__S                               
1001cb68  ti_sysbios_gates_GateMutex_Instance_State_sem__O                          
1001bec1  ti_sysbios_gates_GateMutex_Instance_finalize__E                           
1001bc71  ti_sysbios_gates_GateMutex_Instance_init__E                               
0000104c  ti_sysbios_gates_GateMutex_Module__FXNS__C                                
00001288  ti_sysbios_gates_GateMutex_Module__id__C                                  
20001f64  ti_sysbios_gates_GateMutex_Module__root__V                                
000010b0  ti_sysbios_gates_GateMutex_Object__DESC__C                                
1001caf0  ti_sysbios_gates_GateMutex_Object__PARAMS__C                              
1001b36d  ti_sysbios_gates_GateMutex_Object__create__S                              
1001b88d  ti_sysbios_gates_GateMutex_Object__delete__S                              
1001b9f9  ti_sysbios_gates_GateMutex_Object__destruct__S                            
20001e20  ti_sysbios_gates_GateMutex_Object__table__V                               
1001bfb5  ti_sysbios_gates_GateMutex_Params__init__S                                
1001b541  ti_sysbios_gates_GateMutex_construct                                      
1001b39d  ti_sysbios_gates_GateMutex_create                                         
1001c0b5  ti_sysbios_gates_GateMutex_delete                                         
1001c0b9  ti_sysbios_gates_GateMutex_destruct                                       
1001b3cd  ti_sysbios_gates_GateMutex_enter__E                                       
1001bdd9  ti_sysbios_gates_GateMutex_leave__E                                       
1001c0bd  ti_sysbios_gates_GateMutex_query__E                                       
1001b939  ti_sysbios_hal_Hwi_HwiProxy_Module__startupDone__S                        
1001b939  ti_sysbios_hal_Hwi_HwiProxy_Module__startupDone__S__mangled__             
1001bed1  ti_sysbios_hal_Hwi_HwiProxy_Object__create__S                             
1001b959  ti_sysbios_hal_Hwi_HwiProxy_Object__delete__S                             
1001bf79  ti_sysbios_hal_Hwi_HwiProxy_Params__init__S                               
1001bf79  ti_sysbios_hal_Hwi_HwiProxy_Params__init__S__mangled__                    
00004e31  ti_sysbios_hal_Hwi_HwiProxy_clearInterrupt__E                             
1001bc8d  ti_sysbios_hal_Hwi_HwiProxy_create                                        
1001c0c1  ti_sysbios_hal_Hwi_HwiProxy_delete                                        
1001af45  ti_sysbios_hal_Hwi_HwiProxy_disableInterrupt__E                           
1001af45  ti_sysbios_hal_Hwi_HwiProxy_disableInterrupt__E__mangled__                
1001af89  ti_sysbios_hal_Hwi_HwiProxy_enableInterrupt__E                            
1001af89  ti_sysbios_hal_Hwi_HwiProxy_enableInterrupt__E__mangled__                 
1001b099  ti_sysbios_hal_Hwi_HwiProxy_getStackInfo__E                               
1001b099  ti_sysbios_hal_Hwi_HwiProxy_getStackInfo__E__mangled__                    
1001c04b  ti_sysbios_hal_Hwi_HwiProxy_startup__E                                    
1001c04b  ti_sysbios_hal_Hwi_HwiProxy_startup__E__mangled__                         
1001be35  ti_sysbios_hal_Hwi_HwiProxy_switchFromBootStack__E                        
1001be35  ti_sysbios_hal_Hwi_HwiProxy_switchFromBootStack__E__mangled__             
1001c039  ti_sysbios_hal_Hwi_Instance_finalize__E                                   
1001b81d  ti_sysbios_hal_Hwi_Instance_init__E                                       
20001f6c  ti_sysbios_hal_Hwi_Module__root__V                                        
1001be5d  ti_sysbios_hal_Hwi_Module_startup__E                                      
000010d0  ti_sysbios_hal_Hwi_Object__DESC__C                                        
1001ca18  ti_sysbios_hal_Hwi_Object__PARAMS__C                                      
1001ba19  ti_sysbios_hal_Hwi_Object__delete__S                                      
00004e31  ti_sysbios_hal_Hwi_clearInterrupt__E                                      
1001a881  ti_sysbios_hal_Hwi_create                                                 
1001c0c5  ti_sysbios_hal_Hwi_delete                                                 
1001af45  ti_sysbios_hal_Hwi_disableInterrupt__E                                    
1001af45  ti_sysbios_hal_Hwi_disableInterrupt__E                                    
1001af89  ti_sysbios_hal_Hwi_enableInterrupt__E                                     
1001af89  ti_sysbios_hal_Hwi_enableInterrupt__E                                     
1001b099  ti_sysbios_hal_Hwi_getStackInfo__E                                        
1001b099  ti_sysbios_hal_Hwi_getStackInfo__E                                        
1001b56d  ti_sysbios_hal_Hwi_initStack                                              
1001c04b  ti_sysbios_hal_Hwi_startup__E                                             
1001c04b  ti_sysbios_hal_Hwi_startup__E                                             
1001be35  ti_sysbios_hal_Hwi_switchFromBootStack__E                                 
1001be35  ti_sysbios_hal_Hwi_switchFromBootStack__E                                 
00001228  ti_sysbios_heaps_HeapMem_E_memory__C                                      
1001ba39  ti_sysbios_heaps_HeapMem_Handle__label__S                                 
20000208  ti_sysbios_heaps_HeapMem_Instance_State_0_buf__A                          
1001b18d  ti_sysbios_heaps_HeapMem_Instance_init__E                                 
1001b9d9  ti_sysbios_heaps_HeapMem_Module_GateProxy_Handle__label__S                
1001b9d9  ti_sysbios_heaps_HeapMem_Module_GateProxy_Handle__label__S__mangled__     
1001b88d  ti_sysbios_heaps_HeapMem_Module_GateProxy_Object__delete__S               
1001bfb5  ti_sysbios_heaps_HeapMem_Module_GateProxy_Params__init__S                 
1001bfb5  ti_sysbios_heaps_HeapMem_Module_GateProxy_Params__init__S__mangled__      
1001c0c9  ti_sysbios_heaps_HeapMem_Module_GateProxy_enter__E                        
1001c0cd  ti_sysbios_heaps_HeapMem_Module_GateProxy_leave__E                        
1001c0bd  ti_sysbios_heaps_HeapMem_Module_GateProxy_query__E                        
1001c0bd  ti_sysbios_heaps_HeapMem_Module_GateProxy_query__E__mangled__             
00001000  ti_sysbios_heaps_HeapMem_Module__FXNS__C                                  
0000122c  ti_sysbios_heaps_HeapMem_Module__gateObj__C                               
0000128a  ti_sysbios_heaps_HeapMem_Module__id__C                                    
20001f74  ti_sysbios_heaps_HeapMem_Module__root__V                                  
000010f0  ti_sysbios_heaps_HeapMem_Object__DESC__C                                  
1001ca6c  ti_sysbios_heaps_HeapMem_Object__PARAMS__C                                
00001230  ti_sysbios_heaps_HeapMem_Object__count__C                                 
1001b599  ti_sysbios_heaps_HeapMem_Object__create__S                                
1001ba59  ti_sysbios_heaps_HeapMem_Object__delete__S                                
1001b5c5  ti_sysbios_heaps_HeapMem_Object__get__S                                   
00001234  ti_sysbios_heaps_HeapMem_Object__table__C                                 
20001f00  ti_sysbios_heaps_HeapMem_Object__table__V                                 
1001a615  ti_sysbios_heaps_HeapMem_allocUnprotected__E                              
1001ab15  ti_sysbios_heaps_HeapMem_alloc__E                                         
1001ab6d  ti_sysbios_heaps_HeapMem_freeUnprotected__E                               
1001b3fd  ti_sysbios_heaps_HeapMem_free__E                                          
1001aefd  ti_sysbios_heaps_HeapMem_getStats__E                                      
1001b235  ti_sysbios_heaps_HeapMem_init__I                                          
1001c06d  ti_sysbios_heaps_HeapMem_isBlocking__E                                    
00001238  ti_sysbios_heaps_HeapMem_reqAlign__C                                      
1001bf41  ti_sysbios_heaps_HeapMem_restore__E                                       
1001be09  ti_sysbios_knl_Clock_Instance_finalize__E                                 
1001b1c5  ti_sysbios_knl_Clock_Instance_init__E                                     
1001cb6c  ti_sysbios_knl_Clock_Module_State_clockQ__O                               
20001f7c  ti_sysbios_knl_Clock_Module__root__V                                      
20000178  ti_sysbios_knl_Clock_Module__state__V                                     
1001ba79  ti_sysbios_knl_Clock_Module_startup__E                                    
00001110  ti_sysbios_knl_Clock_Object__DESC__C                                      
1001ca90  ti_sysbios_knl_Clock_Object__PARAMS__C                                    
1001b8b1  ti_sysbios_knl_Clock_Object__delete__S                                    
1001ba99  ti_sysbios_knl_Clock_Object__destruct__S                                  
20001e88  ti_sysbios_knl_Clock_Object__table__V                                     
1001bfc1  ti_sysbios_knl_Clock_Params__init__S                                      
1001b8f9  ti_sysbios_knl_Clock_TimerProxy_Module__startupDone__S                    
1001b8f9  ti_sysbios_knl_Clock_TimerProxy_Module__startupDone__S__mangled__         
1001bee1  ti_sysbios_knl_Clock_TimerProxy_getCurrentTick__E                         
1001c0d1  ti_sysbios_knl_Clock_TimerProxy_getExpiredTicks__E                        
1001bef1  ti_sysbios_knl_Clock_TimerProxy_getMaxTicks__E                            
1001c0d5  ti_sysbios_knl_Clock_TimerProxy_getPeriod__E                              
1001bf01  ti_sysbios_knl_Clock_TimerProxy_setNextTick__E                            
1001b4e9  ti_sysbios_knl_Clock_TimerProxy_startup__E                                
1001b4e9  ti_sysbios_knl_Clock_TimerProxy_startup__E__mangled__                     
1001b7a5  ti_sysbios_knl_Clock_addI__E                                              
1001b269  ti_sysbios_knl_Clock_construct                                            
1001b1fd  ti_sysbios_knl_Clock_create                                               
1001c0d9  ti_sysbios_knl_Clock_delete                                               
1001c0dd  ti_sysbios_knl_Clock_destruct                                             
00005115  ti_sysbios_knl_Clock_doTick__I                                            
00004a8d  ti_sysbios_knl_Clock_getTicksUntilInterrupt__E                            
1001b29d  ti_sysbios_knl_Clock_getTicks__E                                          
1001bfcd  ti_sysbios_knl_Clock_getTimerHandle__E                                    
1001b843  ti_sysbios_knl_Clock_logTick__E                                           
1001c0e1  ti_sysbios_knl_Clock_removeI__E                                           
1001bca9  ti_sysbios_knl_Clock_scheduleNextTick__E                                  
1001c0e5  ti_sysbios_knl_Clock_setTimeout__E                                        
1001a1f1  ti_sysbios_knl_Clock_startI__E                                            
1001be1f  ti_sysbios_knl_Clock_start__E                                             
1001bab9  ti_sysbios_knl_Clock_stop__E                                              
0000128e  ti_sysbios_knl_Clock_tickMode__C                                          
00000724  ti_sysbios_knl_Clock_tickPeriod__C                                        
0000123c  ti_sysbios_knl_Clock_triggerClock__C                                      
1001bdbf  ti_sysbios_knl_Clock_triggerFunc__I                                       
1001a2f1  ti_sysbios_knl_Clock_walkQueueDynamic__E                                  
00003165  ti_sysbios_knl_Clock_workFuncDynamic__E                                   
1001a369  ti_sysbios_knl_Clock_workFunc__E                                          
1001cb70  ti_sysbios_knl_Event_Instance_State_pendQ__O                              
1001be49  ti_sysbios_knl_Event_Instance_init__E                                     
20001f84  ti_sysbios_knl_Event_Module__root__V                                      
00001130  ti_sysbios_knl_Event_Object__DESC__C                                      
1001cb08  ti_sysbios_knl_Event_Object__PARAMS__C                                    
1001bad9  ti_sysbios_knl_Event_Object__delete__S                                    
1001bcc5  ti_sysbios_knl_Event_Object__destruct__S                                  
1001bfd9  ti_sysbios_knl_Event_Params__init__S                                      
1001baf9  ti_sysbios_knl_Event_checkEvents__I                                       
1001b5f1  ti_sysbios_knl_Event_construct                                            
1001b42d  ti_sysbios_knl_Event_create                                               
1001c0e9  ti_sysbios_knl_Event_delete                                               
1001c0ed  ti_sysbios_knl_Event_destruct                                             
1001b61d  ti_sysbios_knl_Event_pendTimeout__I                                       
10019bf9  ti_sysbios_knl_Event_pend__E                                              
1001a455  ti_sysbios_knl_Event_post__E                                              
1001be6f  ti_sysbios_knl_Event_sync__E                                              
00000728  ti_sysbios_knl_Idle_funcList__A                                           
000011f0  ti_sysbios_knl_Idle_funcList__C                                           
1001c053  ti_sysbios_knl_Idle_loop__E                                               
1001bb19  ti_sysbios_knl_Idle_run__E                                                
1001cb74  ti_sysbios_knl_Mailbox_Instance_State_dataQue__O                          
1001cb78  ti_sysbios_knl_Mailbox_Instance_State_dataSem__O                          
1001cb7c  ti_sysbios_knl_Mailbox_Instance_State_freeQue__O                          
1001cb80  ti_sysbios_knl_Mailbox_Instance_State_freeSem__O                          
1001a4c5  ti_sysbios_knl_Mailbox_Instance_finalize__E                               
10019dad  ti_sysbios_knl_Mailbox_Instance_init__E                                   
20001f8c  ti_sysbios_knl_Mailbox_Module__root__V                                    
1001afcd  ti_sysbios_knl_Mailbox_Module_startup__E                                  
00001150  ti_sysbios_knl_Mailbox_Object__DESC__C                                    
1001c9b4  ti_sysbios_knl_Mailbox_Object__PARAMS__C                                  
00001240  ti_sysbios_knl_Mailbox_Object__count__C                                   
1001bb39  ti_sysbios_knl_Mailbox_Object__delete__S                                  
1001bce1  ti_sysbios_knl_Mailbox_Object__destruct__S                                
1001b649  ti_sysbios_knl_Mailbox_Object__get__S                                     
00001244  ti_sysbios_knl_Mailbox_Object__table__C                                   
1001bfe5  ti_sysbios_knl_Mailbox_Params__init__S                                    
1001abc5  ti_sysbios_knl_Mailbox_construct                                          
1001a945  ti_sysbios_knl_Mailbox_create                                             
1001c0f1  ti_sysbios_knl_Mailbox_delete                                             
1001c0f5  ti_sysbios_knl_Mailbox_destruct                                           
00001248  ti_sysbios_knl_Mailbox_maxTypeAlign__C                                    
1001a535  ti_sysbios_knl_Mailbox_pend__E                                            
1001b675  ti_sysbios_knl_Mailbox_postInit__I                                        
1001a0ed  ti_sysbios_knl_Mailbox_post__E                                            
1001c073  ti_sysbios_knl_Queue_Instance_init__E                                     
20001f94  ti_sysbios_knl_Queue_Module__root__V                                      
00001170  ti_sysbios_knl_Queue_Object__DESC__C                                      
1001cb20  ti_sysbios_knl_Queue_Object__PARAMS__C                                    
0000124c  ti_sysbios_knl_Queue_Object__count__C                                     
1001bb59  ti_sysbios_knl_Queue_Object__delete__S                                    
1001bcfd  ti_sysbios_knl_Queue_Object__destruct__S                                  
1001bb79  ti_sysbios_knl_Queue_Object__get__S                                       
00001250  ti_sysbios_knl_Queue_Object__table__C                                     
1001b6a1  ti_sysbios_knl_Queue_construct                                            
1001b6cd  ti_sysbios_knl_Queue_create                                               
1001c0f9  ti_sysbios_knl_Queue_delete                                               
1001bff1  ti_sysbios_knl_Queue_dequeue__E                                           
1001c0fd  ti_sysbios_knl_Queue_destruct                                             
1001c079  ti_sysbios_knl_Queue_elemClear__E                                         
1001bf4f  ti_sysbios_knl_Queue_empty__E                                             
1001bffd  ti_sysbios_knl_Queue_enqueue__E                                           
1001bd19  ti_sysbios_knl_Queue_get__E                                               
1001c101  ti_sysbios_knl_Queue_head__E                                              
1001c105  ti_sysbios_knl_Queue_next__E                                              
1001bd35  ti_sysbios_knl_Queue_put__E                                               
1001bf5d  ti_sysbios_knl_Queue_remove__E                                            
1001cb84  ti_sysbios_knl_Semaphore_Instance_State_pendQ__O                          
1001b7cd  ti_sysbios_knl_Semaphore_Instance_finalize__E                             
1001a685  ti_sysbios_knl_Semaphore_Instance_init__E                                 
20001f9c  ti_sysbios_knl_Semaphore_Module__root__V                                  
00001190  ti_sysbios_knl_Semaphore_Object__DESC__C                                  
1001cab4  ti_sysbios_knl_Semaphore_Object__PARAMS__C                                
1001b8d5  ti_sysbios_knl_Semaphore_Object__delete__S                                
1001bb99  ti_sysbios_knl_Semaphore_Object__destruct__S                              
1001c009  ti_sysbios_knl_Semaphore_Params__init__S                                  
1001b45d  ti_sysbios_knl_Semaphore_construct                                        
1001b2d1  ti_sysbios_knl_Semaphore_create                                           
1001c109  ti_sysbios_knl_Semaphore_delete                                           
1001c10d  ti_sysbios_knl_Semaphore_destruct                                         
00001254  ti_sysbios_knl_Semaphore_eventPost__C                                     
00001258  ti_sysbios_knl_Semaphore_eventSync__C                                     
1001b6f9  ti_sysbios_knl_Semaphore_pendTimeout__I                                   
10019b05  ti_sysbios_knl_Semaphore_pend__E                                          
1001a3e1  ti_sysbios_knl_Semaphore_post__E                                          
1001bf77  ti_sysbios_knl_Swi_Instance_finalize__E                                   
1001a9a5  ti_sysbios_knl_Swi_Instance_init__E                                       
20001cb8  ti_sysbios_knl_Swi_Module_State_0_readyQ__A                               
20001fa4  ti_sysbios_knl_Swi_Module__root__V                                        
200001c8  ti_sysbios_knl_Swi_Module__state__V                                       
1001c07f  ti_sysbios_knl_Swi_Module_startup__E                                      
000011b0  ti_sysbios_knl_Swi_Object__DESC__C                                        
1001ca44  ti_sysbios_knl_Swi_Object__PARAMS__C                                      
0000125c  ti_sysbios_knl_Swi_Object__count__C                                       
1001bbb9  ti_sysbios_knl_Swi_Object__delete__S                                      
1001bd51  ti_sysbios_knl_Swi_Object__destruct__S                                    
1001b725  ti_sysbios_knl_Swi_Object__get__S                                         
00001260  ti_sysbios_knl_Swi_Object__table__C                                       
20001e58  ti_sysbios_knl_Swi_Object__table__V                                       
1001c015  ti_sysbios_knl_Swi_Params__init__S                                        
1001ad79  ti_sysbios_knl_Swi_construct                                              
00004e4d  ti_sysbios_knl_Swi_construct2__E                                          
1001ac1d  ti_sysbios_knl_Swi_create                                                 
1001c111  ti_sysbios_knl_Swi_delete                                                 
1001c115  ti_sysbios_knl_Swi_destruct                                               
1001bf11  ti_sysbios_knl_Swi_disable__E                                             
1001bf21  ti_sysbios_knl_Swi_enabled__E                                             
000052b1  ti_sysbios_knl_Swi_getTrigger__E                                          
00001264  ti_sysbios_knl_Swi_numPriorities__C                                       
00004fbd  ti_sysbios_knl_Swi_or__E                                                  
1001c119  ti_sysbios_knl_Swi_postInit__I                                            
1001b011  ti_sysbios_knl_Swi_post__E                                                
1001a6ed  ti_sysbios_knl_Swi_restoreHwi__E                                          
1001b305  ti_sysbios_knl_Swi_restore__E                                             
1001adc9  ti_sysbios_knl_Swi_runLoop__I                                             
1001ac75  ti_sysbios_knl_Swi_run__I                                                 
1001ad25  ti_sysbios_knl_Swi_schedule__I                                            
1001c085  ti_sysbios_knl_Swi_startup__E                                             
20001208  ti_sysbios_knl_Task_Instance_State_0_stack__A                             
1001a059  ti_sysbios_knl_Task_Instance_finalize__E                                  
10019ce1  ti_sysbios_knl_Task_Instance_init__E                                      
20001fc8  ti_sysbios_knl_Task_Module_State_0_idleTask__A                            
20001ea8  ti_sysbios_knl_Task_Module_State_0_readyQ__A                              
1001cb88  ti_sysbios_knl_Task_Module_State_inactiveQ__O                             
20001fac  ti_sysbios_knl_Task_Module__root__V                                       
20000100  ti_sysbios_knl_Task_Module__state__V                                      
1001aa05  ti_sysbios_knl_Task_Module_startup__E                                     
000011d0  ti_sysbios_knl_Task_Object__DESC__C                                       
1001c978  ti_sysbios_knl_Task_Object__PARAMS__C                                     
00001268  ti_sysbios_knl_Task_Object__count__C                                      
1001bbd9  ti_sysbios_knl_Task_Object__delete__S                                     
1001bd6d  ti_sysbios_knl_Task_Object__destruct__S                                   
1001bbf9  ti_sysbios_knl_Task_Object__get__S                                        
0000126c  ti_sysbios_knl_Task_Object__table__C                                      
20001d8c  ti_sysbios_knl_Task_Object__table__V                                      
1001c021  ti_sysbios_knl_Task_Params__init__S                                       
1001c0ad  ti_sysbios_knl_Task_SupportProxy_Module__startupDone__S                   
1001c0ad  ti_sysbios_knl_Task_SupportProxy_Module__startupDone__S__mangled__        
1001bf9d  ti_sysbios_knl_Task_SupportProxy_getStackAlignment__E                     
1001bf9d  ti_sysbios_knl_Task_SupportProxy_getStackAlignment__E__mangled__          
1001b155  ti_sysbios_knl_Task_SupportProxy_start__E                                 
1001b155  ti_sysbios_knl_Task_SupportProxy_start__E__mangled__                      
1001c969  ti_sysbios_knl_Task_SupportProxy_swap__E                                  
1001c969  ti_sysbios_knl_Task_SupportProxy_swap__E__mangled__                       
00001270  ti_sysbios_knl_Task_allBlockedFunc__C                                     
1001b055  ti_sysbios_knl_Task_allBlockedFunction__I                                 
1001b339  ti_sysbios_knl_Task_blockI__E                                             
1001ae19  ti_sysbios_knl_Task_construct                                             
1001accd  ti_sysbios_knl_Task_create                                                
00001274  ti_sysbios_knl_Task_defaultStackHeap__C                                   
00001278  ti_sysbios_knl_Task_defaultStackSize__C                                   
1001c11d  ti_sysbios_knl_Task_delete                                                
1001c121  ti_sysbios_knl_Task_destruct                                              
1001bf31  ti_sysbios_knl_Task_disable__E                                            
1001c08b  ti_sysbios_knl_Task_enable__E                                             
1001bd89  ti_sysbios_knl_Task_enter__I                                              
1001b119  ti_sysbios_knl_Task_exit__E                                               
0000128c  ti_sysbios_knl_Task_initStackFlag__C                                      
0000127c  ti_sysbios_knl_Task_numConstructedTasks__C                                
1001a271  ti_sysbios_knl_Task_postInit__I                                           
1001b48d  ti_sysbios_knl_Task_processVitalTaskFlag__I                               
1001bc19  ti_sysbios_knl_Task_restoreHwi__E                                         
1001b7f5  ti_sysbios_knl_Task_restore__E                                            
1001ae69  ti_sysbios_knl_Task_schedule__I                                           
1001c02d  ti_sysbios_knl_Task_self__E                                               
1001bda5  ti_sysbios_knl_Task_sleepTimeout__I                                       
1001a5a5  ti_sysbios_knl_Task_sleep__E                                              
1001aa61  ti_sysbios_knl_Task_startCore__E                                          
1001c125  ti_sysbios_knl_Task_startup__E                                            
1001c971  ti_sysbios_knl_Task_swapReturn                                            
1001b751  ti_sysbios_knl_Task_unblockI__E                                           
1001bdf1  ti_sysbios_knl_Task_unblock__E                                            
1001b0d9  ti_sysbios_knl_Task_yield__E                                              
00001304  ti_sysbios_rom_ROM_ti_sysbios_family_arm_cc26xx_Timer_getCount64__E       
00001308  ti_sysbios_rom_ROM_ti_sysbios_family_arm_cc26xx_Timer_getCurrentTick__E   
0000130c  ti_sysbios_rom_ROM_ti_sysbios_family_arm_cc26xx_Timer_getMaxTicks__E      
00001310  ti_sysbios_rom_ROM_ti_sysbios_family_arm_cc26xx_Timer_initDevice__I       
00001314  ti_sysbios_rom_ROM_ti_sysbios_family_arm_cc26xx_Timer_setNextTick__E      
00001318  ti_sysbios_rom_ROM_ti_sysbios_family_arm_cc26xx_Timer_setThreshold__I     
0000131c  ti_sysbios_rom_ROM_ti_sysbios_family_arm_cc26xx_Timer_start__E            
00001320  ti_sysbios_rom_ROM_ti_sysbios_family_arm_cc26xx_TimestampProvider_get32__E
00001324  ti_sysbios_rom_ROM_xdc_runtime_Startup_getState__I                        
00001328  ti_sysbios_rom_ROM_xdc_runtime_System_SupportProxy_abort__E               
0000132c  ti_sysbios_rom_ROM_xdc_runtime_System_SupportProxy_exit__E                
10019b00  ti_sysbios_rom_cortexm_cc26xx_r2_CC26xx_REVISION__C                       
00004df7  ti_sysbios_rom_cortexm_cc26xx_r2_CC26xx_badRomRevision__E                 
00004fd5  ti_sysbios_rom_cortexm_cc26xx_r2_CC26xx_checkRevision__E                  
20001a84  uart                                                                      
00000664  uartCC26XXHWAttrs                                                         
200015fc  uartCC26XXObjects                                                         
200019e0  uartCC26XXRingBuffer                                                      
000012a0  xdc_runtime_Assert_E_assertFailed__C                                      
1001c465  xdc_runtime_Assert_raise__I                                               
1001c5b9  xdc_runtime_Core_assignLabel__I                                           
1001c4ad  xdc_runtime_Core_assignParams__I                                          
1001c4f5  xdc_runtime_Core_constructObject__I                                       
1001c2c9  xdc_runtime_Core_createObject__I                                          
1001c3b5  xdc_runtime_Core_deleteObject__I                                          
1001c6a5  xdc_runtime_Core_destructObject__I                                        
000012a4  xdc_runtime_Error_E_memory__C                                             
20001ec8  xdc_runtime_Error_IgnoreBlock                                             
20000204  xdc_runtime_Error_Module__state__V                                        
1001c6bd  xdc_runtime_Error_check__E                                                
00004fed  xdc_runtime_Error_init__E                                                 
000012f8  xdc_runtime_Error_maxDepth__C                                             
00002cf9  xdc_runtime_Error_policyDefault__E                                        
000012a8  xdc_runtime_Error_policyFxn__C                                            
1001c413  xdc_runtime_Error_policySpin__E                                           
00001300  xdc_runtime_Error_policy__C                                               
000012ac  xdc_runtime_Error_raiseHook__C                                            
1001c66d  xdc_runtime_Error_raiseX__E                                               
000041e9  xdc_runtime_Error_setX__E                                                 
1001c795  xdc_runtime_Gate_enterSystem__E                                           
1001c789  xdc_runtime_Gate_leaveSystem__E                                           
000012b0  xdc_runtime_IGateProvider_Interface__BASE__C                              
000012b4  xdc_runtime_IHeap_Interface__BASE__C                                      
000012b8  xdc_runtime_IModule_Interface__BASE__C                                    
1001b999  xdc_runtime_Main_Module_GateProxy_Handle__label__S                        
1001c0b1  xdc_runtime_Main_Module_GateProxy_query__E                                
1001ba39  xdc_runtime_Memory_HeapProxy_Handle__label__S                             
1001ba39  xdc_runtime_Memory_HeapProxy_Handle__label__S__mangled__                  
1001ba59  xdc_runtime_Memory_HeapProxy_Object__delete__S                            
1001c775  xdc_runtime_Memory_HeapProxy_alloc__E                                     
1001c77f  xdc_runtime_Memory_HeapProxy_free__E                                      
000012fa  xdc_runtime_Memory_Module__id__C                                          
20000200  xdc_runtime_Memory_Module__state__V                                       
1001c349  xdc_runtime_Memory_alloc__E                                               
1001c751  xdc_runtime_Memory_calloc__E                                              
000012bc  xdc_runtime_Memory_defaultHeapInstance__C                                 
1001c705  xdc_runtime_Memory_free__E                                                
1001c75d  xdc_runtime_Memory_getMaxDefaultTypeAlign__E                              
1001c689  xdc_runtime_Memory_valloc__E                                              
200001f0  xdc_runtime_Startup_Module__state__V                                      
00000001  xdc_runtime_Startup__EXECFXN__C                                           
00000001  xdc_runtime_Startup__RESETFXN__C                                          
000012c0  xdc_runtime_Startup_execImpl__C                                           
1001c415  xdc_runtime_Startup_exec__E                                               
0000515f  xdc_runtime_Startup_exec__I                                               
000006fc  xdc_runtime_Startup_firstFxns__A                                          
00001290  xdc_runtime_Startup_firstFxns__C                                          
00003c59  xdc_runtime_Startup_getState__I                                           
00001298  xdc_runtime_Startup_lastFxns__C                                           
000012c4  xdc_runtime_Startup_maxPasses__C                                          
000052bd  xdc_runtime_Startup_reset__I                                              
1001c769  xdc_runtime_Startup_rtsDone__E                                            
000006b0  xdc_runtime_Startup_sfxnRts__A                                            
000012c8  xdc_runtime_Startup_sfxnRts__C                                            
00000618  xdc_runtime_Startup_sfxnTab__A                                            
000012cc  xdc_runtime_Startup_sfxnTab__C                                            
000012d0  xdc_runtime_Startup_startModsFxn__C                                       
1001c129  xdc_runtime_Startup_startMods__I                                          
000012d4  xdc_runtime_SysCallback_abortFxn__C                                       
1001c715  xdc_runtime_SysCallback_abort__E                                          
0000524f  xdc_runtime_SysCallback_defaultAbort                                      
0000538b  xdc_runtime_SysCallback_defaultExit                                       
000012d8  xdc_runtime_SysCallback_exitFxn__C                                        
1001c725  xdc_runtime_SysCallback_exit__E                                           
20001408  xdc_runtime_SysMin_Module_State_0_outbuf__A                               
20001f38  xdc_runtime_SysMin_Module__state__V                                       
00004d7d  xdc_runtime_SysMin_Module_startup__E                                      
000048f9  xdc_runtime_SysMin_abort__E                                               
0000072c  xdc_runtime_SysMin_bufSize__C                                             
00004e69  xdc_runtime_SysMin_exit__E                                                
00000712  xdc_runtime_SysMin_flushAtExit__C                                         
0000422d  xdc_runtime_SysMin_flush__E                                               
00000730  xdc_runtime_SysMin_outputFunc__C                                          
00004c99  xdc_runtime_SysMin_output__I                                              
00004635  xdc_runtime_SysMin_putch__E                                               
1001b999  xdc_runtime_System_Module_GateProxy_Handle__label__S                      
1001b999  xdc_runtime_System_Module_GateProxy_Handle__label__S__mangled__           
1001b9b9  xdc_runtime_System_Module_GateProxy_Object__delete__S                     
1001c799  xdc_runtime_System_Module_GateProxy_enter__E                              
1001c79d  xdc_runtime_System_Module_GateProxy_leave__E                              
1001c0b1  xdc_runtime_System_Module_GateProxy_query__E                              
1001c0b1  xdc_runtime_System_Module_GateProxy_query__E__mangled__                   
20001fb4  xdc_runtime_System_Module_State_0_atexitHandlers__A                       
200001f8  xdc_runtime_System_Module__state__V                                       
1001c78f  xdc_runtime_System_Module_startup__E                                      
000048f9  xdc_runtime_System_SupportProxy_abort__E                                  
00004e69  xdc_runtime_System_SupportProxy_exit__E                                   
0000422d  xdc_runtime_System_SupportProxy_flush__E                                  
00004635  xdc_runtime_System_SupportProxy_putch__E                                  
000012dc  xdc_runtime_System_abortFxn__C                                            
1001c7a1  xdc_runtime_System_abortSpin__E                                           
1001c64d  xdc_runtime_System_abort__E                                               
1001c581  xdc_runtime_System_atexit__E                                              
000012e0  xdc_runtime_System_exitFxn__C                                             
1001c7a3  xdc_runtime_System_exitSpin__E                                            
1001c6d5  xdc_runtime_System_exit__E                                                
0000422d  xdc_runtime_System_flush__E                                               
000012e4  xdc_runtime_System_maxAtexitHandlers__C                                   
1001c5ed  xdc_runtime_System_processAtExit__E                                       
000012fc  xdc_runtime_Text_charCnt__C                                               
00000711  xdc_runtime_Text_charTab__A                                               
000012e8  xdc_runtime_Text_charTab__C                                               
1001c621  xdc_runtime_Text_cordText__E                                              
000012fe  xdc_runtime_Text_isLoaded__C                                              
000012ec  xdc_runtime_Text_nameEmpty__C                                             
000012f0  xdc_runtime_Text_nameStatic__C                                            
000012f4  xdc_runtime_Text_nameUnknown__C                                           
1001c6ed  xdc_runtime_Text_ropeText__E                                              
1001c735  xdc_runtime_Timestamp_SupportProxy_get32__E                               
00005205  xdc_runtime_Timestamp_SupportProxy_get32__E__mangled__                    
1001b77d  xdc_runtime_Timestamp_SupportProxy_get64__E                               
1001b77d  xdc_runtime_Timestamp_SupportProxy_get64__E__mangled__                    
1001bf6b  xdc_runtime_Timestamp_SupportProxy_getFreq__E                             
1001bf6b  xdc_runtime_Timestamp_SupportProxy_getFreq__E__mangled__                  
1001c735  xdc_runtime_Timestamp_get32__E                                            
1001c735  xdc_runtime_Timestamp_get32__E                                            
1001b77d  xdc_runtime_Timestamp_get64__E                                            
1001b77d  xdc_runtime_Timestamp_get64__E                                            
1001bf6b  xdc_runtime_Timestamp_getFreq__E                                          
1001bf6b  xdc_runtime_Timestamp_getFreq__E                                          


GLOBAL SYMBOLS: SORTED BY Symbol Address 

address   name                                                                      
-------   ----                                                                      
00000000  __ASM__                                                                   
00000000  __TI_static_base__                                                        
00000000  ti_sysbios_family_arm_m3_Hwi_resetVectors                                 
00000001  xdc_runtime_Startup__EXECFXN__C                                           
00000001  xdc_runtime_Startup__RESETFXN__C                                          
00000071  __ISA__                                                                   
00000083  __PLAT__                                                                  
000000aa  __TARG__                                                                  
000000cf  __TRDR__                                                                  
00000300  __STACK_SIZE                                                              
00000480  resourceDB                                                                
00000554  inPinTypes                                                                
00000560  outPinStrengths                                                           
0000056c  outPinTypes                                                               
00000594  scifDriverSetup                                                           
000005c4  BoardGpioInitTable                                                        
000005f0  UARTCC26XX_fxnTable                                                       
00000618  xdc_runtime_Startup_sfxnTab__A                                            
00000640  UART_defaultParams                                                        
00000664  uartCC26XXHWAttrs                                                         
00000684  PowerCC26XX_config                                                        
0000069c  GPIOCC26XX_config                                                         
000006b0  xdc_runtime_Startup_sfxnRts__A                                            
000006e4  BoardGpioInitTable1                                                       
000006f0  UART_config                                                               
000006fc  xdc_runtime_Startup_firstFxns__A                                          
00000708  ADCBuf_count                                                              
00000709  ADC_count                                                                 
0000070a  Display_count                                                             
0000070b  I2C_count                                                                 
0000070c  NVS_count                                                                 
0000070d  PWM_count                                                                 
0000070e  SPI_count                                                                 
0000070f  UART_count                                                                
00000710  Watchdog_count                                                            
00000711  xdc_runtime_Text_charTab__A                                               
00000712  xdc_runtime_SysMin_flushAtExit__C                                         
00000714  PINCC26XX_hwAttrs                                                         
0000071c  ti_sysbios_family_arm_m3_Hwi_swiDisable__C                                
00000720  ti_sysbios_family_arm_m3_Hwi_swiRestoreHwi__C                             
00000724  ti_sysbios_knl_Clock_tickPeriod__C                                        
00000728  ti_sysbios_knl_Idle_funcList__A                                           
0000072c  xdc_runtime_SysMin_bufSize__C                                             
00000730  xdc_runtime_SysMin_outputFunc__C                                          
00000914  __TI_Handler_Table_Base                                                   
00000920  __TI_Handler_Table_Limit                                                  
0000095c  __TI_CINIT_Base                                                           
000009c4  __TI_CINIT_Limit                                                          
00001000  ti_sysbios_heaps_HeapMem_Module__FXNS__C                                  
00001028  ti_sysbios_gates_GateHwi_Module__FXNS__C                                  
0000104c  ti_sysbios_gates_GateMutex_Module__FXNS__C                                
00001070  ti_sysbios_family_arm_m3_Hwi_Object__DESC__C                              
00001090  ti_sysbios_gates_GateHwi_Object__DESC__C                                  
000010b0  ti_sysbios_gates_GateMutex_Object__DESC__C                                
000010d0  ti_sysbios_hal_Hwi_Object__DESC__C                                        
000010f0  ti_sysbios_heaps_HeapMem_Object__DESC__C                                  
00001110  ti_sysbios_knl_Clock_Object__DESC__C                                      
00001130  ti_sysbios_knl_Event_Object__DESC__C                                      
00001150  ti_sysbios_knl_Mailbox_Object__DESC__C                                    
00001170  ti_sysbios_knl_Queue_Object__DESC__C                                      
00001190  ti_sysbios_knl_Semaphore_Object__DESC__C                                  
000011b0  ti_sysbios_knl_Swi_Object__DESC__C                                        
000011d0  ti_sysbios_knl_Task_Object__DESC__C                                       
000011f0  ti_sysbios_knl_Idle_funcList__C                                           
000011f8  ti_sysbios_family_arm_cc26xx_Timer_startupNeeded__C                       
000011fc  ti_sysbios_family_arm_m3_Hwi_E_alreadyDefined__C                          
00001200  ti_sysbios_family_arm_m3_Hwi_E_hwiLimitExceeded__C                        
00001204  ti_sysbios_family_arm_m3_Hwi_NUM_INTERRUPTS__C                            
00001208  ti_sysbios_family_arm_m3_Hwi_Object__count__C                             
0000120c  ti_sysbios_family_arm_m3_Hwi_Object__table__C                             
00001210  ti_sysbios_family_arm_m3_Hwi_ccr__C                                       
00001214  ti_sysbios_family_arm_m3_Hwi_excHandlerFunc__C                            
00001218  ti_sysbios_family_arm_m3_Hwi_nullIsrFunc__C                               
0000121c  ti_sysbios_family_arm_m3_Hwi_numSparseInterrupts__C                       
00001220  ti_sysbios_family_arm_m3_Hwi_priGroup__C                                  
00001224  ti_sysbios_family_arm_m3_TaskSupport_stackAlignment__C                    
00001228  ti_sysbios_heaps_HeapMem_E_memory__C                                      
0000122c  ti_sysbios_heaps_HeapMem_Module__gateObj__C                               
00001230  ti_sysbios_heaps_HeapMem_Object__count__C                                 
00001234  ti_sysbios_heaps_HeapMem_Object__table__C                                 
00001238  ti_sysbios_heaps_HeapMem_reqAlign__C                                      
0000123c  ti_sysbios_knl_Clock_triggerClock__C                                      
00001240  ti_sysbios_knl_Mailbox_Object__count__C                                   
00001244  ti_sysbios_knl_Mailbox_Object__table__C                                   
00001248  ti_sysbios_knl_Mailbox_maxTypeAlign__C                                    
0000124c  ti_sysbios_knl_Queue_Object__count__C                                     
00001250  ti_sysbios_knl_Queue_Object__table__C                                     
00001254  ti_sysbios_knl_Semaphore_eventPost__C                                     
00001258  ti_sysbios_knl_Semaphore_eventSync__C                                     
0000125c  ti_sysbios_knl_Swi_Object__count__C                                       
00001260  ti_sysbios_knl_Swi_Object__table__C                                       
00001264  ti_sysbios_knl_Swi_numPriorities__C                                       
00001268  ti_sysbios_knl_Task_Object__count__C                                      
0000126c  ti_sysbios_knl_Task_Object__table__C                                      
00001270  ti_sysbios_knl_Task_allBlockedFunc__C                                     
00001274  ti_sysbios_knl_Task_defaultStackHeap__C                                   
00001278  ti_sysbios_knl_Task_defaultStackSize__C                                   
0000127c  ti_sysbios_knl_Task_numConstructedTasks__C                                
00001280  ti_sysbios_family_arm_cc26xx_Timer_Module__id__C                          
00001282  ti_sysbios_family_arm_cc26xx_TimestampProvider_useClockTimer__C           
00001284  ti_sysbios_family_arm_m3_Hwi_Module__id__C                                
00001286  ti_sysbios_gates_GateHwi_Module__id__C                                    
00001288  ti_sysbios_gates_GateMutex_Module__id__C                                  
0000128a  ti_sysbios_heaps_HeapMem_Module__id__C                                    
0000128c  ti_sysbios_knl_Task_initStackFlag__C                                      
0000128e  ti_sysbios_knl_Clock_tickMode__C                                          
00001290  xdc_runtime_Startup_firstFxns__C                                          
00001298  xdc_runtime_Startup_lastFxns__C                                           
000012a0  xdc_runtime_Assert_E_assertFailed__C                                      
000012a4  xdc_runtime_Error_E_memory__C                                             
000012a8  xdc_runtime_Error_policyFxn__C                                            
000012ac  xdc_runtime_Error_raiseHook__C                                            
000012b0  xdc_runtime_IGateProvider_Interface__BASE__C                              
000012b4  xdc_runtime_IHeap_Interface__BASE__C                                      
000012b8  xdc_runtime_IModule_Interface__BASE__C                                    
000012bc  xdc_runtime_Memory_defaultHeapInstance__C                                 
000012c0  xdc_runtime_Startup_execImpl__C                                           
000012c4  xdc_runtime_Startup_maxPasses__C                                          
000012c8  xdc_runtime_Startup_sfxnRts__C                                            
000012cc  xdc_runtime_Startup_sfxnTab__C                                            
000012d0  xdc_runtime_Startup_startModsFxn__C                                       
000012d4  xdc_runtime_SysCallback_abortFxn__C                                       
000012d8  xdc_runtime_SysCallback_exitFxn__C                                        
000012dc  xdc_runtime_System_abortFxn__C                                            
000012e0  xdc_runtime_System_exitFxn__C                                             
000012e4  xdc_runtime_System_maxAtexitHandlers__C                                   
000012e8  xdc_runtime_Text_charTab__C                                               
000012ec  xdc_runtime_Text_nameEmpty__C                                             
000012f0  xdc_runtime_Text_nameStatic__C                                            
000012f4  xdc_runtime_Text_nameUnknown__C                                           
000012f8  xdc_runtime_Error_maxDepth__C                                             
000012fa  xdc_runtime_Memory_Module__id__C                                          
000012fc  xdc_runtime_Text_charCnt__C                                               
000012fe  xdc_runtime_Text_isLoaded__C                                              
00001300  xdc_runtime_Error_policy__C                                               
00001304  ti_sysbios_rom_ROM_ti_sysbios_family_arm_cc26xx_Timer_getCount64__E       
00001308  ti_sysbios_rom_ROM_ti_sysbios_family_arm_cc26xx_Timer_getCurrentTick__E   
0000130c  ti_sysbios_rom_ROM_ti_sysbios_family_arm_cc26xx_Timer_getMaxTicks__E      
00001310  ti_sysbios_rom_ROM_ti_sysbios_family_arm_cc26xx_Timer_initDevice__I       
00001314  ti_sysbios_rom_ROM_ti_sysbios_family_arm_cc26xx_Timer_setNextTick__E      
00001318  ti_sysbios_rom_ROM_ti_sysbios_family_arm_cc26xx_Timer_setThreshold__I     
0000131c  ti_sysbios_rom_ROM_ti_sysbios_family_arm_cc26xx_Timer_start__E            
00001320  ti_sysbios_rom_ROM_ti_sysbios_family_arm_cc26xx_TimestampProvider_get32__E
00001324  ti_sysbios_rom_ROM_xdc_runtime_Startup_getState__I                        
00001328  ti_sysbios_rom_ROM_xdc_runtime_System_SupportProxy_abort__E               
0000132c  ti_sysbios_rom_ROM_xdc_runtime_System_SupportProxy_exit__E                
00001331  PowerCC26XX_auxISR                                                        
00001645  Power_sleep                                                               
00001889  NOROM_SysCtrlSetRechargeBeforePowerDown                                   
00001a95  __aeabi_uldivmod                                                          
00001c89  PIN_init                                                                  
00001e45  PowerCC26XX_doCalibrate                                                   
00001fd5  UARTCC26XX_open                                                           
00002131  Power_init                                                                
0000225d  UARTCC26XX_read                                                           
00002379  UARTCC26XX_hwiIntFxn                                                      
0000248d  scifInit                                                                  
0000258d  UARTCC26XX_write                                                          
00002689  GPIO_setConfig                                                            
00002779  PowerCC26XX_standbyPolicy                                                 
00002a1d  GPIO_init                                                                 
00002ad9  Power_releaseDependency                                                   
00002b95  Power_setDependency                                                       
00002cf9  xdc_runtime_Error_policyDefault__E                                        
00002da9  NOROM_SetupTrimDevice                                                     
00002da9  ti_sysbios_family_arm_cc26xx_Boot_trimDevice                              
00002ef9  __TI_auto_init                                                            
00002f99  __aeabi_memcpy                                                            
00002f99  __aeabi_memcpy4                                                           
00002f99  __aeabi_memcpy8                                                           
00002f99  memcpy                                                                    
00003035  PIN_open                                                                  
00003165  ti_sysbios_knl_Clock_workFuncDynamic__E                                   
00003289  UARTCC26XX_close                                                          
00003315  UARTCC26XX_writeCancel                                                    
000033a1  scifInitIo                                                                
000034b9  main                                                                      
00003539  __aeabi_memclr                                                            
00003539  __aeabi_memclr4                                                           
00003539  __aeabi_memclr8                                                           
0000353b  __aeabi_memset                                                            
0000353b  __aeabi_memset4                                                           
0000353b  __aeabi_memset8                                                           
00003541  memset                                                                    
0000362b  scCtrlReadyCallback                                                       
0000362d  scifUartSetBaudRate                                                       
000036a1  ti_sysbios_family_arm_cc26xx_Timer_start__E                               
00003715  NOROM_SysCtrlAdjustRechargeAfterPowerDown                                 
000037f5  NOROM_OSCHF_AttemptToSwitchToXosc                                         
00003861  PowerCC26XX_initiateCalibration                                           
00003939  NOROM_SysCtrl_DCDC_VoltageConditionalControl                              
000039a1  UARTCC26XX_readCancel                                                     
00003a09  __TI_decompress_lzss                                                      
00003a71  __TI_writemsg                                                             
00003a9f  C$$IO$$                                                                   
00003aa3  __TI_readmsg                                                              
00003ad9  PIN_add                                                                   
00003b3d  taskFxn1                                                                  
00003ba1  PowerCC26XX_RCOSC_clockFunc                                               
00003bfd  PowerCC26XX_calibrate                                                     
00003c59  xdc_runtime_Startup_getState__I                                           
00003cb5  PIN_remove                                                                
00003d0d  UARTCC26XX_control                                                        
00003d65  HOSTwrite                                                                 
00003dbd  scifReinitIo                                                              
00003e15  scifUninitIo                                                              
00003e6d  taskFxn                                                                   
00003ec5  GPIO_write                                                                
00003fb5  copy_in                                                                   
00004001  ClockP_construct                                                          
00004049  PIN_setOutputEnable                                                       
00004091  ti_sysbios_family_arm_cc26xx_Timer_setThreshold__I                        
000040d9  NOROM_OSCHF_SwitchToRcOscTurnOffXosc                                      
0000411d  RingBuf_put                                                               
00004161  ResetISR                                                                  
00004161  _c_int00                                                                  
000041e9  xdc_runtime_Error_setX__E                                                 
0000422d  xdc_runtime_SysMin_flush__E                                               
0000422d  xdc_runtime_System_SupportProxy_flush__E                                  
0000422d  xdc_runtime_System_flush__E                                               
000042b1  UART_init                                                                 
000042f1  UART_open                                                                 
00004331  scifUartGetRxFifoCount                                                    
00004371  HwiP_construct                                                            
000043af  RingBuf_get                                                               
000043ed  NOROM_OSC_HPOSCRelativeFrequencyOffsetGet                                 
00004429  SwiP_construct                                                            
000044a1  scifUartRxGetChar                                                         
000044dd  scifUartTxPutChar                                                         
00004519  ti_sysbios_family_arm_m3_Hwi_construct2__E                                
00004555  GPIO_enableInt                                                            
0000458d  PIN_setOutputValue                                                        
000045c5  UARTCC26XX_swiIntFxn                                                      
000045fd  ti_sysbios_family_arm_cc26xx_Timer_getCurrentTick__E                      
00004635  xdc_runtime_SysMin_putch__E                                               
00004635  xdc_runtime_System_SupportProxy_putch__E                                  
0000466d  GPIO_setCallback                                                          
000046a1  PIN_setConfig                                                             
000046d5  Power_releaseConstraint                                                   
00004709  scifAckAlertEvents                                                        
0000473d  scifOsalInit                                                              
00004771  ti_sysbios_family_arm_cc26xx_Timer_initDevice__I                          
000047a5  scTaskAlertCallback                                                       
000047d7  ti_sysbios_family_arm_cc26xx_Timer_setNextTick__E                         
00004809  Power_setConstraint                                                       
00004899  ti_sysbios_BIOS_atExitFunc__I                                             
000048c9  ti_sysbios_BIOS_startFunc__I                                              
000048f9  xdc_runtime_SysMin_abort__E                                               
000048f9  xdc_runtime_System_SupportProxy_abort__E                                  
00004985  NOROM_ChipInfo_GetChipFamily                                              
000049b1  PINCC26XX_setMux                                                          
000049dd  SemaphoreP_constructBinary                                                
00004a09  SemaphoreP_createBinary                                                   
00004a8d  ti_sysbios_knl_Clock_getTicksUntilInterrupt__E                            
00004ab9  NOROM_ChipInfo_GetChipType                                                
00004ae1  Power_registerNotify                                                      
00004b09  SafeHapiVoid                                                              
00004b59  GPIO_hwiIntFxn                                                            
00004b7d  NOROM_OSCHF_TurnOnXosc                                                    
00004ba1  Uart_rxcallback                                                           
00004bc5  scifUartSetEventMask                                                      
00004be9  ti_sysbios_BIOS_registerRTSLock__I                                        
00004c0d  ti_sysbios_BIOS_removeRTSLock__I                                          
00004c31  ti_sysbios_family_arm_cc26xx_Timer_getMaxTicks__E                         
00004c55  List_put                                                                  
00004c77  NOROM_UARTConfigSetExpClk                                                 
00004c99  xdc_runtime_SysMin_output__I                                              
00004cbb  ti_sysbios_BIOS_nullFunc__I                                               
00004cbd  NOROM_UARTDisable                                                         
00004cdd  PowerCC26XX_schedulerDisable                                              
00004cfd  PowerCC26XX_schedulerRestore                                              
00004d1d  Power_unregisterNotify                                                    
00004d3d  ti_sysbios_BIOS_rtsLock__I                                                
00004d5d  ti_sysbios_family_arm_cc26xx_Timer_dynamicStub__E                         
00004d7d  xdc_runtime_SysMin_Module_startup__E                                      
00004d9d  PIN_close                                                                 
00004dbb  Power_getTransitionLatency                                                
00004df7  ti_sysbios_rom_cortexm_cc26xx_r2_CC26xx_badRomRevision__E                 
00004e31  ti_sysbios_family_arm_m3_Hwi_clearInterrupt__E                            
00004e31  ti_sysbios_hal_Hwi_HwiProxy_clearInterrupt__E                             
00004e31  ti_sysbios_hal_Hwi_clearInterrupt__E                                      
00004e4d  ti_sysbios_knl_Swi_construct2__E                                          
00004e69  xdc_runtime_SysMin_exit__E                                                
00004e69  xdc_runtime_System_SupportProxy_exit__E                                   
00004e85  NOROM_ChipInfo_GetPackageType                                             
00004e9d  Power_idleFunc                                                            
00004eb5  UARTCC26XX_init                                                           
00004ecd  UART_Params_init                                                          
00004efd  _args_main                                                                
00004f15  __aeabi_lmul                                                              
00004f2d  scifClearAlertIntSource                                                   
00004f45  scifUartRxEnable                                                          
00004f5d  scifUartSetRxEnableReqIdleCount                                           
00004f75  scifUartSetRxFifoThr                                                      
00004f8d  scifUartSetRxTimeout                                                      
00004fa5  ti_sysbios_BIOS_rtsUnlock__I                                              
00004fbd  ti_sysbios_knl_Swi_or__E                                                  
00004fd5  ti_sysbios_rom_cortexm_cc26xx_r2_CC26xx_checkRevision__E                  
00004fed  xdc_runtime_Error_init__E                                                 
00005005  List_remove                                                               
0000501b  ti_sysbios_BIOS_errorRaiseHook__I                                         
00005031  ti_sysbios_BIOS_exitFunc__I                                               
00005089  NOROM_IOCIntEnable                                                        
000050b1  _register_unlock                                                          
000050b7  _register_lock                                                            
000050bf  _nop                                                                      
000050c5  scifOsalRegisterCtrlReadyCallback                                         
000050d9  scifOsalRegisterTaskAlertCallback                                         
00005101  ti_sysbios_family_arm_cc26xx_Timer_getCount64__E                          
00005115  ti_sysbios_knl_Clock_doTick__I                                            
00005129  RingBuf_construct                                                         
0000513b  SemaphoreP_pend                                                           
0000514d  scifExecuteTasksOnceNbl                                                   
0000515f  xdc_runtime_Startup_exec__I                                               
00005171  HwiP_Params_init                                                          
00005181  PINCC26XX_getPinCount                                                     
00005191  SwiP_Params_init                                                          
000051b1  NOROM_ThisLibraryIsFor_CC26x0R2_HaltIfViolated                            
000051bf  NOROM_UARTCharGetNonBlocking                                              
000051cd  NOROM_UARTCharPutNonBlocking                                              
000051db  __TI_decompress_none                                                      
00005205  ti_sysbios_family_arm_cc26xx_TimestampProvider_get32__E                   
00005205  xdc_runtime_Timestamp_SupportProxy_get32__E__mangled__                    
00005213  List_empty                                                                
0000521f  NOROM_CPUcpsid                                                            
0000522b  NOROM_CPUcpsie                                                            
00005237  NOROM_OSC_HPOSCRelativeFrequencyOffsetToRFCoreFormatConvert               
00005243  PIN_registerIntCb                                                         
0000524f  xdc_runtime_SysCallback_defaultAbort                                      
00005251  Power_getConstraintMask                                                   
0000525d  Power_getDependencyCount                                                  
00005269  SemaphoreP_delete                                                         
00005275  __TI_zero_init                                                            
0000528d  scifOsalLeaveCriticalSection                                              
00005299  scifUartClearEvents                                                       
000052b1  ti_sysbios_knl_Swi_getTrigger__E                                          
000052bd  xdc_runtime_Startup_reset__I                                              
000052c9  UART_read                                                                 
000052d3  UART_write                                                                
00005305  scifOsalDisableTaskAlertInt                                               
0000530f  scifOsalEnableTaskAlertInt                                                
00005321  scifOsalEnterCriticalSection                                              
00005331  ClockP_Params_init                                                        
00005337  UARTCC26XX_readPolling                                                    
0000533d  UARTCC26XX_writePolling                                                   
00005347  ClockP_destruct                                                           
0000534b  ClockP_getCpuFreq                                                         
0000534f  ClockP_setTimeout                                                         
00005353  ClockP_start                                                              
00005357  ClockP_stop                                                               
0000535b  HwiP_destruct                                                             
0000535f  HwiP_disable                                                              
00005363  List_head                                                                 
00005367  List_next                                                                 
0000536b  SemaphoreP_destruct                                                       
0000536f  SemaphoreP_post                                                           
00005373  SwiP_destruct                                                             
00005377  SwiP_disable                                                              
0000537b  SwiP_getTrigger                                                           
0000537f  SwiP_or                                                                   
00005383  SwiP_post                                                                 
0000538b  xdc_runtime_SysCallback_defaultExit                                       
0001ffa8  __ccfg                                                                    
10019b00  ti_sysbios_rom_cortexm_cc26xx_r2_CC26xx_REVISION__C                       
10019b05  ti_sysbios_knl_Semaphore_pend__E                                          
10019bf9  ti_sysbios_knl_Event_pend__E                                              
10019ce1  ti_sysbios_knl_Task_Instance_init__E                                      
10019dad  ti_sysbios_knl_Mailbox_Instance_init__E                                   
10019e75  ti_sysbios_family_arm_m3_Hwi_postInit__I                                  
10019f25  ti_sysbios_family_arm_cc26xx_Timer_periodicStub__E                        
10019fc1  ti_sysbios_family_arm_m3_Hwi_Instance_init__E                             
1001a059  ti_sysbios_knl_Task_Instance_finalize__E                                  
1001a0ed  ti_sysbios_knl_Mailbox_post__E                                            
1001a171  ti_sysbios_family_arm_m3_Hwi_initNVIC__E                                  
1001a1f1  ti_sysbios_knl_Clock_startI__E                                            
1001a271  ti_sysbios_knl_Task_postInit__I                                           
1001a2f1  ti_sysbios_knl_Clock_walkQueueDynamic__E                                  
1001a369  ti_sysbios_knl_Clock_workFunc__E                                          
1001a3e1  ti_sysbios_knl_Semaphore_post__E                                          
1001a455  ti_sysbios_knl_Event_post__E                                              
1001a4c5  ti_sysbios_knl_Mailbox_Instance_finalize__E                               
1001a535  ti_sysbios_knl_Mailbox_pend__E                                            
1001a5a5  ti_sysbios_knl_Task_sleep__E                                              
1001a615  ti_sysbios_heaps_HeapMem_allocUnprotected__E                              
1001a683  ti_sysbios_BIOS_linkedWithIncorrectBootLibrary__E                         
1001a685  ti_sysbios_knl_Semaphore_Instance_init__E                                 
1001a6ed  ti_sysbios_knl_Swi_restoreHwi__E                                          
1001a755  ti_sysbios_family_arm_m3_Hwi_Instance_finalize__E                         
1001a7b9  ti_sysbios_family_arm_m3_Hwi_Object__create__S                            
1001a81d  ti_sysbios_family_arm_m3_Hwi_dispatchC__I                                 
1001a881  ti_sysbios_hal_Hwi_create                                                 
1001a8e5  ti_sysbios_family_arm_m3_Hwi_create                                       
1001a945  ti_sysbios_knl_Mailbox_create                                             
1001a9a5  ti_sysbios_knl_Swi_Instance_init__E                                       
1001aa05  ti_sysbios_knl_Task_Module_startup__E                                     
1001aa61  ti_sysbios_knl_Task_startCore__E                                          
1001aabd  ti_sysbios_family_arm_m3_Hwi_construct                                    
1001ab15  ti_sysbios_heaps_HeapMem_alloc__E                                         
1001ab6d  ti_sysbios_heaps_HeapMem_freeUnprotected__E                               
1001abc5  ti_sysbios_knl_Mailbox_construct                                          
1001ac1d  ti_sysbios_knl_Swi_create                                                 
1001ac75  ti_sysbios_knl_Swi_run__I                                                 
1001accd  ti_sysbios_knl_Task_create                                                
1001ad25  ti_sysbios_knl_Swi_schedule__I                                            
1001ad79  ti_sysbios_knl_Swi_construct                                              
1001adc9  ti_sysbios_knl_Swi_runLoop__I                                             
1001ae19  ti_sysbios_knl_Task_construct                                             
1001ae69  ti_sysbios_knl_Task_schedule__I                                           
1001aeb5  ti_sysbios_family_arm_m3_Hwi_Module_startup__E                            
1001aefd  ti_sysbios_heaps_HeapMem_getStats__E                                      
1001af45  ti_sysbios_family_arm_m3_Hwi_disableInterrupt__E                          
1001af45  ti_sysbios_hal_Hwi_HwiProxy_disableInterrupt__E                           
1001af45  ti_sysbios_hal_Hwi_HwiProxy_disableInterrupt__E__mangled__                
1001af45  ti_sysbios_hal_Hwi_disableInterrupt__E                                    
1001af45  ti_sysbios_hal_Hwi_disableInterrupt__E                                    
1001af89  ti_sysbios_family_arm_m3_Hwi_enableInterrupt__E                           
1001af89  ti_sysbios_hal_Hwi_HwiProxy_enableInterrupt__E                            
1001af89  ti_sysbios_hal_Hwi_HwiProxy_enableInterrupt__E__mangled__                 
1001af89  ti_sysbios_hal_Hwi_enableInterrupt__E                                     
1001af89  ti_sysbios_hal_Hwi_enableInterrupt__E                                     
1001afcd  ti_sysbios_knl_Mailbox_Module_startup__E                                  
1001b011  ti_sysbios_knl_Swi_post__E                                                
1001b055  ti_sysbios_knl_Task_allBlockedFunction__I                                 
1001b099  ti_sysbios_family_arm_m3_Hwi_getStackInfo__E                              
1001b099  ti_sysbios_hal_Hwi_HwiProxy_getStackInfo__E                               
1001b099  ti_sysbios_hal_Hwi_HwiProxy_getStackInfo__E__mangled__                    
1001b099  ti_sysbios_hal_Hwi_getStackInfo__E                                        
1001b099  ti_sysbios_hal_Hwi_getStackInfo__E                                        
1001b0d9  ti_sysbios_knl_Task_yield__E                                              
1001b119  ti_sysbios_knl_Task_exit__E                                               
1001b153  ti_sysbios_gates_GateHwi_Instance_init__E                                 
1001b155  ti_sysbios_family_arm_m3_TaskSupport_start__E                             
1001b155  ti_sysbios_knl_Task_SupportProxy_start__E                                 
1001b155  ti_sysbios_knl_Task_SupportProxy_start__E__mangled__                      
1001b18d  ti_sysbios_heaps_HeapMem_Instance_init__E                                 
1001b1c5  ti_sysbios_knl_Clock_Instance_init__E                                     
1001b1fd  ti_sysbios_knl_Clock_create                                               
1001b235  ti_sysbios_heaps_HeapMem_init__I                                          
1001b269  ti_sysbios_knl_Clock_construct                                            
1001b29d  ClockP_getSystemTicks                                                     
1001b29d  ti_sysbios_knl_Clock_getTicks__E                                          
1001b2d1  ti_sysbios_knl_Semaphore_create                                           
1001b305  SwiP_restore                                                              
1001b305  ti_sysbios_knl_Swi_restore__E                                             
1001b339  ti_sysbios_knl_Task_blockI__E                                             
1001b36d  ti_sysbios_gates_GateMutex_Object__create__S                              
1001b39d  ti_sysbios_gates_GateMutex_create                                         
1001b3cd  ti_sysbios_gates_GateMutex_enter__E                                       
1001b3fd  ti_sysbios_heaps_HeapMem_free__E                                          
1001b42d  ti_sysbios_knl_Event_create                                               
1001b45d  ti_sysbios_knl_Semaphore_construct                                        
1001b48d  ti_sysbios_knl_Task_processVitalTaskFlag__I                               
1001b4bd  ti_sysbios_family_arm_cc26xx_Timer_postInit__I                            
1001b4e9  ti_sysbios_family_arm_cc26xx_Timer_startup__E                             
1001b4e9  ti_sysbios_knl_Clock_TimerProxy_startup__E                                
1001b4e9  ti_sysbios_knl_Clock_TimerProxy_startup__E__mangled__                     
1001b515  ti_sysbios_family_arm_m3_Hwi_Object__get__S                               
1001b541  ti_sysbios_gates_GateMutex_construct                                      
1001b56d  ti_sysbios_hal_Hwi_initStack                                              
1001b599  ti_sysbios_heaps_HeapMem_Object__create__S                                
1001b5c5  ti_sysbios_heaps_HeapMem_Object__get__S                                   
1001b5f1  ti_sysbios_knl_Event_construct                                            
1001b61d  ti_sysbios_knl_Event_pendTimeout__I                                       
1001b649  ti_sysbios_knl_Mailbox_Object__get__S                                     
1001b675  ti_sysbios_knl_Mailbox_postInit__I                                        
1001b6a1  ti_sysbios_knl_Queue_construct                                            
1001b6cd  ti_sysbios_knl_Queue_create                                               
1001b6f9  ti_sysbios_knl_Semaphore_pendTimeout__I                                   
1001b725  ti_sysbios_knl_Swi_Object__get__S                                         
1001b751  ti_sysbios_knl_Task_unblockI__E                                           
1001b77d  ti_sysbios_family_arm_cc26xx_TimestampProvider_get64__E                   
1001b77d  xdc_runtime_Timestamp_SupportProxy_get64__E                               
1001b77d  xdc_runtime_Timestamp_SupportProxy_get64__E__mangled__                    
1001b77d  xdc_runtime_Timestamp_get64__E                                            
1001b77d  xdc_runtime_Timestamp_get64__E                                            
1001b7a5  ti_sysbios_knl_Clock_addI__E                                              
1001b7cd  ti_sysbios_knl_Semaphore_Instance_finalize__E                             
1001b7f5  ti_sysbios_knl_Task_restore__E                                            
1001b81d  ti_sysbios_hal_Hwi_Instance_init__E                                       
1001b843  ti_sysbios_knl_Clock_logTick__E                                           
1001b845  ti_sysbios_family_arm_cc26xx_Timer_Module_startup__E                      
1001b869  ti_sysbios_gates_GateHwi_Object__create__S                                
1001b88d  ti_sysbios_BIOS_RtsGateProxy_Object__delete__S                            
1001b88d  ti_sysbios_gates_GateMutex_Object__delete__S                              
1001b88d  ti_sysbios_heaps_HeapMem_Module_GateProxy_Object__delete__S               
1001b8b1  ti_sysbios_knl_Clock_Object__delete__S                                    
1001b8d5  ti_sysbios_knl_Semaphore_Object__delete__S                                
1001b8f9  ti_sysbios_family_arm_cc26xx_Timer_Module__startupDone__S                 
1001b8f9  ti_sysbios_knl_Clock_TimerProxy_Module__startupDone__S                    
1001b8f9  ti_sysbios_knl_Clock_TimerProxy_Module__startupDone__S__mangled__         
1001b919  ti_sysbios_family_arm_cc26xx_TimestampProvider_Module_startup__E          
1001b939  ti_sysbios_family_arm_m3_Hwi_Module__startupDone__S                       
1001b939  ti_sysbios_hal_Hwi_HwiProxy_Module__startupDone__S                        
1001b939  ti_sysbios_hal_Hwi_HwiProxy_Module__startupDone__S__mangled__             
1001b959  ti_sysbios_family_arm_m3_Hwi_Object__delete__S                            
1001b959  ti_sysbios_hal_Hwi_HwiProxy_Object__delete__S                             
1001b979  ti_sysbios_family_arm_m3_Hwi_excHandler__I                                
1001b999  ti_sysbios_gates_GateHwi_Handle__label__S                                 
1001b999  xdc_runtime_Main_Module_GateProxy_Handle__label__S                        
1001b999  xdc_runtime_System_Module_GateProxy_Handle__label__S                      
1001b999  xdc_runtime_System_Module_GateProxy_Handle__label__S__mangled__           
1001b9b9  ti_sysbios_gates_GateHwi_Object__delete__S                                
1001b9b9  xdc_runtime_System_Module_GateProxy_Object__delete__S                     
1001b9d9  ti_sysbios_BIOS_RtsGateProxy_Handle__label__S                             
1001b9d9  ti_sysbios_BIOS_RtsGateProxy_Handle__label__S__mangled__                  
1001b9d9  ti_sysbios_gates_GateMutex_Handle__label__S                               
1001b9d9  ti_sysbios_heaps_HeapMem_Module_GateProxy_Handle__label__S                
1001b9d9  ti_sysbios_heaps_HeapMem_Module_GateProxy_Handle__label__S__mangled__     
1001b9f9  ti_sysbios_gates_GateMutex_Object__destruct__S                            
1001ba19  ti_sysbios_hal_Hwi_Object__delete__S                                      
1001ba39  ti_sysbios_heaps_HeapMem_Handle__label__S                                 
1001ba39  xdc_runtime_Memory_HeapProxy_Handle__label__S                             
1001ba39  xdc_runtime_Memory_HeapProxy_Handle__label__S__mangled__                  
1001ba59  ti_sysbios_heaps_HeapMem_Object__delete__S                                
1001ba59  xdc_runtime_Memory_HeapProxy_Object__delete__S                            
1001ba79  ti_sysbios_knl_Clock_Module_startup__E                                    
1001ba99  ti_sysbios_knl_Clock_Object__destruct__S                                  
1001bab9  ti_sysbios_knl_Clock_stop__E                                              
1001bad9  ti_sysbios_knl_Event_Object__delete__S                                    
1001baf9  ti_sysbios_knl_Event_checkEvents__I                                       
1001bb19  ti_sysbios_knl_Idle_run__E                                                
1001bb39  ti_sysbios_knl_Mailbox_Object__delete__S                                  
1001bb59  ti_sysbios_knl_Queue_Object__delete__S                                    
1001bb79  ti_sysbios_knl_Queue_Object__get__S                                       
1001bb99  ti_sysbios_knl_Semaphore_Object__destruct__S                              
1001bbb9  ti_sysbios_knl_Swi_Object__delete__S                                      
1001bbd9  ti_sysbios_knl_Task_Object__delete__S                                     
1001bbf9  ti_sysbios_knl_Task_Object__get__S                                        
1001bc19  ti_sysbios_knl_Task_restoreHwi__E                                         
1001bc39  ti_sysbios_family_arm_m3_Hwi_Object__destruct__S                          
1001bc55  ti_sysbios_family_arm_m3_Hwi_setPriority__E                               
1001bc71  ti_sysbios_gates_GateMutex_Instance_init__E                               
1001bc8d  ti_sysbios_hal_Hwi_HwiProxy_create                                        
1001bca9  ti_sysbios_knl_Clock_scheduleNextTick__E                                  
1001bcc5  ti_sysbios_knl_Event_Object__destruct__S                                  
1001bce1  ti_sysbios_knl_Mailbox_Object__destruct__S                                
1001bcfd  ti_sysbios_knl_Queue_Object__destruct__S                                  
1001bd19  ti_sysbios_knl_Queue_get__E                                               
1001bd35  ti_sysbios_knl_Queue_put__E                                               
1001bd51  ti_sysbios_knl_Swi_Object__destruct__S                                    
1001bd6d  ti_sysbios_knl_Task_Object__destruct__S                                   
1001bd89  ti_sysbios_knl_Task_enter__I                                              
1001bda5  ti_sysbios_knl_Task_sleepTimeout__I                                       
1001bdbf  ti_sysbios_knl_Clock_triggerFunc__I                                       
1001bdc1  ti_sysbios_family_arm_m3_Hwi_plug__E                                      
1001bdd9  ti_sysbios_gates_GateMutex_leave__E                                       
1001bdf1  ti_sysbios_knl_Task_unblock__E                                            
1001be09  ti_sysbios_knl_Clock_Instance_finalize__E                                 
1001be1f  ti_sysbios_knl_Clock_start__E                                             
1001be35  ti_sysbios_family_arm_m3_Hwi_switchFromBootStack__E                       
1001be35  ti_sysbios_hal_Hwi_HwiProxy_switchFromBootStack__E                        
1001be35  ti_sysbios_hal_Hwi_HwiProxy_switchFromBootStack__E__mangled__             
1001be35  ti_sysbios_hal_Hwi_switchFromBootStack__E                                 
1001be35  ti_sysbios_hal_Hwi_switchFromBootStack__E                                 
1001be49  ti_sysbios_knl_Event_Instance_init__E                                     
1001be5d  ti_sysbios_hal_Hwi_Module_startup__E                                      
1001be6f  ti_sysbios_knl_Event_sync__E                                              
1001be81  ti_sysbios_BIOS_exit__E                                                   
1001be91  ti_sysbios_BIOS_getCpuFreq__E                                             
1001bea1  ti_sysbios_BIOS_setThreadType__E                                          
1001beb1  ti_sysbios_BIOS_start__E                                                  
1001bec1  ti_sysbios_gates_GateMutex_Instance_finalize__E                           
1001bed1  ti_sysbios_hal_Hwi_HwiProxy_Object__create__S                             
1001bee1  ti_sysbios_knl_Clock_TimerProxy_getCurrentTick__E                         
1001bef1  ti_sysbios_knl_Clock_TimerProxy_getMaxTicks__E                            
1001bf01  ti_sysbios_knl_Clock_TimerProxy_setNextTick__E                            
1001bf11  ti_sysbios_knl_Swi_disable__E                                             
1001bf21  ti_sysbios_knl_Swi_enabled__E                                             
1001bf31  ti_sysbios_knl_Task_disable__E                                            
1001bf41  ti_sysbios_heaps_HeapMem_restore__E                                       
1001bf4f  ti_sysbios_knl_Queue_empty__E                                             
1001bf5d  ti_sysbios_knl_Queue_remove__E                                            
1001bf6b  ti_sysbios_family_arm_cc26xx_TimestampProvider_getFreq__E                 
1001bf6b  xdc_runtime_Timestamp_SupportProxy_getFreq__E                             
1001bf6b  xdc_runtime_Timestamp_SupportProxy_getFreq__E__mangled__                  
1001bf6b  xdc_runtime_Timestamp_getFreq__E                                          
1001bf6b  xdc_runtime_Timestamp_getFreq__E                                          
1001bf77  ti_sysbios_knl_Swi_Instance_finalize__E                                   
1001bf79  ti_sysbios_family_arm_m3_Hwi_Params__init__S                              
1001bf79  ti_sysbios_hal_Hwi_HwiProxy_Params__init__S                               
1001bf79  ti_sysbios_hal_Hwi_HwiProxy_Params__init__S__mangled__                    
1001bf85  ti_sysbios_family_arm_m3_Hwi_disableFxn__E                                
1001bf91  ti_sysbios_family_arm_m3_Hwi_enableFxn__E                                 
1001bf9d  ti_sysbios_family_arm_m3_TaskSupport_getStackAlignment__E                 
1001bf9d  ti_sysbios_knl_Task_SupportProxy_getStackAlignment__E                     
1001bf9d  ti_sysbios_knl_Task_SupportProxy_getStackAlignment__E__mangled__          
1001bfa9  ti_sysbios_gates_GateHwi_enter__E                                         
1001bfb5  ti_sysbios_BIOS_RtsGateProxy_Params__init__S                              
1001bfb5  ti_sysbios_BIOS_RtsGateProxy_Params__init__S__mangled__                   
1001bfb5  ti_sysbios_gates_GateMutex_Params__init__S                                
1001bfb5  ti_sysbios_heaps_HeapMem_Module_GateProxy_Params__init__S                 
1001bfb5  ti_sysbios_heaps_HeapMem_Module_GateProxy_Params__init__S__mangled__      
1001bfc1  ti_sysbios_knl_Clock_Params__init__S                                      
1001bfcd  ti_sysbios_knl_Clock_getTimerHandle__E                                    
1001bfd9  ti_sysbios_knl_Event_Params__init__S                                      
1001bfe5  ti_sysbios_knl_Mailbox_Params__init__S                                    
1001bff1  ti_sysbios_knl_Queue_dequeue__E                                           
1001bffd  ti_sysbios_knl_Queue_enqueue__E                                           
1001c009  ti_sysbios_knl_Semaphore_Params__init__S                                  
1001c015  ti_sysbios_knl_Swi_Params__init__S                                        
1001c021  ti_sysbios_knl_Task_Params__init__S                                       
1001c02d  ti_sysbios_knl_Task_self__E                                               
1001c039  ti_sysbios_hal_Hwi_Instance_finalize__E                                   
1001c043  ti_sysbios_family_arm_m3_Hwi_doSwiRestore__I                              
1001c04b  ti_sysbios_family_arm_m3_Hwi_startup__E                                   
1001c04b  ti_sysbios_hal_Hwi_HwiProxy_startup__E                                    
1001c04b  ti_sysbios_hal_Hwi_HwiProxy_startup__E__mangled__                         
1001c04b  ti_sysbios_hal_Hwi_startup__E                                             
1001c04b  ti_sysbios_hal_Hwi_startup__E                                             
1001c053  ti_sysbios_knl_Idle_loop__E                                               
1001c05b  ti_sysbios_family_arm_m3_Hwi_doTaskRestore__I                             
1001c061  HwiP_restore                                                              
1001c061  ti_sysbios_family_arm_m3_Hwi_restoreFxn__E                                
1001c067  ti_sysbios_gates_GateHwi_leave__E                                         
1001c06d  ti_sysbios_heaps_HeapMem_isBlocking__E                                    
1001c073  ti_sysbios_knl_Queue_Instance_init__E                                     
1001c079  ti_sysbios_knl_Queue_elemClear__E                                         
1001c07f  ti_sysbios_knl_Swi_Module_startup__E                                      
1001c085  ti_sysbios_knl_Swi_startup__E                                             
1001c08b  ti_sysbios_knl_Task_enable__E                                             
1001c091  ti_sysbios_BIOS_RtsGateProxy_enter__E                                     
1001c095  ti_sysbios_BIOS_RtsGateProxy_leave__E                                     
1001c099  ti_sysbios_family_arm_cc26xx_Timer_getExpiredTicks__E                     
1001c09d  ti_sysbios_family_arm_cc26xx_Timer_getPeriod__E                           
1001c0a1  ti_sysbios_family_arm_cc26xx_Timer_setPeriod__E                           
1001c0a5  ti_sysbios_family_arm_m3_Hwi_delete                                       
1001c0a9  ti_sysbios_family_arm_m3_Hwi_destruct                                     
1001c0ad  ti_sysbios_family_arm_m3_TaskSupport_Module__startupDone__S               
1001c0ad  ti_sysbios_knl_Task_SupportProxy_Module__startupDone__S                   
1001c0ad  ti_sysbios_knl_Task_SupportProxy_Module__startupDone__S__mangled__        
1001c0b1  ti_sysbios_gates_GateHwi_query__E                                         
1001c0b1  xdc_runtime_Main_Module_GateProxy_query__E                                
1001c0b1  xdc_runtime_System_Module_GateProxy_query__E                              
1001c0b1  xdc_runtime_System_Module_GateProxy_query__E__mangled__                   
1001c0b5  ti_sysbios_gates_GateMutex_delete                                         
1001c0b9  ti_sysbios_gates_GateMutex_destruct                                       
1001c0bd  ti_sysbios_BIOS_RtsGateProxy_query__E                                     
1001c0bd  ti_sysbios_BIOS_RtsGateProxy_query__E__mangled__                          
1001c0bd  ti_sysbios_gates_GateMutex_query__E                                       
1001c0bd  ti_sysbios_heaps_HeapMem_Module_GateProxy_query__E                        
1001c0bd  ti_sysbios_heaps_HeapMem_Module_GateProxy_query__E__mangled__             
1001c0c1  ti_sysbios_hal_Hwi_HwiProxy_delete                                        
1001c0c5  ti_sysbios_hal_Hwi_delete                                                 
1001c0c9  ti_sysbios_heaps_HeapMem_Module_GateProxy_enter__E                        
1001c0cd  ti_sysbios_heaps_HeapMem_Module_GateProxy_leave__E                        
1001c0d1  ti_sysbios_knl_Clock_TimerProxy_getExpiredTicks__E                        
1001c0d5  ti_sysbios_knl_Clock_TimerProxy_getPeriod__E                              
1001c0d9  ti_sysbios_knl_Clock_delete                                               
1001c0dd  ti_sysbios_knl_Clock_destruct                                             
1001c0e1  ti_sysbios_knl_Clock_removeI__E                                           
1001c0e5  ti_sysbios_knl_Clock_setTimeout__E                                        
1001c0e9  ti_sysbios_knl_Event_delete                                               
1001c0ed  ti_sysbios_knl_Event_destruct                                             
1001c0f1  ti_sysbios_knl_Mailbox_delete                                             
1001c0f5  ti_sysbios_knl_Mailbox_destruct                                           
1001c0f9  ti_sysbios_knl_Queue_delete                                               
1001c0fd  ti_sysbios_knl_Queue_destruct                                             
1001c101  ti_sysbios_knl_Queue_head__E                                              
1001c105  ti_sysbios_knl_Queue_next__E                                              
1001c109  ti_sysbios_knl_Semaphore_delete                                           
1001c10d  ti_sysbios_knl_Semaphore_destruct                                         
1001c111  ti_sysbios_knl_Swi_delete                                                 
1001c115  ti_sysbios_knl_Swi_destruct                                               
1001c119  ti_sysbios_knl_Swi_postInit__I                                            
1001c11d  ti_sysbios_knl_Task_delete                                                
1001c121  ti_sysbios_knl_Task_destruct                                              
1001c125  ti_sysbios_knl_Task_startup__E                                            
1001c129  xdc_runtime_Startup_startMods__I                                          
1001c2c9  xdc_runtime_Core_createObject__I                                          
1001c349  xdc_runtime_Memory_alloc__E                                               
1001c3b5  xdc_runtime_Core_deleteObject__I                                          
1001c413  xdc_runtime_Error_policySpin__E                                           
1001c415  xdc_runtime_Startup_exec__E                                               
1001c465  xdc_runtime_Assert_raise__I                                               
1001c4ad  xdc_runtime_Core_assignParams__I                                          
1001c4f5  xdc_runtime_Core_constructObject__I                                       
1001c581  xdc_runtime_System_atexit__E                                              
1001c5b9  xdc_runtime_Core_assignLabel__I                                           
1001c5ed  xdc_runtime_System_processAtExit__E                                       
1001c621  xdc_runtime_Text_cordText__E                                              
1001c64d  xdc_runtime_System_abort__E                                               
1001c66d  xdc_runtime_Error_raiseX__E                                               
1001c689  xdc_runtime_Memory_valloc__E                                              
1001c6a5  xdc_runtime_Core_destructObject__I                                        
1001c6bd  xdc_runtime_Error_check__E                                                
1001c6d5  xdc_runtime_System_exit__E                                                
1001c6ed  xdc_runtime_Text_ropeText__E                                              
1001c705  xdc_runtime_Memory_free__E                                                
1001c715  xdc_runtime_SysCallback_abort__E                                          
1001c725  xdc_runtime_SysCallback_exit__E                                           
1001c735  xdc_runtime_Timestamp_SupportProxy_get32__E                               
1001c735  xdc_runtime_Timestamp_get32__E                                            
1001c735  xdc_runtime_Timestamp_get32__E                                            
1001c751  xdc_runtime_Memory_calloc__E                                              
1001c75d  xdc_runtime_Memory_getMaxDefaultTypeAlign__E                              
1001c769  xdc_runtime_Startup_rtsDone__E                                            
1001c775  xdc_runtime_Memory_HeapProxy_alloc__E                                     
1001c77f  xdc_runtime_Memory_HeapProxy_free__E                                      
1001c789  xdc_runtime_Gate_leaveSystem__E                                           
1001c78f  xdc_runtime_System_Module_startup__E                                      
1001c795  xdc_runtime_Gate_enterSystem__E                                           
1001c799  xdc_runtime_System_Module_GateProxy_enter__E                              
1001c79d  xdc_runtime_System_Module_GateProxy_leave__E                              
1001c7a1  xdc_runtime_System_abortSpin__E                                           
1001c7a3  xdc_runtime_System_exitSpin__E                                            
1001c7a5  ti_sysbios_family_arm_m3_Hwi_dispatch__I                                  
1001c86d  ti_sysbios_family_arm_m3_TaskSupport_buildTaskStack                       
1001c8b9  ti_sysbios_family_arm_m3_Hwi_initStacks__E                                
1001c901  ti_sysbios_family_arm_m3_Hwi_excHandlerAsm__I                             
1001c921  ti_sysbios_family_xxx_Hwi_switchAndRunFunc                                
1001c93f  ti_sysbios_family_arm_m3_Hwi_pendSV__I                                    
1001c957  ti_sysbios_family_arm_m3_Hwi_return                                       
1001c959  ti_sysbios_family_arm_m3_TaskSupport_glue                                 
1001c969  ti_sysbios_family_arm_m3_TaskSupport_swap__E                              
1001c969  ti_sysbios_knl_Task_SupportProxy_swap__E                                  
1001c969  ti_sysbios_knl_Task_SupportProxy_swap__E__mangled__                       
1001c971  ti_sysbios_knl_Task_swapReturn                                            
1001c978  ti_sysbios_knl_Task_Object__PARAMS__C                                     
1001c9b4  ti_sysbios_knl_Mailbox_Object__PARAMS__C                                  
1001c9e8  ti_sysbios_family_arm_m3_Hwi_Object__PARAMS__C                            
1001ca18  ti_sysbios_hal_Hwi_Object__PARAMS__C                                      
1001ca44  ti_sysbios_knl_Swi_Object__PARAMS__C                                      
1001ca6c  ti_sysbios_heaps_HeapMem_Object__PARAMS__C                                
1001ca90  ti_sysbios_knl_Clock_Object__PARAMS__C                                    
1001cab4  ti_sysbios_knl_Semaphore_Object__PARAMS__C                                
1001cad8  ti_sysbios_gates_GateHwi_Object__PARAMS__C                                
1001caf0  ti_sysbios_gates_GateMutex_Object__PARAMS__C                              
1001cb08  ti_sysbios_knl_Event_Object__PARAMS__C                                    
1001cb20  ti_sysbios_knl_Queue_Object__PARAMS__C                                    
1001cb68  ti_sysbios_gates_GateMutex_Instance_State_sem__O                          
1001cb6c  ti_sysbios_knl_Clock_Module_State_clockQ__O                               
1001cb70  ti_sysbios_knl_Event_Instance_State_pendQ__O                              
1001cb74  ti_sysbios_knl_Mailbox_Instance_State_dataQue__O                          
1001cb78  ti_sysbios_knl_Mailbox_Instance_State_dataSem__O                          
1001cb7c  ti_sysbios_knl_Mailbox_Instance_State_freeQue__O                          
1001cb80  ti_sysbios_knl_Mailbox_Instance_State_freeSem__O                          
1001cb84  ti_sysbios_knl_Semaphore_Instance_State_pendQ__O                          
1001cb88  ti_sysbios_knl_Task_Module_State_inactiveQ__O                             
20000000  ti_sysbios_family_arm_m3_Hwi_ramVectors                                   
20000100  ti_sysbios_knl_Task_Module__state__V                                      
20000144  ti_sysbios_family_arm_m3_Hwi_Module__state__V                             
20000178  ti_sysbios_knl_Clock_Module__state__V                                     
200001a4  ti_sysbios_BIOS_Module__state__V                                          
200001c8  ti_sysbios_knl_Swi_Module__state__V                                       
200001e4  ti_sysbios_family_arm_cc26xx_Timer_Module__state__V                       
200001ec  ti_sysbios_family_arm_cc26xx_TimestampProvider_Module__state__V           
200001f0  xdc_runtime_Startup_Module__state__V                                      
200001f8  xdc_runtime_System_Module__state__V                                       
20000200  xdc_runtime_Memory_Module__state__V                                       
20000204  xdc_runtime_Error_Module__state__V                                        
20000208  ti_sysbios_heaps_HeapMem_Instance_State_0_buf__A                          
20000a08  myTaskStack                                                               
20000e08  myTaskStack1                                                              
20001208  ti_sysbios_knl_Task_Instance_State_0_stack__A                             
20001408  xdc_runtime_SysMin_Module_State_0_outbuf__A                               
200015fc  uartCC26XXObjects                                                         
20001728  __CIOBUF_                                                                 
20001848  ti_sysbios_family_arm_m3_Hwi_dispatchTable                                
20001910  myTask                                                                    
20001960  myTask1                                                                   
200019e0  uartCC26XXRingBuffer                                                      
20001a68  PowerCC26XX_taskKey                                                       
20001a6c  PowerCC26XX_swiKey                                                        
20001a78  parmbuf                                                                   
20001a80  ClockP_tickPeriod                                                         
20001a84  uart                                                                      
20001a8a  driverlib_release_0_49664                                                 
20001a90  pinUpperBound                                                             
20001a94  pinLowerBound                                                             
20001b28  pinHandleTable                                                            
20001ba4  PowerCC26XX_module                                                        
20001cb8  ti_sysbios_knl_Swi_Module_State_0_readyQ__A                               
20001d8c  ti_sysbios_knl_Task_Object__table__V                                      
20001dd8  ti_sysbios_family_arm_cc26xx_Timer_Object__table__V                       
20001e20  ti_sysbios_gates_GateMutex_Object__table__V                               
20001e58  ti_sysbios_knl_Swi_Object__table__V                                       
20001e88  ti_sysbios_knl_Clock_Object__table__V                                     
20001ea8  ti_sysbios_knl_Task_Module_State_0_readyQ__A                              
20001ec8  xdc_runtime_Error_IgnoreBlock                                             
20001ee8  ti_sysbios_family_arm_m3_Hwi_Object__table__V                             
20001f00  ti_sysbios_heaps_HeapMem_Object__table__V                                 
20001f18  gpioPinConfigs                                                            
20001f38  xdc_runtime_SysMin_Module__state__V                                       
20001f44  _lock                                                                     
20001f48  _unlock                                                                   
20001f4c  gpioCallbackFunctions                                                     
20001f54  ti_sysbios_family_arm_m3_Hwi_Module__root__V                              
20001f5c  ti_sysbios_gates_GateHwi_Module__root__V                                  
20001f64  ti_sysbios_gates_GateMutex_Module__root__V                                
20001f6c  ti_sysbios_hal_Hwi_Module__root__V                                        
20001f74  ti_sysbios_heaps_HeapMem_Module__root__V                                  
20001f7c  ti_sysbios_knl_Clock_Module__root__V                                      
20001f84  ti_sysbios_knl_Event_Module__root__V                                      
20001f8c  ti_sysbios_knl_Mailbox_Module__root__V                                    
20001f94  ti_sysbios_knl_Queue_Module__root__V                                      
20001f9c  ti_sysbios_knl_Semaphore_Module__root__V                                  
20001fa4  ti_sysbios_knl_Swi_Module__root__V                                        
20001fac  ti_sysbios_knl_Task_Module__root__V                                       
20001fb4  xdc_runtime_System_Module_State_0_atexitHandlers__A                       
20001fbc  main_func_sp                                                              
20001fc0  ti_sysbios_family_arm_m3_Hwi_Module_State_0_excContext__A                 
20001fc4  ti_sysbios_family_arm_m3_Hwi_Module_State_0_excStack__A                   
20001fc8  ti_sysbios_knl_Task_Module_State_0_idleTask__A                            
20001fcc  ti_sysbios_family_arm_m3_Hwi_Module_State_0_excActive__A                  
20004d00  __stack                                                                   
20005000  __STACK_END                                                               
20005000  __STACK_TOP                                                               
e000e000  ti_sysbios_family_arm_m3_Hwi_nvic                                         
ffffffff  __TI_pprof_out_hndl                                                       
ffffffff  __TI_prof_data_size                                                       
ffffffff  __TI_prof_data_start                                                      
ffffffff  __binit__                                                                 
ffffffff  __c_args__                                                                
ffffffff  binit                                                                     
UNDEFED   SHT$$INIT_ARRAY$$Base                                                     
UNDEFED   SHT$$INIT_ARRAY$$Limit                                                    

[816 symbols]
